:100000000C94E5160C9416170C9416170C941617EE
:100010000C9416170C9416170C9416170C941617AC
:100020000C9416170C9416170C9416170C9416179C
:100030000C9416170C945A4A0C9416170C94161715
:100040000C9416170C9490940C9416170C94161785
:100050000C9416170C9416170C94364C0C944C7A7E
:100060000C9416170C944F450C9416170C941617F5
:100070000C9416170C9416170C9416170C9416174C
:100080000C9428C80C9416170C9416170C94161779
:100090000C9416170C9416170C9416170C9416172C
:1000A0000C9416170C9416170C94FBC70C94161787
:1000B0000C9416170C9416170C9416170C94CEC7A4
:1000C0000C9416170C9416170C9416170C941617FC
:1000D0000C9416170C9416170C9461490C94224931
:1000E0000C941617CE31EB311C3239324E32773246
:1000F000E6324C33F933F6360437FD3638373C37C1
:100100004D37B43B6237AE37E03707383038853883
:100110009638A738B838C938DA38B43B303AB43BE7
:100120003B3A203B343B603BB8B5BBB5AAB5AEB556
:10013000B4B5F2B5BFB5C3B5C9B5CDB5D1B5D7B5B1
:10014000DBB5DFB5F2B5E5B5E9B5EDB596BA9BBA65
:10015000A0BAAABAB4BA2DBBBEBAC6BACEBAD8BA79
:10016000E2BAECBAFBBA05BB2DBB0FBB19BB23BB74
:10017000084AD73B3BCE016E84BCBFFDC12F3D6C0E
:1001800074319ABD56833DDA3D00C77F11BED9E474
:10019000BB4C3E916BAAAABE000000803F05A84C54
:1001A000CDB2D44EB93836A9020C50B99186880820
:1001B0003CA6AAAA2ABE000000803F004E414E493C
:1001C0004E495459494E46CDCCCC3D0AD7233C1715
:1001D000B7D13877CC2B329595E6241FB14F0A0062
:1001E0000020410000C84200401C4620BCBE4CCA52
:1001F0001B0E5AAEC59D74434F4D4D554E4943415C
:1002000054494F4E0044525952554E004552524F98
:10021000525300494E464F004543484F0047322F46
:1002200047332062616420706172616D657465722C
:10023000730A00205A3A200020593A20004265648F
:1002400020583A20004D65736820706F696E7420E5
:1002500063616E6E6F74206265207265736F6C7679
:1002600065640A00456E642066696C65206C69737C
:10027000740A00426567696E2066696C65206C6966
:1002800073740A00286E6F2066696C6529005344F8
:10029000207072696E74696E6720627974652000DF
:1002A0004E6F74205344207072696E74696E670AD1
:1002B0000043757272656E742066696C653A200041
:1002C0002569730025696D202569730025696820FB
:1002D00025696D20256973002569642025696820DA
:1002E00025696D20256973002569792025696420B9
:1002F0002569682025696D20256973005072696E33
:10030000742074696D653A2000180213020C02050E
:1003100002F7016F66660044454255473A004B4973
:100320004C4C45442E20004D3131332053006F6B2F
:10033000002C20002C2000544845524D414C5F5069
:10034000524F54454354494F4E004155544F524526
:10035000504F52545F53445F5354415455530045DA
:100360004D455247454E43595F5041525345520007
:10037000434153455F4C494748545F4252494748BF
:10038000544E45535300544F47474C455F4C4947E3
:1003900048545300534F4654574152455F504F57AE
:1003A0004552004255494C445F50455243454E54D6
:1003B000004C4556454C494E475F44415441005A14
:1003C0005F50524F4245004155544F4C4556454CA5
:1003D000005052494E545F4A4F420050524F4752CC
:1003E000455353004155544F5245504F52545F545A
:1003F000454D5000564F4C554D45545249430045CC
:100400004550524F4D0053455249414C5F584F4E55
:100410005F584F4646004649524D574152455F4E40
:10042000414D453A4D61726C696E20312E312E3945
:1004300020284769746875622920534F55524345F7
:100440005F434F44455F55524C3A68747470733A39
:100450002F2F6769746875622E636F6D2F4D6172FF
:100460006C696E4669726D776172652F4D61726C51
:10047000696E2050524F544F434F4C5F5645525374
:10048000494F4E3A312E30204D414348494E455F49
:10049000545950453A3344205072696E7465722045
:1004A00045585452554445525F434F554E543A3186
:1004B00020555549443A33646135396339392D3112
:1004C0003832302D343436342D616166332D363573
:1004D000346539353364363362340A002F2F2000F7
:1004E000205400205200416363656C657261746939
:1004F0006F6E3A205000546F6F20666172206672F2
:100500006F6D207265666572656E636520706F69D8
:100510006E740A0020466C6F773A2000000136376F
:1005200026032BFFFFFF3C3D382AFFFFFFFF2E3045
:100530003E12FFFFFFFFFF02FF0809FF2C071A1CF6
:1005400018FFFFFF08440A2C4324221E206F7574F5
:10055000206F662072616E67650A00536572766F60
:1005600020003A200020536572766F200043290A4C
:100570000061626C656420286D696E2074656D7021
:100580002000436F6C642065787472756465732015
:10059000617265200020643A0020693A0020703AB8
:1005A000004E6F2063617365206C696768740A0090
:1005B0004D65736820706F696E742063616E6E6F35
:1005C00074206265207265736F6C7665640A004DF5
:1005D00034323120696E636F7272656374207061AA
:1005E00072616D657465722075736167650A004597
:1005F0004550524F4D204F4B0A00205A0044756120
:100600006C20456E6473746F702041646A757374F6
:100610006D656E7420286D6D293A20003F5A206F59
:100620007574206F662072616E676520282D3230E8
:1006300020746F203230290A003A200050726F6215
:1006400065205A204F6666736574003F4B207661C3
:100650006C7565206F7574206F662072616E6765BA
:100660002028302D3130292E0A00416476616E63D6
:1006700065204B3D0041637469766520457874724E
:10068000756465723A2000496E76616C6964206514
:10069000787472756465720A0043616E6E6F7420BF
:1006A000656E746572207375626469723A20004DDC
:1006B000353031005370656369616C204D656E752E
:1006C0003A205265616420454550524F4D0A004D15
:1006D000353030005370656369616C204D656E750F
:1006E0003A205361766520454550524F4D0A0047E8
:1006F00032380A473239005370656369616C204DA6
:10070000656E753A204175746F20426564204C65B2
:1007100076656C696E670A004D33303320433820AC
:1007200053323030005370656369616C204D656EE3
:10073000753A204175746F2054756E652050494498
:100740000A003C5370656369616C5F4D656E753E70
:10075000003C5370656369616C5F4D656E753E006A
:100760002F002F002F002F2E2E0A002F2E2E002FAD
:100770002E2E003C5370656369616C5F4D656E752C
:100780003E0A003C5370656369616C204D656E756F
:100790003E003C5370656369616C204D656E753E2B
:1007A000003C5265616420454550524F4D3E003C2F
:1007B0005265616420454550524F4D3E003C5361A7
:1007C000766520454550524F4D3E003C536176655D
:1007D00020454550524F4D3E003C4175746F2042BC
:1007E0006564204C6576656C696E673E003C4175BA
:1007F000746F20426564204C6576656C696E673E57
:10080000003C4175746F2054756E6520486F7465A7
:100810006E64205049443E003C4175746F2054750D
:100820006E6520486F74656E64205049443E003CFC
:10083000457869743E003C457869743E0056313114
:1008400036004A333320004D3530300A4D343230D3
:100850002053310A4731205A313020463234300A91
:10086000473120583020593020463630303000543F
:100870004654204C6576656C20736176696E6720FE
:10088000646174612E2E2E0A004D353030004D38D3
:100890003531205A003E0A00413956200054465452
:1008A0002073656E64696E672063757272656E741D
:1008B000207A2D70726F6265206F66667365742092
:1008C000646174612E2E2E203C0041395620005464
:1008D00046542053657269616C2044656275673ABD
:1008E000204C6576656C696E67207072696E742045
:1008F0007465737420776974682068656174696EC3
:100900006720646F6E652E2E2E204A32320A004A0E
:10091000323200544654204C6576656C206368651D
:10092000636B2068656174696E672E2E2E0A005411
:1009300046542053657269616C2044656275673A5C
:10094000204C6576656C696E67207072696E7420E4
:100950007465737420646F6E652E2E2E204A3232B9
:100960000A004A323200544654204C6576656C20A9
:10097000636865636B206E6F2068656174696E677C
:100980002E2E2E0A004731205A3520463234300AA6
:1009900047312058313930205932302046363030F6
:1009A000300A4731205A3020463234300054465401
:1009B000204C6576656C20636865636B706F696E4B
:1009C00074206261636B2072696768742E2E2E0A30
:1009D000004731205A3520463234300A47312058FA
:1009E00031393020593139302046363030300A47DD
:1009F00031205A30204632343000544654204C6561
:100A000076656C20636865636B706F696E742062D5
:100A100061636B2072696768742E2E2E0A0047315D
:100A2000205A3520463234300A4731205831393087
:100A3000205932302046363030300A4731205A3083
:100A4000204632343000544654204C6576656C2084
:100A5000636865636B706F696E742066726F6E7425
:100A60002072696768742E2E2E0A004739310A47B2
:100A700031205A313020463234300A4739300A4763
:100A800032380A4732390A47312058323020593239
:100A9000302046363030300A4731205A3020463236
:100AA000343000544654204C6576656C696E67207E
:100AB0007374617274656420616E64206D6F766911
:100AC0006E7420746F2066726F6E74206C6566742D
:100AD0002E2E2E0A0054465420456E746572696E9F
:100AE00067206C6576656C206D656E75652E2E2EA3
:100AF0000A005446542053657269616C2044656253
:100B000075673A205344206361726420696E69748A
:100B100069616C697A65642E2E2E204A30320A0093
:100B20004A3032005446542053657269616C204447
:100B3000656275673A20436F6F6C696E6720646FFA
:100B4000776E2E2E2E204A31320A004A313200476B
:100B500031205A3130004F4B004731205A3130009C
:100B60004739300047312045256946353030004748
:100B70003120452D302E3146256900473120453042
:100B80002E31462569004731205A256946256900DE
:100B90004731205A2D302E31462569004731205AE1
:100BA000302E31462569004731205925694625698F
:100BB00000473120592D302E31462569004731201C
:100BC00059302E3146256900473120582569462580
:100BD0006900473120582D302E31462569004731B4
:100BE0002058302E314625690047393100473238C8
:100BF00000473238205A00473238205900473238EF
:100C00002058004132305620004731205A31300000
:100C10005446542053657269616C2044656275675F
:100C20003A205374617274696E6720534420507285
:100C3000696E742E2E2E204A30340A004A30340059
:100C40005446542053657269616C2044656275672F
:100C50003A2046696C65206F70656E206661696C2C
:100C600065642E2E2E204A32310A004A3231005459
:100C700046542053657269616C2044656275673A19
:100C80002046696C65206F70656E207375636365BF
:100C9000737366756C2E2E2E204A32300A004A324B
:100CA00030004B494C4C45442E20005446542053B0
:100CB000657269616C2044656275673A205344200F
:100CC0007072696E7420737461727465642E2E2E56
:100CD000204A30340A004A303400454E4400464E23
:100CE00020004A3032003939393A393939004D005B
:100CF00048004137562000413656202D2D2D004A00
:100D000030320041365620005A3A2000593A20002D
:100D1000583A2000413556004134562000413356A0
:100D200020004132562000413156200041305620EB
:100D3000005446542053657269616C20436F6D6D99
:100D4000616E643A20004D38340054465420536597
:100D50007269616C2044656275673A205344207063
:100D600072696E742073746F707065642E2E2E20FD
:100D70004A31360A004A31360054465420536572CF
:100D800069616C2044656275673A20534420707233
:100D9000696E742070617573656420646F6E652E72
:100DA0002E2E204A31380A004A3138004739310A9C
:100DB0004731205A313020463234300A473930002A
:100DC0005446542053657269616C204465627567AE
:100DD0003A205344207072696E7420646F6E652EE1
:100DE0002E2E204A31340A004A3134005446542011
:100DF00053657269616C2044656275673A2053449B
:100E0000206361726420696E7365727465642E2E4E
:100E10002E204A30300A004A3030005446542053C5
:100E2000657269616C2044656275673A205344209D
:100E3000636172642072656D6F7665642E2E2E205C
:100E40004A30310A004A303100544654205365720A
:100E500069616C2044656275673A20486F74656EFD
:100E6000642074656D70657261747572652061626D
:100E70006E6F726D616C2E2E2E204A32300A004A3F
:100E80003130003D003F2061646472657373203A25
:100E90002000206279746573206F66206D656D6F28
:100EA000727920696E697469616C697A65642E0A69
:100EB0000A00556E61626C6520746F20696E6974FA
:100EC00069616C697A652E0A0A00496E6974696104
:100ED0006C697A696E672066726565206D656D6FF5
:100EE000727920626C6F636B2E0A0A0A0074727545
:100EF000650A002072657475726E3D000A4D656D5D
:100F00006F727920436F7272757074696F6E2064AE
:100F10006574656374656420696E2066726565201A
:100F20006D656D6F727920617265612E0A002020F7
:100F3000626C6F636B5F666F756E643D002020208E
:100F4000002920666F756E643D00202800207370B4
:100F5000203C204865617020002073703D000A5FCE
:100F60005F6273735F656E643A20003D000A265F1E
:100F70005F62726B76616C3A20000A666D632829A5
:100F8000206E3D00636865636B5F666F725F6672BB
:100F900065655F6D656D6F72795F636F7272757095
:100FA00074696F6E2829203D200020627974657372
:100FB00020617420000A4C61726765737420667248
:100FC000656520626C6F636B20697320000A4D6554
:100FD0006D6F727920436F7272757074696F6E20D5
:100FE000646574656374656420696E206672656506
:100FF000206D656D6F727920617265612E0A002027
:10100000627974657320667265652061742000469C
:101010006F756E6420000A436F7272757074696E2A
:101020006720616464726573733A2000436F727263
:10103000757074696E672066726565206D656D6F89
:10104000727920626C6F636B2E0A0A000A53746116
:10105000636B20506F696E746572203A20000A73CA
:1010600074617274206F66206672656520737061AA
:101070006365203A20000A5F5F6273735F656E6488
:10108000203A20000A5F5F62726B76616C203A2022
:10109000001000C90210012C01400122017001184A
:1010A00001B0010E01F00104015002FA00B002F09B
:1010B000003003E600D003DC009004D2007005C8C5
:1010C00000A006BE000008B400B009AA00D00BA022
:1010D00000600E960060118C0000158200201978C7
:1010E00000C01D6E00A0226400B0275A00902C5052
:1010F0000000314600E0343C0010383200903A28BD
:1011000000603C1E00A03D1400803E0A00203F000D
:10111000002CFFFFFFFFFF00010101010162656478
:101120000A002C2073797374656D2073746F70706E
:10113000656421204865617465725F49443A200006
:101140004265642068656174696E67206661696CD8
:1011500065640048656174696E67206661696C65E5
:10116000640045312048656174696E672066616975
:101170006C65640048656174696E67206661696CBE
:1011800065640070012C0190012701B0012201C0AB
:10119000011D01F00118011002130130020E01605F
:1011A00002090190020401C002FF000003FA00409E
:1011B00003F5008003F000D003EB002004E600708C
:1011C00004E100E004DC004005D700C005D2004087
:1011D00006CD00D006C8008007C3003008BE00F06E
:1011E00008B900C009B400B00AAF00B00BAA00D023
:1011F0000CA500000EA000500F9B00C010960050E0
:1012000012910000148C00C0158700B0178200B046
:10121000197D00D01B7800001E730040206E0090E6
:10122000226900F024640040275F0090295A00E002
:101230002B5500102E500020304B0010324600E09D
:1012400033410090353C001037370070383200A031
:10125000392D00B03A2800A03B2300603C1E00104E
:101260003D1900903D1400103E0F00703E0A00C072
:101270003E0500003F0000403FFBFF803FF6FFC0FF
:101280003FF1FF453120544845524D414C205255C5
:101290004E415741590042454420544845524D4122
:1012A0004C2052554E4157415900546865726D614A
:1012B0006C2052756E6177617900453120457272FC
:1012C0003A204D415854454D50004572723A204DD8
:1012D000415854454D5020424544004D41585445D5
:1012E0004D502074726967676572656400453120EE
:1012F0004572723A204D494E54454D500045727228
:101300003A204D494E54454D5020424544004D49E8
:101310004E54454D5020747269676765726564006C
:101320004D383420582059205A20450020280020CC
:101330002F002042403A0020403A000220746F6F94
:10134000206C6F6E6720657874727573696F6E209C
:1013500070726576656E7465640A0020636F6C64F4
:1013600020657874727573696F6E2070726576652A
:101370006E7465640A0020746F6F206C6F6E672056
:10138000657874727573696F6E2070726576656EBC
:101390007465640A0020636F6C64206578747275EC
:1013A00073696F6E2070726576656E7465640A008D
:1013B000627573793A2070617573656420666F7227
:1013C00020696E7075740A00627573793A207061D5
:1013D0007573656420666F7220757365720A0062AA
:1013E0007573793A2070726F63657373696E670AFB
:1013F000005446542053657269616C2044656275DF
:10140000673A2046696C616D656E742072756E6F07
:1014100075742E2E2E204A31350A004A313500547B
:1014200046542053657269616C2044656275673A61
:101430002046696C616D656E742072756E6F75748F
:10144000207265636F76657265640A004B494C4C87
:1014500045442E20004B494C4C20636175736564F4
:10146000206279204B494C4C20627574746F6E2F4A
:1014700070696E0A004B494C4C45442E20004B4984
:101480004C4C2063617573656420627920746F6FC2
:10149000206D75636820696E616374697665207478
:1014A000696D65202D2063757272656E7420636F9F
:1014B0006D6D616E643A2000544654205365726924
:1014C000616C2044656275673A204B696C6C2063DF
:1014D0006F6D6D616E642E2E2E204A31310A004AE6
:1014E0003131005072696E7465722068616C746588
:1014F000642E206B696C6C28292063616C6C6564B8
:10150000210A000000A0C000000000000000000050
:1015100000C8420000C8420000A04100000000577F
:1015200061726E696E673A20486F6D696E6720421E
:10153000756D702044697669736F72203C20310AA2
:10154000000202040000A0400000A0400000004093
:10155000000057430000524300004D43FFFFFF458A
:101560004550524F4D206461746173697A652065FE
:1015700072726F722E0A00290A00206279746573F4
:101580003B20637263200053657474696E67732037
:1015900053746F726564202800290A0020627974F0
:1015A00065733B2063726320002073746F726564FF
:1015B0002073657474696E677320726574726965EF
:1015C000766564202800202863616C63756C617403
:1015D000656429210A0020213D2000454550524FD5
:1015E0004D20435243206D69736D61746368202DF3
:1015F000202873746F7265642920002053697A650E
:101600003A2000496E6465783A2000204D61726C82
:10161000696E3D563535290A0028454550524F4DD3
:101620003D00454550524F4D2076657273696F6E8F
:10163000206D69736D6174636820005446542053B3
:10164000657269616C2044656275673A2046696C11
:10165000616D656E742072756E6F75742E2E2E20FE
:101660004A31350A004A3135004A3132004A3137B1
:10167000002020506C616E6E657242756666657200
:1016800042797465733A20002046726565204D6585
:101690006D6F72793A2000436F6D70696C65643AC2
:1016A000204A616E20203820323031390A00207CF7
:1016B00020417574686F723A2028646572686F7093
:1016C000702C20416E796375626963206933204D07
:1016D0006567612C206D6F646F666965642062794F
:1016E00020526F62657274205068616E2C206564B0
:1016F000697465642062792074686F6D61734074E9
:1017000072756574656E2E64652C20303130383208
:10171000303139290A00323031382D30372D33310C
:1017200000204C61737420557064617465643A20C4
:1017300000312E312E390A004D61726C696E002025
:10174000536F6674776172652052657365740A0021
:10175000205761746368646F672052657365740A0B
:10176000002042726F776E206F757420526573652A
:10177000740A002045787465726E616C205265733E
:1017800065740A00506F77657255700A0073746152
:1017900072740A004D3234004D32332025730061DB
:1017A00075746F25692E67006572726F722077728B
:1017B0006974696E6720746F2066696C650A002021
:1017C000503A00205A3A0020593A0020583A006511
:1017D0006E6473746F7073206869743A2000446F8C
:1017E0006E6520736176696E672066696C652E0A86
:1017F000004D323900486F6D696E67206661696C13
:10180000656400202844525952554E290047323908
:10181000204175746F20426564204C6576656C6963
:101820006E67003F20284C2C522C462C4229206FFA
:101830007574206F6620626F756E64732E0A003FA8
:101840002856296572626F7365206C6576656C2019
:10185000697320696D706C61757369626C652028AD
:10186000302D34292E0A00426164205A2076616CA2
:1018700075650A004E6F2062696C696E6561722041
:10188000677269640A0046696C652064656C6574FA
:1018900065643A0044656C6574696F6E20666169C1
:1018A0006C65642C2046696C653A200050726F7438
:1018B00065637465642050696E0A00544654205371
:1018C000657269616C2044656275673A204E6F7A73
:1018D0007A6C652069732068656174696E672E2E65
:1018E0002E204A30360A004A3036005446542053DF
:1018F000657269616C2044656275673A20436F6E5A
:1019000074696E75696E67205344207072696E74D5
:101910002061667465722068656174696E672E2E39
:101920002E204A30340A004A3034005446542053A2
:10193000657269616C2044656275673A204E6F7A02
:101940007A6C652068656174696E672069732064CC
:101950006F6E652E2E2E204A30370A004A3037002F
:1019600020573A005446542053657269616C2044F4
:10197000656275673A204265642069732068656115
:1019800074696E672E2E2E204A30380A004A30388D
:10199000005446542053657269616C204465627539
:1019A000673A204265642068656174696E672069E2
:1019B0007320646F6E652E2E2E204A30390A004A3D
:1019C00030390020573A006F70656E206661696C8F
:1019D00065642C2046696C653A200043616E6E6F29
:1019E00074206F70656E2073756264697220005494
:1019F00046542053657269616C2044656275673A8C
:101A0000205344207072696E742070617573656430
:101A10002E2E2E204A30350A004A303500544654C6
:101A20002053657269616C2044656275673A20468F
:101A3000696C616D656E742072756E6F7574207758
:101A400068696C65207072696E74696E672E2E2EDF
:101A5000204A32330A004A3233004739310A4731CB
:101A6000205A2D313020463234300A473930005365
:101A7000442063617264206F6B0A006F70656E5260
:101A80006F6F74206661696C65640A00766F6C75AF
:101A90006D652E696E6974206661696C65640A0003
:101AA0004572726F723A00534420696E6974206601
:101AB00061696C0A006563686F3A00656E717565EF
:101AC0007565696E672022004B494C4C45442E20B9
:101AD000005072696E7465722073746F7070656403
:101AE0002064756520746F206572726F72732E208A
:101AF00046697820746865206572726F7220616E25
:101B00006420757365204D39393920746F207265F2
:101B100073746172742E202854656D7065726174DF
:101B20007572652069732072657365742E20536524
:101B300074206974206166746572207265737461C3
:101B40007274696E67290A004E6F20436865636B83
:101B500073756D2077697468206C696E65206E7589
:101B60006D6265722C204C617374204C696E653A0D
:101B700020004E6F20436865636B73756D20776935
:101B80007468206C696E65206E756D6265722C20BC
:101B90004C617374204C696E653A2000636865631C
:101BA0006B73756D206D69736D617463682C204C67
:101BB000617374204C696E653A20004C696E652033
:101BC0004E756D626572206973206E6F74204C6172
:101BD0007374204C696E65204E756D6265722B3191
:101BE0002C204C617374204C696E653A20004D3195
:101BF0003130004D333100534420726561642065FB
:101C000072726F720A00446F6E65207072696E7432
:101C1000696E672066696C650A0020496E76616CA2
:101C2000696420657874727564657220000000A094
:101C3000C0000000000000000000005243000052FD
:101C40004300004D435072696E7465722073746F67
:101C5000707065642064756520746F206572726FA2
:101C600072732E2046697820746865206572726FE1
:101C70007220616E6420757365204D393939207486
:101C80006F20726573746172742E202854656D70B4
:101C9000657261747572652069732072657365740D
:101CA0002E205365742069742061667465722072F9
:101CB000657374617274696E67290A0053544F50DA
:101CC0002063616C6C656420626563617573652077
:101CD0006F6620424C546F756368206572726F7234
:101CE000202D207265737461727420776974682086
:101CF0004D3939390A0042696C696E656172204C50
:101D00006576656C696E6720477269643A0A0024DB
:101D1000F4D43050C38E20C2A24017828B701112AF
:101D20007A910D816CD90AA861E108C758660761EC
:101D30005143061E4B5D05C145A7041A4111040914
:101D40003D9803713931034036DB0265339102D48B
:101D5000305402802E1D02632CEE01752AC501B09D
:101D600028A001102781018F2564012B244B01E05D
:101D7000223401AC211F018D200D01801FFC008445
:101D80001EED00971DDF00B81CD200E61BC6002028
:101D90001BBC00641AB200B219A8000A19A0006A9C
:101DA000189900D117910040178B00B516840031A7
:101DB000167E00B31579003A157300C7146F0058EA
:101DC000146A00EE1366008813630025135E00C7D3
:101DD000125B006C12570015125400C111510070B3
:101DE000114F0021114B00D61049008D10470046BD
:101DF00010440002104200C00F4000800F3E00421D
:101E00000F3C00060F3B00CB0E3800930E37005CF2
:101E10000E3500270E3400F30D3200C10D31009055
:101E20000D3000600D2E00320D2D00050D2C00D957
:101E30000C2B00AE0C2900850C29005C0C2700350A
:101E40000C27000E0C2600E80B2400C40B2400A075
:101E50000B23007D0B23005A0B2100390B210018A6
:101E60000B2000F80A1F00D90A1E00BB0A1E009DA5
:101E70000A1D00800A1D00630A1C00470A1B002C73
:101E80000A1B00110A1A00F7091A00DD091900C41B
:101E9000091900AB091900920917007B09180063A2
:101EA0000917004C09160036091600200916000A09
:101EB000091500F5081500E0081400CC081400B856
:101EC000081400A4081400900813007D0812006B89
:101ED00008130058081200460812003408110023A5
:101EE0000811001208110001081100F0071000E0AD
:101EF000071000D0071000C0071000B0070F00A1A6
:101F000007100091070E0083070F0074070F00658C
:101F1000070E0057070E0049070E003B070D002E65
:101F2000070E0020070D0013070D0006070D00F92E
:101F3000060C00ED060D00E0060C00D4060C00C8EF
:101F4000060C00BC060C00B0060C00A4060B0099A1
:101F5000060C008D060B0082060B0077060B006C4A
:101F6000060B0061060A0057060B004C060A0042E9
:101F7000060A0038060A002E060A0024060A001A7D
:101F8000060A001006090007060A00FD050900F40C
:101F9000050900EB050900E2050900D9050900D093
:101FA000050900C7050900BE050900B5050800AD13
:101FB000050800A50509009C050800940508008C8B
:101FC000050800840508007C050800740508006CFD
:101FD000050700650508005D050700560508004E69
:101FE00005070047050700400508003805070031D0
:101FF0000507002A050700230507001C0506001633
:102000000507000F0507000805060002050700FB8D
:10201000040600F5040700EE040600E8040600E2EA
:10202000040700DB040600D5040600CF040600C93F
:10203000040600C3040600BD040600B7040600B190
:10204000040500AC040600A6040600A00405009BDD
:1020500004060095040500900406008A0405008526
:10206000040500800406007A04050075040500706C
:102070000405006B04050066040500610405005CAE
:1020800004050057040500520405004D04050048EE
:10209000040500430405003E0404003A040500352D
:1020A000040500300404002C040500270404002368
:1020B0000405001E0404001A04040016040500119F
:1020C0000404000D040400090405000404040000D5
:1020D000040400FC030400F8030400F4030400F00B
:1020E000030400EC030400E8030400E4030400E03C
:1020F000030400DC030400D8030400D4030400D06C
:10210000030400CC030400C8030300C50303002438
:10211000F404D9201BC40C5C0E9804C4095F02654A
:10212000077101F405F900FB04B30048048700C1FE
:102130000369005803550003034500BE023A0084BA
:1021400002310053022A002902250004022000E483
:10215000011C00C8011900AF011700980114008488
:10216000011300710110006101100051010E0043C4
:10217000010D0036010B002B010B0020010B001597
:102180000109000C01090003010800FB000800F32D
:10219000000800EB000700E4000600DE000600D89F
:1021A000000600D2000600CC000500C7000500C2F2
:1021B000000500BD000400B9000400B5000400B132
:1021C000000400AD000400A9000400A5000300A263
:1021D0000003009F0004009B00030098000300958B
:1021E00000020093000300900003008D0002008BAA
:1021F00000030088000200860002008400030081C2
:102200000002007F0002007D0002007B00020079D6
:1022100000020077000100760002007400020072E4
:10222000000100710002006F0002006D0001006CEF
:102230000002006A000100690002006700010066F8
:1022400000010065000100640002006200010061FD
:10225000000100600001005F0002005D0001005C01
:102260000001005B0001005A000100590001005804
:102270000001005700010056000100550001005404
:102280000001005300000053000100520001005102
:10229000000100500001004F0001004E0000004E00
:1022A0000001004D0001004C0001004B0000004BFC
:1022B0000001004A000100490001004800000048F8
:1022C00000010047000100460000004600010045F3
:1022D00000000045000100440001004300000043ED
:1022E00000010042000000420001004100000041E6
:1022F000000100400001003F0000003F0001003EDF
:102300000000003E0001003D0000003D0001003CD7
:102310000000003C0000003C0001003B0000003BCE
:102320000001003A0000003A0001003900000039C5
:1023300000010038000000380000003800010037BC
:1023400000000037000100360000003600000036B3
:1023500000010035000000350000003500010034A8
:10236000000000340000003400010033000000339E
:102370000000003300010032000000320000003293
:102380000001003100000031000000310001003088
:1023900000000030000000300001002F0000002F7E
:1023A0000000002F0000002F0001002E0000002E72
:1023B0000000002E0001002D0000002D0000002D67
:1023C0000000002D0001002C0000002C0000002C5B
:1023D0000000002C0001002B0000002B0000002B4F
:1023E0000000002B0001002A0000002A0000002A43
:1023F0000000002A00010029000000290000002937
:102400000000002900000029000100280000002829
:10241000000000280000002800000028000100271C
:102420000000002700000027000000270000002710
:102430000001002600000026000000260000002603
:1024400000000026000100250000002500000025F6
:1024500000000025000000250000002500010024E8
:1024600000000024000000240000002400000024DC
:1024700000010023000000230000002300000023CF
:1024800000000023000000230000002300010022C0
:1024900000000022000000220000002200000022B4
:1024A00000000022000100210000002100000021A6
:1024B0000000002100000021000000210000002198
:1024C000000100200000002000000020000000208B
:1024D000000000200000002000000020000000207C
:1024E0000001001F0000001F0000001F0000001F6F
:1024F0000000001F0000001F0000001F0001001E60
:102500000000001E0000001E0000001E000000C2AF
:102510003100001C260000F4190000D80F0000EB69
:10252000080000C004000075020000400100002007
:102530005A3A0020593A0020436F756E7420583A79
:102540000020453A00205A3A0020593A00583A00F3
:102550003A004361703A005741524E494E4721209C
:102560004C6F77205A204A65726B206D6179206C20
:1025700065616420746F20756E77616E7465642088
:102580007061757365732E0A00205A002059005837
:102590000020204D61783A2000205A002059005830
:1025A0000020204D696E3A20004F6E20004F666675
:1025B00000536F667420656E6473746F70733A2095
:1025C0000020643A0020693A0020703A00496E7693
:1025D000616C69642065787472756465720A004B79
:1025E00064200023646566696E6520444546415554
:1025F0004C545F004B69200023646566696E65205A
:1026000044454641554C545F004B7020002364659F
:1026100066696E652044454641554C545F005049FB
:1026200044204175746F74756E652066696E6973B8
:10263000686564212050757420746865206C61732E
:1026400074204B702C204B6920616E64204B6420F9
:10265000636F6E7374616E74732066726F6D206247
:10266000656C6F7720696E746F20436F6E66696763
:1026700075726174696F6E2E680A0050494420417A
:1026800075746F74756E65206661696C6564212070
:1026900074696D656F75740A004531205448455260
:1026A0004D414C2052554E4157415900424544201E
:1026B000544845524D414C2052554E4157415900C6
:1026C000546865726D616C2052756E617761790036
:1026D00045312048656174696E67206661696C6583
:1026E00064004265642068656174696E6720666194
:1026F000696C65640048656174696E67206661692C
:102700006C656400504944204175746F74756E6542
:10271000206661696C6564212054656D7065726125
:102720007475726520746F6F20686967680A00208D
:102730004B643A2000204B693A2000204B703A202D
:10274000000A20436C617373696320504944200A76
:10275000002054753A2000204B753A2000206D610E
:10276000783A2000206D696E3A200020643A2000FB
:1027700020626961733A2000504944204175746FAA
:1027800074756E65206661696C65642120426164C0
:10279000206578747275646572206E756D626572FD
:1027A0000A00504944204175746F74756E6520733A
:1027B000746172740A004F66660A0046616465209F
:1027C0004865696768742000426564204C657665D9
:1027D0006C696E6720004661696C656420746F20C7
:1027E000656E61626C6520426564204C6576656C3F
:1027F000696E670A007C3C3E5E2B3D3F2F5B5D3B74
:102800002C2A225C0048617264636F646564204412
:10281000656661756C742053657474696E677320A6
:102820004C6F616465640A00B80B0000B80B0000CF
:102830003C000000102700000000FA430000FA43AB
:102840000000C040000070420000A0420000A04212
:102850000000C8433333B9423A0A0020286D6D297D
:102860000020204D393030204B004C696E6561727C
:1028700020416476616E63653A0A0020204D383548
:1028800031205A005A2D50726F6265204F66667370
:1028900065740020440020490020204D333034204E
:1028A000500020440020490020204D33303120507A
:1028B000005049442073657474696E67733A0A0066
:1028C000205A0020204D36363600456E6473746FF2
:1028D000702061646A7573746D656E743A0A0020C5
:1028E0005A00204A00202047323920572049002032
:1028F0005A0020204D3432302053004175746F202F
:10290000426564204C6576656C696E673A0A002002
:102910005A0020590020204D323036205800486F90
:102920006D65206F66667365743A0A002045002065
:102930005A00205900205800205400205300202025
:102940004D32303520510020453C6D61785F655F28
:102950006A65726B3E0020583C6D61785F785F6AF3
:1029600065726B3E20593C6D61785F795F6A657274
:102970006B3E205A3C6D61785F7A5F6A65726B3E90
:1029800000416476616E6365643A20513C6D696E06
:102990005F7365676D656E745F74696D655F757390
:1029A0003E20533C6D696E5F666565647261746557
:1029B0003E20543C6D696E5F74726176656C5F6633
:1029C000656564726174653E0020540020520020E9
:1029D000204D323034205000416363656C65726174
:1029E00074696F6E2028756E6974732F7332293A7B
:1029F00020503C7072696E745F616363656C3E2049
:102A0000523C726574726163745F616363656C3EAE
:102A100020543C74726176656C5F616363656C3EE3
:102A20000A00204500205A0020590020204D323055
:102A3000312058004D6178696D756D204163636583
:102A40006C65726174696F6E2028756E6974732F7E
:102A50007332293A0A00204500205A0020590020EC
:102A6000204D3230332058004D6178696D756D20EE
:102A70006665656472617465732028756E69747328
:102A80002F73293A0A00204500205A0020590020BF
:102A9000204D393220580053746570732070657270
:102AA00020756E69743A0A0020204D32303020447F
:102AB000300A0020204D3230302044002044697319
:102AC00061626C65640A0046696C616D656E7420B4
:102AD00073657474696E67733A0020204732312041
:102AE0002020203B0000002100240027002A002D88
:102AF000003000330001010000040107010A010059
:102B0000002200250028002B002E00310034000296
:102B1000010000050108010B010000200023002630
:102B20000029002C002F00320000010000030106E4
:102B30000109010505050507050808080802020244
:102B4000020A0A0808040404040101010101010148
:102B5000010303030303030303040707070C0C0C1F
:102B60000C0C0C0C0C0202020206060606060606F7
:102B7000060B0B0B0B0B0B0B0B0102102020080894
:102B800010204010204080020102010804020101CF
:102B900002040810204080804020100804020180B8
:102BA000040201804020100804020108040201010F
:102BB0000204081020408001020408102040800018
:102BC000000A0B02090C0D0E0807030401000000A7
:102BD00000000000000000000000000000000000F5
:102BE00000000000000000000000001211100000B2
:102BF00000000000000000000000000000000000D5
:102C00000000000000556E6B6E6F776E20636F6D75
:102C10006D616E643A20220050726F62696E6720A7
:102C20006661696C65640A00205A3A200020593AAE
:102C3000200042656420583A20002066697273744F
:102C40000A005A0059005800486F6D65200045720F
:102C5000726F722077726974696E6720746F204595
:102C60004550524F4D210A0054524947474552455D
:102C700044006F70656E003A20007A5F70726F6278
:102C800065007A325F6D696E007A5F6D696E0079FA
:102C90005F6D696E00785F6D696E005265706F726E
:102CA00074696E6720656E6473746F7020737461ED
:102CB0007475730A0057726974696E6720746F20A7
:102CC00066696C653A20006F70656E206661696C9C
:102CD00065642C2046696C653A20006F70656E2033
:102CE0006661696C65642C2046696C653A20004613
:102CF000696C652073656C65637465640A002053B4
:102D0000697A653A200046696C65206F70656E656A
:102D1000643A20002066696C653A2000646F696E31
:102D200067006672657368004E6F772000454E44F9
:102D300020535542524F5554494E450A00222070A7
:102D40006F73002220706172656E743A22005355D1
:102D500042524F5554494E452043414C4C207461DA
:102D6000726765743A22004B494C4C45442E200052
:102D7000747279696E6720746F2063616C6C207364
:102D800075622D67636F64652066696C6573207773
:102D900069746820746F6F206D616E79206C657640
:102DA000656C732E204D4158206C6576656C2069EA
:102DB000733A00736C6F743A00526573656E643ACF
:102DC00020006F6B0000F8D7E0D111241FBECFEFB9
:102DD000D1E2DEBFCDBF00E00CBF14E0A0E0B2E066
:102DE000EAE8FDEC01E00BBF02C007900D92A630AF
:102DF000B107D9F727E1A6E0B4E001C01D92A43ADB
:102E0000B207E1F716E1C4EED6E100E006C0219773
:102E10000109802FFE010E9422E6C33ED10780E017
:102E20000807A9F70E9401D20C94B4E60C940000A4
:102E30002F923F924F925F926F927F928F929F92CA
:102E4000AF92BF92CF92DF92EF92FF920F931F93B8
:102E5000CF93DF93CDB7DEB7CB56D1090FB6F89439
:102E6000DEBF0FBECDBF91E0909324058091EF1699
:102E70008D3411F40C941E20843511F40C94F32D30
:102E8000873411F00C943F2E2090ED163090EE1602
:102E90002CE12216310409F42EC69CF444E02416D9
:102EA000310444F452E025163104C4F537FE2FC036
:102EB0000C941A2084E02816310409F4DDC50C9422
:102EC0001A20AAE22A16310409F405C764F4EDE1D8
:102ED0002E16310409F426C6FEE12F16310409F43A
:102EE00025C60C941A202BE52216310409F4CBC711
:102EF0003CE52316310409F4CAC74AE52416310417
:102F000011F00C941A2010920C040C94412E809114
:102F1000030281110C94462E0C94412E80910302E1
:102F2000882311F40C94412E0E948C7C82E50E942F
:102F30006946882309F44CC10E94F7434B015C01A8
:102F400020E030E0A9010E94E1DE882309F470C18D
:102F500080911A0490911B04A0911C04B0911D044F
:102F600088AF99AFAAAFBBAF20911E0430911F0468
:102F700040912004509121042CAF3DAF4EAF5FAF84
:102F800080913E0590913F05A0914005B09141058B
:102F90002C968CAF9DAFAEAFBFAF2C972091420562
:102FA00030914305409144055091450528962CAF3A
:102FB0003DAF4EAF5FAF28979C01AD0168AD79ADD5
:102FC0008AAD9BAD0E94E1DE81110FC028962CAD29
:102FD0003DAD4EAD5FAD28976CAD7DAD8EAD9FAD77
:102FE0000E94E1DE882309F423C111E032E02316B8
:102FF000310409F010E020E030E0A901C501B4017E
:103000000E94E1DE881F8827881F181759F080E08A
:1030100090E0A0E8BFEB64968CAF9DAFAEAFBFAFC2
:1030200064970AC020E030E040E85FE364962CAF8C
:103030003DAF4EAF5FAF649728AD39AD4AAD5BADE4
:103040002C966CAD7DAD8EAD9FAD2C970E9426E386
:1030500060966CAF7DAF8EAF9FAF60972CAD3DADEE
:103060004EAD5FAD28966CAD7DAD8EAD9FAD289712
:103070000E9426E36B017C0160962CAD3DAD4EAD08
:103080005FAD6097CA01B9010E9446DF2B013C0188
:10309000A7019601C701B6010E9446DF9B01AC0162
:1030A000C301B2010E9427E30E9492E524966CAF0F
:1030B0007DAF8EAF9FAF249720E030E040E05FE32C
:1030C0000E9446DF2B013C01A5019401C501B4011A
:1030D0000E9446DF4B015C01A3019201C301B201D2
:1030E0000E9446DF9B01AC01C501B4010E9426E3AA
:1030F0000E9492E564962CAD3DAD4EAD5FAD6497F8
:103100000E9446DF4B015C01C701B601905824962E
:103110002CAD3DAD4EAD5FAD24970E9403E4A501FB
:1031200094010E9446DF6B017C012C962CAD3DADD5
:103130004EAD5FAD2C9768AD79AD8AAD9BAD0E9469
:1031400027E320E030E040E05FE30E9446DF9B01A0
:10315000AC01C701B6010E9427E328AD39AD4AADE5
:103160005BAD0E9426E36B017C0128962CAD3DAD42
:103170004EAD5FAD28976CAD7DAD8EAD9FAD0E941D
:1031800027E320E030E040E05FE30E9446DF2B01D0
:103190003C0124962CAD3DAD4EAD5FAD24976096BD
:1031A0006CAD7DAD8EAD9FAD60970E9403E4A5012F
:1031B00094010E9446DF9B01AC01C301B2010E9451
:1031C00027E32CAD3DAD4EAD5FAD0E9426E314C0AC
:1031D00089E40E946946882329F00E94F7436B0125
:1031E0007C0103C0C12CD12C76018AE40E9469467F
:1031F000882309F10E94F7432C966CAF7DAF8EAF08
:103200009FAF2C9720E030E0A901C701B6010E94D2
:10321000E1DE81111FC020E030E0A9012C966CADE9
:103220007DAD8EAD9FAD2C970E94E1DE811112C065
:10323000E0EAFAE10DC420E030E0A901C701B601DF
:103240000E94E1DE8823A1F32C961CAE1DAE1EAEBB
:103250001FAE2C97D701C601B05888AF99AFAAAF5F
:10326000BBAF2C962CAD3DAD4EAD5FAD2C975058FD
:103270002CAF3DAF4EAF5FAF9C01AD01BC01CD01A6
:103280000E9446DF4B015C012CAD3DAD4EAD5FAD04
:10329000CA01B9010E9446DF9B01AC01C501B4011E
:1032A0000E9427E30E9492E5A0966CAF7DAF8EAF9F
:1032B0009FAFA09780911A0490911B04A0911C04C9
:1032C000B0911D0428968CAF9DAFAEAFBFAF2897CD
:1032D000A7019601BC01CD010E9427E364966CAF63
:1032E0007DAF8EAF9FAF649720911E0430911F0475
:1032F000409120045091210460962CAF3DAF4EAF19
:103300005FAF60972C962CAD3DAD4EAD5FAD2C9769
:1033100060966CAD7DAD8EAD9FAD60970E9427E34A
:10332000A4966CAF7DAF8EAF9FAFA49780913E0502
:1033300090913F05A0914005B091410568968CAFF2
:103340009DAFAEAFBFAF689764962CAD3DAD4EADAF
:103350005FAD6497BC01CD010E9426E36B017C0147
:103360002091420530914305409144055091450517
:103370006C962CAF3DAF4EAF5FAF6C97A4962CAD63
:103380003DAD4EAD5FADA4976C966CAD7DAD8EAD91
:103390009FAD6C970E9426E34B015C018091220453
:1033A00090912304A0912404B0912504A8968CAF99
:1033B0009DAFAEAFBFAFA8979C01AD016091460530
:1033C0007091470580914805909149050E9426E338
:1033D00024966CAF7DAF8EAF9FAF2497A701960167
:1033E00068AD79AD8AAD9BAD0E9446DF2B013C01F3
:1033F000A50194016CAD7DAD8EAD9FAD0E9446DF01
:103400009B01AC01C301B2010E9427E32B013C01E7
:10341000A501940168AD79AD8AAD9BAD0E9446DFF0
:103420004B015C01A70196016CAD7DAD8EAD9FADEA
:103430000E9446DF9B01AC01C501B4010E9426E356
:10344000A30192010E949AE36B017C0120E030E02D
:10345000A9010E94E1DE87FF0AC02BED3FE049ECA5
:1034600050E4C701B6010E9427E36B017C0192E0A2
:103470002916310451F42BED3FE049EC50E4C7012B
:10348000B6010E9426E36B017C0120E030E0A90137
:10349000C701B6010E94E1DE811128C068962CADFB
:1034A0003DAD4EAD5FAD689728966CAD7DAD8EADF0
:1034B0009FAD28970E94E1DE811118C06C962CAD5B
:1034C0003DAD4EAD5FAD6C9760966CAD7DAD8EAD94
:1034D0009FAD60970E94E1DE811108C0FBEDCF2E09
:1034E000FFE0DF2EF9ECEF2EF0E4FF2EA7019601AE
:1034F000A0966CAD7DAD8EAD9FADA0970E9446DFCE
:103500004B015C0120E030E0A90124966CAD7DAD5B
:103510008EAD9FAD24970E94E1DE8823E9F0A501DE
:103520009401C501B4010E9446DF4B015C01249661
:103530002CAD3DAD4EAD5FAD2497CA01B9010E94DF
:1035400046DF9B01AC01C501B4010E9427E30E9444
:1035500092E54B015C010DC020E030E0A901C501FE
:10356000B4010E944DE587FF04C0B7FAB094B7F8E4
:10357000B0942FE632E143E85AE3C501B4010E945A
:10358000E1DE87FF02C00C94412EC501B4010E9408
:103590009CE40E9470E42E967FAF6EAF2E97DB0105
:1035A000AB2B31F4E1E0F0E02E96FFAFEEAF2E97BB
:1035B00040902604509027046090280470902904BD
:1035C0002E962EAD3FAD2E97B90180E090E00E947F
:1035D000E5DE4B015C019B01AC01C701B6010E9415
:1035E00003E428966CAF7DAF8EAF9FAF2897A501FF
:1035F000940124966CAD7DAD8EAD9FAD24970E9455
:1036000003E4A0966CAF7DAF8EAF9FAFA097A301F0
:10361000920160914A0570914B0580914C05909103
:103620004D050E9426E3A50194010E9403E4AC9697
:103630006CAF7DAF8EAF9FAFAC9728962CAD3DADF4
:103640004EAD5FAD2897CA01B9010E9446DF20E068
:1036500030E040E05FE30E9446DF9B01AC0160E0A8
:1036600070E080E89FE30E9426E368966CAF7DAF30
:103670008EAF9FAF6897A8968CAD9DADAEADBFAD38
:10368000A89789879A87AB87BC874D865E866F86A9
:10369000788A6091000270910102072E000C880B5D
:1036A000990B0E94E7DE20913C0230913D0240914F
:1036B0003E0250913F020E9446DF2AE037ED43E28E
:1036C0005CE30E9446DF6CAB7DAB8EAB9FAB0E9490
:1036D000407A9B01AC0128533F4F4F4F5F4F6C9690
:1036E0002CAF3DAF4EAF5FAF6C9748AC59AC6AACF6
:1036F0007BAC22242394312C39E121963FAF2197D2
:103700002E964EAD5FAD2E974215530509F44CC170
:103710000E949B500E94407ADC01CB016C962CAD3C
:103720003DAD4EAD5FAD6C97821B930BA40BB50BFB
:10373000B7FD10C00E94407A9B01AC0128533F4F57
:103740004F4F5F4F6C962CAF3DAF4EAF5FAF6C9756
:103750000E94556721963FAD2197315021963FAF8A
:103760002197332309F445C02CAD3DAD4EAD5FAD7F
:1037700068966CAD7DAD8EAD9FAD68970E9446DFBB
:103780006B017C019201A30128966CAD7DAD8EADDD
:103790009FAD28970E9446DFA70196010E9427E36C
:1037A0007B018C019201A30168966CAD7DAD8EAD5D
:1037B0009FAD68970E9446DF4B015C012CAD3DAD8B
:1037C0004EAD5FAD28966CAD7DAD8EAD9FAD2897AB
:1037D0000E9446DF9B01AC01C501B4010E9426E3B3
:1037E0002B013C01C701D8018CAF9DAFAEAFBFAF7D
:1037F00055C0B10180E090E00E94E5DE28962CAD36
:103800003DAD4EAD5FAD28970E9446DF4B015C0198
:103810000E9400E46B017C01C501B4010E9488E5AF
:103820004B015C01A701960168AD79AD8AAD9BADF6
:103830000E9446DF2B013C012C962CAD3DAD4EADD8
:103840005FAD2C97C501B4010E9446DFA301920130
:103850000E9427E32B013C01A501940168AD79ADDD
:103860008AAD9BAD0E9446DF4B015C012C962CADCE
:103870003DAD4EAD5FAD2C97C701B6010E9446DF4E
:103880009B01AC01C501B4010E9426E36CAF7DAF82
:103890008EAF9FAF49E121964FAF21979201A301CF
:1038A00064966CAD7DAD8EAD9FAD64970E9427E3AD
:1038B00069837A838B839C832CAD3DAD4EAD5FAD28
:1038C000A4966CAD7DAD8EAD9FADA4970E9427E30D
:1038D0006D837E838F839887A0962CAD3DAD4EADD2
:1038E0005FADA09769857A858B859C850E9427E3CB
:1038F00069877A878B879C87AC962CAD3DAD4EADA2
:103900005FADAC976D857E858F8598890E9427E392
:103910006D877E878F87988B80910E02882321F098
:10392000CE0101960E949464E09023051CA61DA67A
:103930001EA61FA689819A81AB81BC8188A399A309
:10394000AAA3BBA38D819E81AF81B8858CA39DA3C3
:10395000AEA3BFA389859A85AB85BC8588A799A7A7
:10396000AAA7BBA7AE01485D5F4FBE016C5D7F4F4C
:10397000CE0180960E943EC2CE018C966C018E01D3
:103980000C5C1F4F9E01235F3F4FAE01485D5F4FB0
:10399000BE016C5D7F4F0C970E945C54882321F020
:1039A0009FEF291A390AACCEE090230518AA19AA6C
:1039B0001AAA1BAA80913E0590913F05A09140054F
:1039C000B091410588A399A3AAA3BBA38091420506
:1039D00090914305A0914405B09145058CA39DA30A
:1039E000AEA3BFA38091460590914705A0914805DD
:1039F000B091490588A799A7AAA7BBA7AE01485DC2
:103A00005F4FBE016C5D7F4FCE0180960E943EC22B
:103A1000DE01D0966D018E010C5C1F4F2AE435E06B
:103A2000AE01485D5F4FBE016C5D7F4FCE01809659
:103A30000E945C5480E1EEE3F5E0AAE1B4E001907D
:103A40000D928A95E1F70C94412E0E943E44F801B4
:103A500084918F010F5F1F4F8111F7CFEDE1F2E0ED
:103A600084918F010F5F1F4F882311F40C94412E16
:103A70000E943E44F801F4CF80E50E946946882305
:103A800079F08091060490910704009749F04AE08C
:103A900050E060E070E00E9460DD6B017C0103C0DB
:103AA000C12CD12C760183E50E946946882361F000
:103AB0000E94F74320E030E04AE754E40E9446DFEA
:103AC0000E9470E46B017C010E947E640E94407A37
:103AD000C60ED71EE81EF91E0E94407ADC01CB01FB
:103AE0008C199D09AE09BF09B7FD02C00C94412E87
:103AF0000E945567F1CF809119048770873011F0CB
:103B00000C944B2E8FE40E946946882319F00E9482
:103B1000114603C08FE40E94204681110C94412E6F
:103B20000C944B2E0E944C7E0C94412EC0901A0493
:103B3000D0901B04E0901C04F0901D0488E50E94C6
:103B40006946811109C020E030E044E052E4C70139
:103B5000B6010E9427E302C00E94F74368A379A33D
:103B60008AA39BA3C0901E04D0901F04E090200461
:103B7000F090210489E50E946946811109C020E086
:103B800030E040EA50E4C701B6010E9427E302C0DA
:103B90000E94F7439B01AC0169837A838B839C83EA
:103BA00068A179A18AA19BA10E945F66882311F474
:103BB0000C94412E80E00E9445930E94968D85E4EE
:103BC0000E946946882321F00E941146182F04C0E4
:103BD00085E40E94204611E086E50E94694688231C
:103BE00021F00E94F045262F01C021E0412FBE01A7
:103BF0006F5F7F4FCE0180960E9406B76B017C01FC
:103C00009B01AC010E94D3E581115FC088A099A0FF
:103C1000AAA0BBA020E030E0A901C501B4010E9428
:103C2000E1DE87FF05C027E137EB41E558EB04C033
:103C300027E137EB41E558E3C501B4010E9427E3D2
:103C4000AB01BC018DE392E00E9472C889809A802A
:103C5000AB80BC8020E030E0A901C501B4010E9426
:103C6000E1DE87FF05C027E137EB41E558EB04C0F3
:103C700027E137EB41E558E3C501B4010E9427E392
:103C8000AB01BC0188E392E00E9472C820E030E002
:103C9000A901C701B6010E94E1DE87FF05C027E147
:103CA00037EB41E558EB04C027E137EB41E558E33A
:103CB000C701B6010E9427E3AB01BC0183E392E098
:103CC0000E9472C88AE00E943E440E947D8D0E943C
:103CD00079A50C94412E80910302882311F40C9451
:103CE000412E89E40E946946082F882321F00E9412
:103CF000F045E62E01C0E12C8AE40E946946182FA7
:103D0000882321F00E94F045F62E01C0F12C0023FB
:103D100019F0B4E0BE1528F0112389F0E4E0EF15A6
:103D200070F4E5E4F2E084918F010F5F1F4F882368
:103D300011F40C94412E0E943E44F801F4CF0E94ED
:103D400034440023F1F020916B1030916C104E2D13
:103D50004203B001439F700D11248091780590912A
:103D60007905680F791F072E000C880B990B0E94AC
:103D7000E7DE60933E0570933F0580934005909386
:103D800041051123F1F020916D1030916E105F2DDF
:103D90005203B001539F700D112480917A059091C8
:103DA0007B05680F791F072E000C880B990B0E946A
:103DB000E7DE60934205709343058093440590933A
:103DC000450580E50E9469468823E9F00E94114676
:103DD0008823A9F10023D9F020E030E044E052E448
:103DE00060913E0570913F0580914005909141059D
:103DF0000E9426E360933E0570933F058093400543
:103E00009093410504C080E50E942046E1CF112334
:103E1000B1F020E030E040EA50E46091420570915A
:103E2000430580914405909145050E9426E36093E7
:103E3000420570934305809344059093450586E4BD
:103E40000E9469468823D9F00E94F7436B017C01E8
:103E500020E030E0A9010E944DE5181684F420E02E
:103E600030E040E752E4C701B6010E9403E46093EA
:103E70003C0270933D0280933E0290933F020E9469
:103E8000366B0C94412E90930C040C94412E43E617
:103E9000242E42E0342E52E3E52E55E0F52E8AE141
:103EA00094E099AF88AF6AEDC62E60E1D62E00E0AF
:103EB00010E0D1018D911D010E946946882309F40B
:103EC0004BC00E94F7432B013C01133049F0F6012F
:103ED00020813181428153810E9426E32B013C01E4
:103EE000A8ADB9AD2D913D914D915C91C301B20149
:103EF0000E9426E34B015C012DEB37E346E855EBCE
:103F00000E944DE587FD0AC02DEB37E346E855E3F7
:103F1000C501B4010E94E1DE1816F4F4133051F427
:103F2000409226045092270460922804709229043B
:103F300001E012C0A5019401F701608171818281C5
:103F400093810E9427E3D7016D937D938D939C937A
:103F50001397812F0E94608F1F5FB4E0EB0EF11C5E
:103F6000E8ADF9AD3496F9AFE8AFF4E0CF0ED11C6F
:103F7000143009F09ECF002309F458C0C0902604E5
:103F8000D0902704E0902804F090290420E030E04D
:103F9000A901C701B6010E9427E320914011309189
:103FA000411140914211509143110E9446DF0E94FD
:103FB00058E560936509709366098093670990934B
:103FC0006809C0925509D0925609E0925709F092BB
:103FD00058099091330980913409981719F00E947B
:103FE000216424C00E947E6480916F00982F92709B
:103FF00081FF05C080916F008D7F80936F0040919D
:10400000650950916609609167097091680940934C
:104010001310509314106093151070931610992379
:1040200029F080916F00826080936F000E9479A5D3
:104030000C94412E0E943DB90C94412E8091ED16B6
:104040009091EE168737910509F495C70CF0D4C00E
:104050008135910509F4BEC50CF066C08B31910520
:1040600009F465C2ACF58631910509F414C20CF56A
:104070008231910509F4C9C584F4419711F00C947B
:10408000F02D5F988A9847988091080181708093FD
:104090000601479812980C94412E8431910509F439
:1040A000BAC1459711F00C94F02D0E94E7860C944C
:1040B000412E8831910509F40AC20CF4F2C189310C
:1040C000910509F40FC24A9709F423C20C94F02D0C
:1040D0008032910509F4D1C284F48D31910511F437
:1040E0000C94412E0CF4BBC28E31910509F4C1C26F
:1040F0004F9709F40EC30C94F02D8B34910509F4FD
:10410000F0C32CF48A9709F4B7C30C94F02D8C34C7
:10411000910509F4EAC38D34910511F00C94F02D4A
:104120000E943F940C94412E8B36910509F440C5B2
:104130006CF58C35910509F4B7C584F48335910588
:1041400009F45EC50CF458C58435910509F45DC5C4
:104150008535910509F48EC50C94F02D88369105AE
:1041600009F4D8C34CF48436910511F00C94F02D69
:104170000E9475460C94412E8936910509F492C42B
:104180008A36910509F4F6C40C94F02D8037910518
:1041900009F453C484F48D36910509F4C5C40CF4B4
:1041A00048C48E36910509F4DEC38F36910509F4B3
:1041B000EDC30C94F02D8337910509F429C154F413
:1041C0008137910509F441C48237910509F4F4C59A
:1041D0000C94F02D8537910511F40C94412E8637FF
:1041E000910511F00C94F02D0091EB161091EC1646
:1041F00083E0D12C40E07EC6803321E0920711F4A9
:104200000C94812B0CF079C08D3C910509F4C2C748
:1042100054F58E3B910509F4A9C484F489379105BE
:1042200009F4B2C60CF4AAC68C38910509F480C40E
:104230008B39910509F451C40C94F02D893C9105FA
:1042400009F4F7C634F4883C910509F4A2C60C942D
:10425000F02D8B3C910509F40CC78C3C910509F4B9
:1042600024C70C94F02D823E910511F40C942C2A55
:104270000CF5833D910511F40C94AD297CF48E3C32
:10428000910511F00C94F02DA3E6CA2EA2E0DA2ECF
:10429000B8E8EB2EB5E0FB2E10E087C78C3D91050A
:1042A00011F40C94B0298D3D910511F40C94BD29A5
:1042B0000C94F02D8D3241E0940711F40C942A2BCC
:1042C0006CF48831A1E09A0711F40C94562A8C32D0
:1042D000914011F40C94012B0C94F02D8E32E1E0FE
:1042E0009E0711F40C942D2B8F32914011F00C94F9
:1042F000F02D0E94FA9D0C94412E853F21E09207FB
:1043000011F40C94B42C0CF046C08A3941E09407A7
:1043100009F497C314F58039A1E09A0711F40C94BD
:10432000142C4CF48336914011F00C94F02DE0EAFB
:10433000FAE10C94012C8139F1E09F0711F40C94FF
:10434000172C8239914011F00C94F02D80E00E94DE
:10435000C38E0E9479A50C94412E853A31E09307D3
:1043600011F40C941D2C4CF4843A914011F00C94EF
:10437000F02D0E9443A60C94412E8C3AA1E09A079E
:1043800009F426C7843F914011F00C94F02D0E944F
:1043900067750C94412E8A39E2E09E0711F40C9463
:1043A000F32CB4F4873F21E0920711F40C94BA2C5B
:1043B00014F40C94B72C883F41E0940711F40C944A
:1043C000C62C8C30924011F40C94EA2C0C94F02DF5
:1043D0008B38A3E09A0711F40C94412E6CF48335CA
:1043E000E3E09E0711F40C94202D8438934011F4DF
:1043F0000C94852D0C94F02D803A23E0920709F45B
:104400007BC1873E934011F40C94DD2D0C94F02D6C
:10441000E6E1F4E00EC5E3E7F2E084918F010F5F7F
:104420001F4F882321F00E943E44F801F6CF1092DE
:10443000770C8AE29AE00E9463AA8BE1EAE2FAE052
:10444000DE01159601900D928A95E1F78091280A78
:104450009091290A9C838B8389EF92E09A838983C8
:1044600040E050E0BE016F5F7F4F80E090E00E942F
:104470003489CE0101960E94E066E4E6F2E0849180
:104480008F010F5F1F4F882311F40C94412E0E945F
:104490003E44F801F4CF1092F9091092FA090C94F5
:1044A000412EE091EB16F091EC168081882329F0E3
:1044B000803209F410823196F8CF40E061E08091BB
:1044C000EB169091EC160E94E7CA0C94412E809155
:1044D000FA09882319F081E08093F9090E941B945E
:1044E0000C94412E1092F90980915D04813011F0F5
:1044F0000C94412E82E080935D040E94407A609388
:10450000590470935A0480935B0490935C040C9458
:10451000412E8091FA09882311F40C94412E83E5F1
:104520000E94694681110C94D42E0C94412E83E490
:104530000E942046882309F450C0E1EBF2E0849108
:104540008F010F5F1F4F882321F00E943E44F80126
:10455000F6CF8091C50B811103C0E4E8F2E012C0F0
:10456000BE016F5F7F4F82EC9BE00E942BA98E0102
:104570000F5F1F4FD8018D918D01882349F10E9453
:104580003E44F8CF84918F010F5F1F4F882301F1C4
:104590000E943E44F801F6CF29E0C22E23E0D22E3D
:1045A000E12CF12C20E08091110590E00E2C02C04E
:1045B000959587950A94E2F780FD18C2AFEFEA1A45
:1045C000FA0AB2E0CB0ED11CE5E0EE16F10459F781
:1045D0008AE00E943E440C94412E8091FA0988237F
:1045E00039F08091F909882319F0EEE8F2E003C070
:1045F000E0EAF2E028C084918F010F5F1F4F88230B
:1046000021F00E943E44F801F6CF6091730C709146
:10461000740C8091750C9091760C4AE00E94454490
:104620008FE20E943E4460916F0C7091700C8091FB
:10463000710C9091720C4AE00E9445448AE00E94FD
:104640003E440C94412E84918F010F5F1F4F8823AD
:1046500011F40C94412E0E943E44F801F4CF40E046
:1046600060E08091EB169091EC160E94E7CA0C94E2
:10467000412E0E94E4840C94412E8091F90981110D
:104680000E947E648091FA09882311F40C94412ED3
:1046900080E50E946946882319F00E94114603C0F4
:1046A00080E50E942046182F482F61E08091EB168C
:1046B0009091EC160E94E7CA83E50E946946882320
:1046C00081F00E94F045AB01BC014093730C509304
:1046D000740C6093750C7093760C82EC9BE00E94D6
:1046E0001CA88091FA09882319F081E08093F909C8
:1046F00011110C94412EF2CE8091EB169091EC1694
:1047000021E02093F80940E060E00E94E7CA0C94A1
:10471000412E0E940D547B018C0120E831E541E0DF
:1047200050E00E94CFE2C9016DE671E00E94FBE516
:104730004B015C01C801B70120E13EE040E050E0E0
:104740000E94CFE2CA01B90128E130E040E050E028
:104750000E94CFE2762E672EC62ED72E3CE3232E64
:10476000312C412C512CC801B701A20191010E94AA
:10477000CFE2F62EE72ECA01B901A20191010E94F3
:10478000CFE2CB018E010F5F1F4F81149104D1F056
:10479000EF92FF927F936F936F927F92BF92AF924F
:1047A0009F928F9288EE92E09F938F931F930F9327
:1047B0000E94B3DE0FB6F894DEBF0FBECDBFE5EBAF
:1047C000FAE145C0A114B10489F0EF92FF927F9302
:1047D0006F936F927F92BF92AF9288ED92E09F931A
:1047E0008F931F930F930E94B3DEE4CFCD2879F00F
:1047F000EF92FF927F936F936F927F928CEC92E097
:104800009F938F931F930F930E94B3DED3CF892B77
:1048100069F0EF92FF927F936F9384EC92E09F9305
:104820008F931F930F930E94B3DEC4CFEF92FF923A
:1048300080EC92E09F938F931F930F930E94B3DEBF
:104840000F900F900F900F900F900F90B8CF849112
:104850007F019FEFE91AF90A882321F00E943E4464
:10486000F701F5CFB8018CEF92E00E94A8C88AE06A
:104870000E943E440C94412E83E50E9469468823A1
:1048800011F40C94412E0E940046E82E80E50E940F
:104890006946882339F00E940046182F87FF03C01D
:1048A0000C94412E1DE089E40E946946882351F052
:1048B0000E94114681110C944C2FECE1F5E08CE440
:1048C00095E00AC089E40E942046F4CF31968E1705
:1048D0009F0711F40C944C2F24911213F7CF0C94D2
:1048E000212F0E941B940C94412E80915D048130F5
:1048F00011F00C94412E82E080935D040E94407A76
:104900006093590470935A0480935B0490935C0401
:104910000C94412E88E690E00E94A08F81110C94A7
:10492000412E8091110583FF02C00C94412E83E536
:104930000E946946882399F00E94F7430E946BE425
:10494000CB010E94F94A0E94F74320E030E044EB9B
:1049500052E40E94E1DE181614F00E943F940E9477
:10496000C3C80C94412E8EE40E946946882311F43A
:104970000C94412E0E94F0456093C9167093CA169C
:104980008093CB169093CC160C94412E83E50E9415
:104990002046882359F083E50E946946882319F050
:1049A0000E94004601C080E080931105E5EBFAE12A
:1049B00084918F010F5F1F4F811103C0E7E1F3E086
:1049C00004C00E943E44F801F3CF84918F010F5F31
:1049D0001F4F882321F00E943E44F801F6CF8091BA
:1049E00011058111D9CDE3E1F3E018C0BB24B394E4
:1049F000B20E222319F08CE20E943E44F60185910A
:104A00009491FC0184918F010F5F1F4F882321F047
:104A10000E943E44F801F6CF2B2DD0CD84918F011A
:104A20000F5F1F4F882309F4D3CD0E943E44F80145
:104A3000F5CF109226020C94412E8EE193E00E9455
:104A400003670E94C19D0C94412E83E50E94694634
:104A5000811103C0E5EBFAE10DC00E9400468D33E1
:104A600020F480930F020C94412E8CE380930F026C
:104A70000C94412E84918F010F5F1F4F882321F0EA
:104A80000E943E44F801F6CF40910F0250E060E0F2
:104A900070E087E293E00E9455C88AE00E943E449D
:104AA0000C94412E89E690E00E94A08F811111C0E4
:104AB000EEE2F3E084918F010F5F1F4F882321F016
:104AC0000E943E44F801F6CF0E94934B8AE00E9478
:104AD0003E44109224050C94612F83E50E946946A0
:104AE000882311F40C94412E0E940046182F8D3318
:104AF00008F01CE3109331050E94407A6B017C01A1
:104B0000212F30E0A8EEB3E00E9417E3C60ED71EB7
:104B1000E81EF91EC0922D05D0922E05E0922F05B9
:104B2000F09230050C94412E0E94C4820C94412EC8
:104B30008091110583FF02C00C94412E83E50E94F1
:104B40006946882311F40C94412E0E94F7430E9479
:104B50006BE46E36710514F06EE670E070932D0410
:104B600060932C040E946D4C0C94412E0E94967A06
:104B70000C94412E80E50E946946811106C083E5B0
:104B80000E946946882361F006C00E940046811198
:104B90000C94412EF4CF0E94F0456F3F710510F048
:104BA0006FEF70E070932B0460932A040C94412EF5
:104BB00080E50E946946811106C010922B04109274
:104BC0002A040C94412E0E94F045672B11F00C949E
:104BD000412EF3CF0E94B94C0E94CAC110922B04FF
:104BE00010922A0468EE73E080E090E00E94EB539C
:104BF0000E947B2F0C94412E10920B040C94412E9A
:104C000081E080930B040C94412E83E50E94694659
:104C10008823A1F00E94F74320E030E04AE754E403
:104C20000E9446DF0E9470E46093100270931102AC
:104C300080931202909313020C94412E88E50E94F7
:104C4000204681110C94E52E89E50E9420468111B1
:104C50000C94E52E8AE50E94204681110C94E52EE5
:104C600085E40E94204681110C94E52E0E94CAC161
:104C70000C94412E83E50E942046882311F40C9465
:104C8000412E0E94F74320E030E04AE754E40E94BE
:104C900046DF0E9470E46093290570932A05809393
:104CA0002B0590932C05EDC783E6C82E82E0D82E05
:104CB00094E3E92E91E1F92E10E0D6018D916D017A
:104CC0000E942046882309F46DC0133009F063C0A8
:104CD0000E94F7434B015C0120E030E040EA51E4E0
:104CE0000E94E1DE87FF4EC0A50194016091401152
:104CF0007091411180914211909143110E9403E4FF
:104D00002B013C019B01AC016091E0047091E10436
:104D10008091E2049091E3040E9446DF6093E004F6
:104D20007093E1048093E2049093E304A301920161
:104D30006091000570910105809102059091030535
:104D40000E9446DF60930005709301058093020581
:104D500090930305609110117091111180911211BF
:104D6000909113110E94E5DEA30192010E9446DF9B
:104D70000E9470E4609310117093111180931211CE
:104D8000909313118092401190924111A092421180
:104D9000B092431107C00E94F743F701608371830B
:104DA000828393831F5FF4E0EF0EF11C143009F04F
:104DB00084CF0E9464CA65C70E947E6483E50E9416
:104DC0006946882309F432C90E94F04562307105B2
:104DD00009F02CC90E94146F8BE50E943E4460913B
:104DE0001705709118058091190590911A0542E0F8
:104DF0000E94CA4440911B0550911C0560911D05FD
:104E000070911E0584E393E00E9472C840911F05D3
:104E100050912005609121057091220581E393E076
:104E20000E9472C88DE50E943E448AE00E943E4482
:104E300028C784918F010F5F1F4F882321F00E94A4
:104E40003E44F801F6CF60E086E094E00E9442A57F
:104E500061E08FEF93E00E9442A561E084EF93E070
:104E60000E9442A561E084EE93E00E9442A560E0CA
:104E70008BED93E00E9442A561E081ED93E00E94FA
:104E800042A561E087EC93E00E9442A561E08FEBD0
:104E900093E00E9442A561E081EB93E00E9442A56D
:104EA00060E083EA93E00E9442A560E084E993E039
:104EB0000E9442A560E086E893E00E9442A560E07F
:104EC00080E793E00E9442A560E08FE593E00E94B6
:104ED00042A560E08AE493E00E9442A561E087E396
:104EE00093E00E9442A5CDC6D8019C91292F2B7F2B
:104EF000213419F08150C1F717C011962C9121333C
:104F0000C9F7913421F0953421F441E002C0DD2449
:104F1000D39498012E5F3F4F89012F5F3F4FF801D7
:104F200090819032C9F3E6CF442369F0E5EBFAE1D2
:104F300084917F012FEFE21AF20A882321F00E9468
:104F40003E44F701F5CFDD2069F0ECEDF4E084910B
:104F50007F013FEFE31AF30A882321F00E943E44C9
:104F6000F701F5CFD8018D918D01882309F430CB5D
:104F70000E943E44F7CF0E94E9C583C681E080933A
:104F80008605809385057DC610928605109285055D
:104F900078C688EC90E00E94A08F811172C684E4EC
:104FA0000E942046882309F441C00E94F7436B0108
:104FB0007C0111E020E030E0A9010E94E1DE8111D6
:104FC00001C010E01093F71020E030E0A901C70104
:104FD000B6010E94E1DE882349F10E94F743E09187
:104FE0008004B4E0EB9FF0011124E450FF4E608395
:104FF00071838283938320E030E0A9016091FC10EB
:105000007091FD108091FE109091FF100E94E1DEE2
:1050100081110CC080E090E0A0EEBFE38093FC1013
:105020009093FD10A093FE10B093FF100E94B3C2A6
:1050300028C603E6E02E02E0F02E04E111E1F701BC
:1050400081917F010E942046882351F00E94F743FE
:105050000E9470E4D8016D937D938D939C93139778
:105060000C5F1F4FB1E104321B0749F70E94F3C8E0
:1050700008C613E6E12E12E0F12E04EF14E0F7016A
:1050800081917F010E942046882341F00E94F743CE
:10509000D8016D937D938D939C9313970C5F1F4F55
:1050A000B5E004301B0759F7ECC583E50E9469465B
:1050B0008823A1F00E94F7436093EC047093ED0401
:1050C0008093EE049093EF046093E8047093E904F6
:1050D0008093EA049093EB0410E001C011E080E5B6
:1050E0000E946946882359F00E94F7436093EC04BC
:1050F0007093ED048093EE049093EF0410E082E54A
:105100000E946946882359F00E94F7436093F00497
:105110007093F1048093F2049093F30410E084E51B
:105120000E946946882359F00E94F7436093E8047F
:105130007093E9048093EA049093EB04A2C51123D1
:1051400009F49FC54091EC045091ED046091EE0488
:105150007091EF0486EE94E00E9472C84091F004D2
:105160005091F1046091F2047091F30483EE94E0A5
:105170000E9472C84091E8045091E9046091EA04E9
:105180007091EB0480EE94E00E9472C88AE00E9465
:105190003E4477C50E94B3A474C51F5FB4E0EB0E14
:1051A000F11C133011F40C941620F60181916F015B
:1051B0000E942046882389F30E94F743D7016D930C
:1051C0007D938D939C931397812F0E94608FE5CFE1
:1051D0000E9409B6811155C503E015E1EAE1F4E04A
:1051E000F9AFE8AF9E012F5F3F4F5901FCE58F2ECD
:1051F000F5E19F2E1901F8016591759185919491C2
:10520000A8ADB9ADCD90DD90ED90FD90B9AFA8AF50
:10521000A70196010E9426E32B013C01F101608366
:1052200071838283938320E030E040EA51EC0E9456
:105230004DE587FD0AC020E030E040EA51E4C301BB
:10524000B2010E94E1DE18162CF4F40184911816C4
:105250000CF4EDC5D101CD90DD90ED90FD901D01D8
:1052600020E030E040EA51ECC701B6010E944DE574
:1052700087FD0AC020E030E040EA51E4C701B601F2
:105280000E94E1DE18164CF5E0EAFAE184918F0104
:105290000F5F1F4F811103C0E6EFF4E004C00E94CE
:1052A0003E44F801F3CF84918F010F5F1F4F882395
:1052B00021F00E943E44F801F6CF88E290E099A3E5
:1052C00088A388EC90E09DA78CA7BE01605E7F4F0D
:1052D000CE018C960E9409B9D4C40C5F1F4FBFEF5A
:1052E0008B1A9B0AE5E10F301E0709F084CFE8E82E
:1052F000EE2EE5E0FE2E10E0F50181919191A19155
:10530000B1915F01F70181939193A193B1937F01D3
:10531000812F0E94608F1F5F133071F70E9479A563
:1053200083E992E09DA78CA704E610E019A308A3E7
:10533000BE01645D7F4FCE0180960E9409B98AEB61
:1053400092E09DA78CA719A308A3BE01645D7F4FBF
:10535000CE0180960E9409B994C40E94D5A391C43D
:1053600083E50E946946882309F48BC40E94F045B6
:10537000709301026093000284C48DED90E00E945E
:10538000A08F81117EC483E50E946946811103C00C
:10539000E5EBFAE13BC00091800410E00E94F0458B
:1053A000000F111FF801E55BFD4F71836083809151
:1053B000800490E08C01000F111F000F111F980155
:1053C000285F3D4F7901880F991FFC01E55BFD4F78
:1053D00060817181072E000C880B990B0E94E7DE1B
:1053E0002AE037ED43E25CE30E9446DFF801E85033
:1053F000FF4E20813181428153810E9446DFD701D7
:105400006D937D938D939C9313973BC484918F01EF
:105410000F5F1F4F882321F00E943E44F801F6CF12
:1054200085E40E943E4480918004805D0E943E4459
:10543000E0918004F0E0EE0FFF1FE55BFD4F60811F
:10544000718184E195E00E948FC885E20E943E440C
:105450008AE00E943E4415C480E50E9420468823CD
:1054600009F40FC40E94F0456B017C0183E50E94A2
:105470006946882321F00E94F0458B0102C00FEF9E
:105480001FEFC8010196039708F0FBC3D7FCF9C3CF
:105490002C2DECE1F5E08CE495E03491231709F430
:1054A000D0C431968E179F07C1F7CEC480E50E9405
:1054B0002046882309F4E5C30E94F0456B017C0176
:1054C0008B01672B19F0E0EAFAE17FC083E50E94C7
:1054D0002046811103C0E5EBFAE107C00E94F045C8
:1054E00086ED99E00E9420C7CCC384917F01BFEF75
:1054F000EB1AFB0A882321F00E943E44F701F5CF06
:1055000060E070E085E695E00E948FC88091D80940
:1055100028E532E06901C81AD10887FDD394CC0C84
:10552000DD1CCC0CDD1C0D2C000CEE08FF0880915E
:10553000D70928E830E04901881A910887FD93943B
:10554000880C991C880C991C092C000CAA08BB0813
:105550008091D6098F3FB9F090E0FC01EE0FFF1F5C
:105560008E0F9F1FFC01E759F64F0181128183E0E6
:10557000000F111F8A95E1F794E0169507959A950B
:10558000E1F70E5F1F4F98012F5F3F4FC901330FA7
:10559000AA0BBB0B9C01AD01281939094A095B090B
:1055A000A4EBB0E00E940DE3A70196012819390988
:1055B0004A095B090E94F1E2B90182E695E00E9486
:1055C0008FC88AE00E943E445CC384918F010F5FC4
:1055D0001F4F882321F00E943E44F801F6CFB60108
:1055E0008BE595E00E948FC8ECE4F5E084918F0193
:1055F0000F5F1F4F882309F444C30E943E44F80103
:10560000F5CF83E50E946946882319F00E94F04592
:1056100002C064E071E079A368A380E50E94694656
:10562000882339F00E94F0456938E3E17E0730F4C1
:1056300002C068EE73E07A83698304C088E893E16E
:105640009A838983BE01605E7F4FCE0101960E94DE
:1056500009B917C30E9432A314C383E50E942046F0
:10566000182F882371F00E94F7430E946BE4709317
:105670000D0260930C0221E0672B09F020E02093DB
:10568000100580E50E942046882359F020910C02E5
:1056900030910D02232B11F00E94114680931005CA
:1056A000F0C21111EEC2E5EBFAE184918F010F5FB8
:1056B0001F4F882321F00E943E44F801F6CF8091CD
:1056C0001005882319F06BE273E002C06EE273E00C
:1056D00082E895E00E94A8C860910C0270910D02CA
:1056E00081E795E00E948FC8EDE6F5E084918F0197
:1056F0000F5F1F4F882309F4C4C20E943E44F80183
:10570000F5CF80E50E942046882351F00E94F743A0
:1057100060936604709367048093680490936904AF
:1057200089E40E942046882381F00E94F7432CEAF6
:1057300035EC47E25EE30E9446DF609362047093BB
:105740006304809364049093650484E40E9420467B
:10575000882381F00E94F7432CEA35EC47E25EE3B0
:105760000E9403E460935E0470935F04809360047E
:1057700090936104E5EBFAE184918F010F5F1F4F75
:10578000882321F00E943E44F801F6CF4091660440
:105790005091670460916804709169048DE995E007
:1057A0000E9472C82CEA35EC47E25EE36091620425
:1057B0007091630480916404909165040E9403E4F5
:1057C000AB01BC0189E995E00E9472C82CEA35EC76
:1057D00047E25EE360915E0470915F048091600433
:1057E000909161040E9446DFAB01BC0185E995E020
:1057F0000E9472C88AE00E943E4443C20E943E4416
:10580000F80184918F010F5F1F4F8111F7CFE1EAFB
:10581000F5E084918F010F5F1F4F882309F431C297
:105820000E943E44F801F5CF0E947E642AC281E0C6
:105830000E94C38E0E9479A524C289E40E94694611
:10584000882321F00E94F045162F01C01FEF8AE443
:105850000E946946882321F00E94F045062F01C06E
:105860000FEF8AE50E942046F82E811105C081E5E0
:105870000E942046D82E01C0D12C17FD06C007FD7E
:1058800004C0F1101CC0D1101AC0E0EAFAE1849102
:105890008F010F5F1F4F811103C0EFECF5E004C0D3
:1058A0000E943E44F801F3CF84918F010F5F1F4F98
:1058B000882309F4E6C10E943E44F801F5CF153073
:1058C00010F40530D0F0E0EAFAE184918F010F5F27
:1058D0001F4F811103C0E0EBF5E004C00E943E447D
:1058E000F801F3CF84918F010F5F1F4F882309F4D4
:1058F000C8C10E943E44F801F5CFE12E110FFF0808
:10590000002E000C110B0E94F743DD2099F025E0DA
:105910002E9DF0012F9DF00D1124E00FF11FEE0FD1
:10592000FF1FEE0FFF1FED58FF4E20813181428196
:10593000538103C020E030E0A901A5E0AE9DF00155
:10594000AF9DF00D11240E0F1F1F000F111F000F30
:10595000111F0D581F4E0E9427E3D8016D937D93B0
:105960008D939C9313978DC10E945B758AC10E9491
:1059700069B487C183E50E942046882321F00E94F4
:10598000114691E089270E9486AF7BC181E0809318
:105990007D050E94516F10927D05882309F471C125
:1059A000E5EBFAE184918F010F5F1F4F811103C076
:1059B000EFEEF5E004C00E943E44F801F3CF84917D
:1059C0008F010F5F1F4F882309F45BC10E943E4483
:1059D000F801F5CF8091F909882309F452C181E0DB
:1059E0008093FC094EC18AE50E946946811103C07B
:1059F000EDEFF5E00BC00E94F74360936F107093DA
:105A0000701080937110909372103BC184918F013C
:105A10000F5F1F4F882321F00E943E44F801F6CF0C
:105A200040916F10509170106091711070917210D0
:105A30008AEF95E00E9472C88AE00E943E4421C12C
:105A40008AE50E946946811103C0E5EBFAE13BC09B
:105A50000E94F7436B017C0120E030E040EA51EC0A
:105A60000E944DE587FD0AC020E030E040EA51E4A5
:105A7000C701B6010E94E1DE18161CF4E0EAFAE163
:105A80000CC0C0921504D0921604E0921704F09254
:105A90001804F7C00E943E44F80184918F010F5F03
:105AA0001F4F8111F7CFECE1F6E084918F010F5F7A
:105AB0001F4F882309F4E5C00E943E44F801F5CF4A
:105AC0000E943E44F80184918F010F5F1F4F8111A6
:105AD000F7CFECE3F6E084918F010F5F1F4F88232F
:105AE00021F00E943E44F801F6CF409115045091F8
:105AF0001604609117047091180489E396E00E94DF
:105B000072C88AE00E943E44BCC08BE40E94694691
:105B1000811103C0E5EBFAE136C08BE40E946946CF
:105B20008823C1F00E94F7436B017C0120E030E044
:105B3000A9010E944DE587FD0AC020E030E040E267
:105B400051E4C701B6010E94E1DE181634F4EBE41B
:105B5000F6E00EC0C12CD12C76010E947E64C0926A
:105B6000E404D092E504E092E604F092E70489C0F0
:105B700084918F010F5F1F4F882309F482C00E9418
:105B80003E44F801F5CF84918F010F5F1F4F8823AA
:105B900021F00E943E44F801F6CF4091E404509178
:105BA000E5046091E6047091E7048AE696E00E94BD
:105BB00072C88AE00E943E4464C081E08093030280
:105BC00083E50E946946882339F00E9411468111BD
:105BD00058C00E9418D055C083E50E942046F7CFD8
:105BE0000E943DB94EC0F090ED160E947E64109167
:105BF000EE1080E00E944593FF2029F1E5EBFAE1E9
:105C000084918F010F5F1F4F882321F00E943E4433
:105C1000F801F6CF84E50E943E446F2D70E080E0ED
:105C200090E04AE00E94454480E20E943E44E7E85A
:105C3000F6E084918F010F5F1F4F882311F10E94BE
:105C40003E44F801F6CF10922305812F0E94459320
:105C5000E5EBFAE184918F010F5F1F4F882321F05C
:105C60000E943E44F801F6CF6091230570E085E77D
:105C700096E00E948FC88AE00E943E4402C00E94C3
:105C80003DB9109224050E94FBCF1BC10E948C7C61
:105C90000E94366BF6CF0E947E6480E00E9445939E
:105CA00080EA90E00E94118D80E00E941C8D0E948D
:105CB000968D11E01093860588E50E942046B82E47
:105CC00089E50E942046082F8AE50E942046A82EDA
:105CD000B11004C0011104C01A2505C0011102C091
:105CE00010E001C01A2D0E94344482E50E946946EA
:105CF000882361F00E94F7436B017C0120E030E0D3
:105D0000A9010E94E1DE882371F106C0C12CD12CCB
:105D100070EAE72E70E4F72E111104C0B11002C032
:105D2000002391F1C0924605D0924705E0924805C4
:105D3000F0924905A7019601609122047091230415
:105D400080912404909125040E94E1DE87FF0BC01E
:105D500019821A821B821C82BE016F5F7F4F86E40C
:105D600095E00E94A58E111105C0B11003C001116C
:105D700006C00AC080E00E9426651123C1F381E0BD
:105D80000E942665111102C0AA2019F082E00E942B
:105D900026650E94FE9280918505809386050E946B
:105DA0007D8D0E9479A56DCF0E94F045AB01BC01AD
:105DB0004093730C5093740C6093750C7093760C35
:105DC00082EC9BE00E941CA85CCF0E947E6488E568
:105DD0000E942046882331F05F9A809119048E7FBB
:105DE0008093190489E50E942046882339F08A9A15
:105DF000479A809119048D7F809319048AE50E9447
:105E00002046882361F080910801809581708093FD
:105E10000601479A809119048B7F8093190485E4C9
:105E20000E942046882309F42CCF129A2ACFF7FA31
:105E3000F094F7F8F094F101C082D182E282F3820B
:105E400009CA0E94DDD71DCF0E947E64BC2C60E091
:105E50008C2D0E94B0B90F3FFFEF1F0759F48C2D16
:105E60000E945AB931E020E0892B09F030E0032F7D
:105E7000122F05C00130110561F401E010E08B2DF7
:105E80000E945AB98017910709F4FBCE0E9455670A
:105E9000F6CF00E010E0F3CF61E0812F0E94B0B9AF
:105EA0006E2D812F0E9482B9F12CB701812F0E94A3
:105EB0006FBA193009F0E5CEF0922B04E0922A0473
:105EC000E0CEC559DF4F0FB6F894DEBF0FBECDBF91
:105ED000DF91CF911F910F91FF90EF90DF90CF90C6
:105EE000BF90AF909F908F907F906F905F904F90FA
:105EF0003F902F9008952F923F924F925F926F9212
:105F00007F928F929F92AF92BF92CF92DF92EF9249
:105F1000FF920F931F93CF93DF93CDB7DEB76F97A9
:105F20000FB6F894DEBF0FBECDBFC0903404D09042
:105F30003504E0903604F090370420E030E040EA89
:105F400050E4C701B6010E94E1DE87FD34C120E0C4
:105F500030E041E953E4C701B6010E944DE518164F
:105F60000CF429C11092160E1092150E80910901A1
:105F70004091140E042E000C550B817021E08227F5
:105F800090E04817590709F452C0809109018170C7
:105F900028272093140E811126C00E94E786E7E18E
:105FA000FEE084918F01882351F0082E000C990B9C
:105FB0000E94E2860F5F1F4FF8018491F4CF8DE0BD
:105FC00090E00E94E2868AE090E00E94E286ECEE99
:105FD000FDE084918F010F5F1F4F882341F10E94E4
:105FE0003E44F801F6CFE5E4FEE084918F0188237A
:105FF00051F0082E000C990B0E94E2860F5F1F4F94
:10600000F8018491F4CF8DE090E00E94E2868AE06E
:1060100090E00E94E286EBE1FEE084918F010F5F49
:106020001F4F882321F00E943E44F801F6CF809153
:10603000070E833009F457C02CF4882351F08130C7
:10604000D9F073C0843009F449C0853009F458C0D0
:106050006CC08091F909882309F467C081E08093BE
:10606000070E0E94407A60930B0E70930C0E809383
:106070000D0E90930E0E59C08091F909811155C0F3
:106080008091C50B882321F082E08093070E4DC0DC
:106090001092070EE8EEFDE084918F01882351F005
:1060A000082E000C990B0E94E2860F5F1F4FF8012B
:1060B0008491F4CF8DE090E00E94E2868AE090E047
:1060C0000E94E286E0ECFDE084918F010F5F1F4F9C
:1060D000882359F10E943E44F801F6CF8091540E76
:1060E000882391F222C08091F90981111EC080910C
:1060F000330990913409891B8F7009F493C015C03E
:106100008091F909811111C080913309909134096E
:10611000891B8F7009F4BCC008C086E49DE0909391
:106120002407809323070E940A908091FC0D909190
:10613000FD0D039724F5BAE0CB2ED12CE12CF12CE8
:1061400082E69FE00E94334018161906C4F480913D
:10615000FC0D9091FD0D049794F482E69FE00E945F
:10616000F73F8093020EE091030EF091040E8A3007
:1061700019F08D3009F0B3C0309709F0B9C08091A3
:10618000FC0D9091FD0D009711F40C94913F019737
:106190009093FD0D8093FC0D8091FE0D9091FF0D6D
:1061A000019664E070E00E940FE69093FF0D8093EB
:1061B000FE0D0C94913F8091150E9091160E813634
:1061C000FAEE9F0748F11092160E1092150EEFE7A7
:1061D000FEE084918F01882351F0082E000C990B6A
:1061E0000E94E2860F5F1F4FF8018491F4CF8DE08B
:1061F00090E00E94E2868AE090E00E94E286E9E474
:10620000FEE084918F010F5F1F4F882309F4AECE0B
:106210000E943E44F801F5CF01969093160E8093AC
:10622000150EA4CE8CEA9DE090932407809323075B
:106230000E940A908091540E882311F082E001C0E0
:1062400084E08093070EE8EAFDE084918F018823C3
:1062500051F0082E000C990B0E94E2860F5F1F4F31
:10626000F8018491F4CF8DE090E00E94E2868AE00C
:1062700090E00E94E286E9E7FDE084918F010F5FE4
:106280001F4F882309F451CF0E943E44F801F5CFF7
:10629000E5E7FDE084918F01882351F0082E000C82
:1062A000990B0E94E2860F5F1F4FF8018491F4CF93
:1062B0008DE090E00E94E2868AE090E00E94E28613
:1062C0001092070EEAE4FDE084918F010F5F1F4FEB
:1062D000882309F422CF0E943E44F801F5CF8A3387
:1062E00009F44ACFEF35F10514F40C94D03B44CFB8
:1062F0008091000E9091010EA0E69A2E989E50017A
:10630000999EB00C112485010458134FE00FF11F22
:10631000108261E470E0C8010E9471E6009711F4F8
:106320000C94B43B9093060E8093050E801B910B4A
:106330008A0D9B1D60E070E08358934F0E94E2DA63
:106340000E946BE42B013C0168307105B4F06431AC
:10635000710509F485C68091000E9091010E989EFA
:10636000B001999E700D11246458734F81E39DE034
:106370000E94A8C88AE00E943E44052C000C6608D2
:106380007708F2E24F16510410F00C94B43BF2017E
:106390008827EE58FF4F8F4F0C9422E6ECE2FDE089
:1063A00084918F01882351F0082E000C990B0E94D4
:1063B000E2860F5F1F4FF8018491F4CF20E030E0B8
:1063C00040E05FE3609134047091350480913604BD
:1063D000909137041EC0E7E2FDE084918F0188238D
:1063E00051F0082E000C990B0E94E2860F5F1F4FA0
:1063F000F8018491F4CF6091320470913304072E38
:10640000000C880B990B0E94E7DE20E030E040E0B2
:106410005FE30E9427E30E946BE4CB010E94EC48FB
:106420000E94D6CC8DE090E00E94E2868AE090E067
:106430000E94E2860C94B43BE2E2FDE084918F017D
:10644000882351F0082E000C990B0E94E2860F5F02
:106450001F4FF8018491F4CF20E030E040E05FE38B
:1064600060912E0470912F0480913004909131043A
:10647000D0CFEDE1FDE084918F01882351F0082E0B
:10648000000C990B0E94E2860F5F1F4FF801849168
:10649000F4CF60912C0470912D04B1CF20912A0487
:1064A00030912B0444E6429FC001439F900D11247C
:1064B0006FEF70E00E940FE68B016536710510F0FA
:1064C00004E610E0E8E1FDE084915F01882359F0E3
:1064D000082E000C990B0E94E286FFEFAF1ABF0A4C
:1064E000F5018491F3CFB80180E090E006C6E4E1C5
:1064F000FDE084918F01882351F0082E000C990B48
:106500000E94E2860F5F1F4FF8018491F4CF80E272
:1065100090E00E94E286E0E1FDE084918F01882313
:1065200051F0082E000C990B0E94E2860F5F1F4F5E
:10653000F8018491F4CF60911A0470911B0480914A
:106540001C0490911D040E9417CD80E290E00E94EF
:10655000E286ECE0FDE084918F01882351F0082E63
:10656000000C990B0E94E2860F5F1F4FF801849187
:10657000F4CF60911E0470911F04809120049091CB
:1065800021040E9417CD80E290E00E94E286E8E0BC
:10659000FDE084918F01882351F0082E000C990BA7
:1065A0000E94E2860F5F1F4FF8018491F4CF609143
:1065B00022047091230480912404909125040E9468
:1065C00017CD80E290E00E94E2862CCF8091F909FD
:1065D000882309F450C0E3E0FDE084918F01882313
:1065E00051F0082E000C990B0E94E2860F5F1F4F9E
:1065F000F8018491F4CF8091FA09882359F18091B0
:10660000C50B882329F180916F0C9091700CA0919B
:10661000710CB091720C0097A105B105C1F0BC01DD
:10662000CD016D597F4F8F4F9F4F24E630E040E002
:1066300050E00E94CFE26091730C7091740C8091D5
:10664000750C9091760C0E94CFE2822F01C080E001
:1066500090E0E4CEEFEFFCE084918F01882309F411
:10666000E1CE082E000C990B0E94E2860F5F1F4FAF
:10667000F8018491F3CFE7EFFCE084918F01882348
:1066800009F4D0CE082E000C990B0E94E2860F5F11
:106690001F4FF8018491F3CFE2EFFCE084918F016A
:1066A000882351F0082E000C990B0E94E2860F5FA0
:1066B0001F4FF8018491F4CF80910B0E90910C0E36
:1066C000A0910D0EB0910E0E892B8A2B8B2B09F405
:1066D0007BC00E94407A20E63AEE40E050E00E9403
:1066E000CFE249015A0160910B0E70910C0E80911E
:1066F0000D0E90910E0E20E63AEE40E050E00E9422
:10670000CFE28401021B130BC8016CE370E00E940E
:10671000FBE5CB019927EAE0F0E0BF010E940FE61C
:10672000282FCB01BF010E940FE6805D80930D04EE
:10673000205D20930E0410920F048DE094E00E94DF
:10674000D6CC80E290E00E94E286E0EFFCE084910B
:106750005F01882359F0082E000C990B0E94E286F5
:10676000FFEFAF1ABF0AF5018491F3CF80E290E00A
:106770000E94E286C8016CE370E00E94FBE56AE0DB
:1067800070E00E940FE6605D60930D04805D809371
:106790000E0410920F048DE094E00E94D6CC80E2AB
:1067A00090E00E94E286EEEEFCE084918F01882367
:1067B00009F438CE082E000C990B0E94E2860F5F78
:1067C0001F4FF8018491F3CF80E290E00E94E286AF
:1067D000E6EEFCE084918F01882309F423CE082E95
:1067E000000C990B0E94E2860F5F1F4FF801849105
:1067F000F3CF1092350E8091090180FF11C0E2EEB7
:10680000FCE084918F01882309F40CCE082E000C43
:10681000990B0E94E2860F5F1F4FF8018491F3CF1E
:1068200083E50E94B2CC882341F00E94CDCC0E9427
:1068300070E470930A0E6093090EEEEDFCE0849113
:106840008F01882351F0082E000C990B0E94E286DC
:106850000F5F1F4FF8018491F4CF8DE090E00E940C
:10686000E2868AE090E00E94E2868091530E8823BF
:1068700009F4F3C08091090E90910A0E009741F03F
:10688000049709F0A2C2EFEAF7E084918F01C1C03A
:10689000E6E3F8E084918F01882351F0082E000C84
:1068A000990B0E94E2860F5F1F4FF8018491F4CF8D
:1068B0008DE090E00E94E2868AE090E00E94E2860D
:1068C000EFE2F8E084918F01882351F0082E000C4C
:1068D000990B0E94E2860F5F1F4FF8018491F4CF5D
:1068E0008DE090E00E94E2868AE090E00E94E286DD
:1068F000E8E1F8E084918F01882351F0082E000C24
:10690000990B0E94E2860F5F1F4FF8018491F4CF2C
:106910008DE090E00E94E2868AE090E00E94E286AC
:10692000E1E0F8E084918F01882351F0082E000CFB
:10693000990B0E94E2860F5F1F4FF8018491F4CFFC
:106940008DE090E00E94E2868AE090E00E94E2867C
:10695000EDEEF7E084918F01882351F0082E000CB2
:10696000990B0E94E2860F5F1F4FF8018491F4CFCC
:106970008DE090E00E94E2868AE090E00E94E2864C
:10698000E9EDF7E084918F01882351F0082E000C87
:10699000990B0E94E2860F5F1F4FF8018491F4CF9C
:1069A0008DE090E00E94E2868AE090E00E94E2861C
:1069B000EBECF7E084918F01882351F0082E000C56
:1069C000990B0E94E2860F5F1F4FF8018491F4CF6C
:1069D0008DE090E00E94E2868AE090E00E94E286EC
:1069E000EDEBF7E084918F01882351F0082E000C25
:1069F000990B0E94E2860F5F1F4FF8018491F4CF3C
:106A00008DE090E00E94E2868AE090E00E94E286BB
:106A1000DCC1882351F0082E000C990B0E94E286FD
:106A20000F5F1F4FF8018491F4CF8DE090E00E943A
:106A3000E2868AE090E00E94E286E1EAF7E0849153
:106A40008F018823E9F2082E000C990B0E94E28640
:106A50000F5F1F4FF8018491F4CF8091FA098823CA
:106A600009F48AC181E08093770C1092790C10921E
:106A7000780C89E49AE00E9463AA8BE1E9E4FAE0E9
:106A8000DE01159601900D928A95E1F78091470AF3
:106A90009091480A9C838B8389EF92E09A83898343
:106AA00040E050E0BE016F5F7F4F80E090E00E94C9
:106AB0003489CE0101960E94E0668090780C909017
:106AC000790C0091090E10910A0EC401801B910BE4
:106AD000049720F04801F3E08F0E911C5BE6252E11
:106AE00057E0352E62E9462E67E0562E73E8672E92
:106AF00077E0772E8016910608F467C1011511051D
:106B000009F0A1C06DEF79E089E49AE00E942BA919
:106B100062E373E08DEF99E00E947CE6892B09F037
:106B20004AC0F201849142E9A42E47E0B42E8823A2
:106B300059F0082E000C990B0E94E286FFEFAF1A65
:106B4000BF0AF5018491F3CF8DE090E00E94E286C8
:106B50008AE090E00E94E286F301849133E8A32E5C
:106B600037E0B32E882359F0082E000C990B0E94B1
:106B7000E286FFEFAF1ABF0AF5018491F3CF8DE0F3
:106B800090E00E94E2868AE090E00E94E2864AE07D
:106B900060E070E0CB010E944544E3E7F7E08491B8
:106BA0005F012FEFA21AB20A882309F4E2C00E9403
:106BB0003E44F501F4CFEFE6F7E084915F018823CE
:106BC00059F0082E000C990B0E94E286FFEFAF1AD5
:106BD000BF0AF5018491F3CF8DE090E00E94E28638
:106BE0008AE090E00E94E286F10184912BE6A22ED9
:106BF00027E0B22E882359F0082E000C990B0E9432
:106C0000E286FFEFAF1ABF0AF5018491F3CF8DE062
:106C100090E00E94E2868AE090E00E94E2864AE0EC
:106C200060E070E0CB010E944544E6E6F7E0849125
:106C30005F012FEFA21AB20A882309F49AC00E94BA
:106C40003E44F501F4CF60E070E0C80101970E9476
:106C5000FA8A8091FB09882309F45FC0E4E6F7E033
:106C600084915F01882359F0082E000C990B0E9433
:106C7000E286FFEFAF1ABF0AF5018491F3CF8DEFE3
:106C800099E00E94D6CC8DE090E00E94E2868AE0F6
:106C900090E00E94E286E2E6F7E084915F018823BB
:106CA00059F0082E000C990B0E94E286FFEFAF1AF4
:106CB000BF0AF5018491F3CF8AE09AE00E94D6CC16
:106CC0008DE090E00E94E2868AE090E00E94E286F9
:106CD000C801A0E0B0E04AE0BC01CD010E944544FB
:106CE000E0E6F7E084915F012FEFA21AB20A882351
:106CF00021F00E943E44F501F5CF9AE0A92E9AE0DA
:106D0000B92EF50181915F01882319F00E943E445C
:106D1000F8CF8AE00E943E442CC08DEF99E00E949B
:106D2000D6CC8DE090E00E94E2868AE090E00E945E
:106D3000E2868AE09AE00E94D6CC8DE090E00E9444
:106D4000E2868AE090E00E94E286C801A0E0B0E01E
:106D50004AE0BC01CD010E9445448AE0A82E8AE0A9
:106D6000B82EF50181915F01882399F20E943E447B
:106D7000F8CF0F5F1F4FBECEE1E5F7E084918F01A2
:106D8000882351F0082E000C990B0E94E2860F5FB9
:106D90001F4FF8018491F4CF8DE090E00E94E286CD
:106DA0008AE090E00E94E286E2E4F7E084918F01BD
:106DB000882309F425CE082E000C990B0E94E28648
:106DC0000F5F1F4FF8018491F3CFEAEDFCE084914F
:106DD0008F01882309F426CB082E000C990B0E9402
:106DE000E2860F5F1F4FF8018491F3CF8091F9097C
:106DF000882339F00E944988B7C48091F909882313
:106E000089F10E94F3B5B0C48091070E823019F069
:106E1000833609F0A9C40E942988E6EDFCE084913C
:106E20008F01882351F0082E000C990B0E94E286F6
:106E30000F5F1F4FF8018491F4CF8DE090E00E9426
:106E4000E2868AE090E00E94E286EBEAFCE0849130
:106E50008F010F5F1F4F882309F486C40E943E44B0
:106E6000F801F5CF8091070E833609F07DC4C9CFB4
:106E700082EA9CE00E940367809133099091340973
:106E8000891B8F7009F070C48091070E823009F45D
:106E90006BC4833609F09CC467C480913309909118
:106EA0003409891B8F7009F05FC48091070E82300E
:106EB00009F45AC4833609F457C48091C50B811173
:106EC00004C552C483E50E94B2CC811126C083E47C
:106ED0000E94B2CC882309F447C480913309909171
:106EE0003409891B8F7009F03FC420E030E040E294
:106EF00051E46091220470912304809124049091C4
:106F000025040E94E1DE87FF08C089E09CE09093A1
:106F10002407809323070E940A900E94CDCC20E092
:106F200030E0A9010E94E1DE87FD10C00E94CDCCB7
:106F300020E030E849E853E40E944DE518164CF093
:106F40000E94CDCC0E9470E4CB0105C080E090E0AF
:106F500002C083E191E00E94F94A06C483E50E94E1
:106F6000B2CC882309F400C40E94CDCC20E030E0EC
:106F7000A9010E94E1DE87FD11C00E94CDCC20E076
:106F800030E046E153E40E944DE518164CF00E94B3
:106F9000CDCC0E9470E4362F272F04C030E001C012
:106FA00036E920E0832F922F8E36910514F08EE67D
:106FB00090E090932D0480932C040E946D4CD4C3D8
:106FC00083E50E94B2CC8823D9F00E94CDCC20E08A
:106FD00030E04FE753E40E9446DF20E030E048EC29
:106FE00052E40E9403E40E9470E46F3F710519F0BF
:106FF00010F06FEF70E070932B0460932A0412CAB4
:107000008FEF90E090932B0480932A040BCA809119
:10701000330990913409891B8F7009F003CA80915C
:10702000F9098111FFC90E94C19D5F9A80911904DD
:107030008E7F809319048A9A479A809119048D7FD4
:1070400080931904809108018095817080930601D6
:10705000479A809119048B7F80931904129AE2C990
:1070600083E50E94B2CC882319F10E94CDCC20E0A8
:1070700030E040E252E40E94E1DE87FD0FC00E9452
:10708000CDCC20E030EC49E754E40E944DE51816E1
:1070900044F00E94CDCC0E946BE405C068E270E031
:1070A00002C067EE73E070930102609300025CC35C
:1070B000E3E0FCE084918F01882351F0082E000C5E
:1070C000990B0E94E2860F5F1F4FF8018491F4CF65
:1070D0008090000290900102092C000CAA08BB08C5
:1070E000B7FE0DC06DE282E69FE034D766277727B2
:1070F000CB01681979098A099B094AE003C04AE073
:10710000C501B4010E94D7CC8DC9809133099091FB
:107110003409891B8F7009F027C38091070E8230D4
:1071200009F422C3833609F0EDC21EC380913309EE
:1071300090913409891B8F7009F074C98091070EF2
:10714000823009F46FC9833609F0F3C36BC98091AB
:10715000330990913409891B8F7009F005C3809120
:10716000070E823009F400C3833609F038C5FCC22B
:107170008091330990913409891B8F7009F0F4C212
:107180008091070E823009F4EFC2833609F05DC5A5
:10719000EBC28091330990913409891B8F7009F0FB
:1071A000E3C28091070E823009F4DEC2833609F013
:1071B00082C5DAC28091350E811103C00E94E78634
:1071C00024C18E3271F58091360E8E3209F0A6C040
:1071D00080919A0B882309F418C1815080939A0BEF
:1071E000882361F090E001974FE1489F9001499F0B
:1071F000300D1124C9018C59954F02C086E29AE0E6
:107200002BE1FC013496A9E4BAE001900D922A9595
:10721000E1F7FC01828193819093480A8093470AA9
:10722000F4C08C3309F07AC064E373E085E39EE038
:107230000E947CE6892B21F481E08093530EE5C007
:1072400063E473E085E39EE00E947CE6892B79F499
:10725000E5E2F7E084918F010F5F1F4F882321F053
:107260000E943E44F801F6CF88E197E044C06AE509
:1072700073E085E39EE00E947CE6892B79F4E7EFDA
:10728000F6E084918F010F5F1F4F882321F00E9449
:107290003E44F801F6CF8FEE96E02DC06EE673E027
:1072A00085E39EE00E947CE6892B79F4E4EDF6E02C
:1072B00084918F010F5F1F4F882321F00E943E446D
:1072C000F801F6CF8FEC96E016C06CE773E085E32B
:1072D0009EE00E947CE6892BA9F4E4EBF6E0849121
:1072E0008F010F5F1F4F882321F00E943E44F80159
:1072F000F6CF8FEA96E090932407809323070E94AD
:107300000A9083C06AE873E085E39EE00E947CE611
:10731000892B09F07AC01092530E77C01D8218860F
:107320001C821B8289EF92E09A83898380914C0AA8
:10733000811103C066E27AE002C065E47AE061157B
:10734000710519F06C5F7F4F02C060E070E021E0D2
:1073500045E35EE0CE0105960E9499AE882361F177
:107360008BE1FE013596A9E4BAE001900D928A9571
:10737000E1F72B813C813093480A2093470A8091A2
:107380009A0B8A3008F03DC091E0980F90939A0BC9
:10739000FFE18F9FC0011124DC01A859B54F4BE1DB
:1073A000E9E4FAE001900D924A95E1F7FC01EC590D
:1073B000F54F3383228325C0E5EBFAE184918F01F9
:1073C0000F5F1F4F882321F00E943E44F801F6CF43
:1073D000E9E9F6E084918F010F5F1F4F882321F0C8
:1073E0000E943E44F801F6CF05E31EE0F8018191CA
:1073F0008F01882319F00E943E44F8CF8AE00E9452
:107400003E44CE0101960E94E0661092350E8091B6
:10741000090180FFA9C1E0E2FBE084918F0188238C
:1074200051F0082E000C990B0E94E2860F5F1F4F4F
:10743000F8018491F4CF8DE090E00E94E2868AE02A
:1074400090E00E94E286E2EFFAE084918F010F5F04
:107450001F4F882309F488C10E943E44F801F5CFEC
:107460008FE40E94B2CC81110C94123283E40E940A
:10747000B2CC0C94123283E50E94B2CC882369F01E
:10748000E5EDFAE084918F010F5F1F4F882309F427
:10749000C5C00E943E44F801F5CF8FE40E94B2CCF3
:1074A000882379F0E3EAFAE084918F010F5F1F4FA0
:1074B000882321F00E943E44F801F6CF8BE69AE043
:1074C00013C084E50E94B2CC8823A9F0E6E4FAE078
:1074D00084918F010F5F1F4F882321F00E943E444B
:1074E000F801F6CF8EE19AE090932407809323076A
:1074F0000E940A9093C083E40E94B2CC882379F062
:10750000EAEFF9E084918F010F5F1F4F882321F08C
:107510000E943E44F801F6CF81ED99E0E5CF81E588
:107520000E94B2CC882379F0EDEAF9E084918F01D2
:107530000F5F1F4F882321F00E943E44F801F6CFD1
:1075400085E899E0D1CF88E40E94B2CC882389F104
:10755000E6E6F9E084918F010F5F1F4F882321F049
:107560000E943E44F801F6CFE2E6F9E084918F01F3
:10757000882351F0082E000C990B0E94E2860F5FC1
:107580001F4FF8018491F4CF8DE090E00E94E286D5
:107590008AE090E00E94E286EFE2F9E084918F01B8
:1075A0000F5F1F4F882309F439C00E943E44F80141
:1075B000F5CF8CE40E94B2CC882381F1E3E1F9E0BD
:1075C00084918F010F5F1F4F882321F00E943E445A
:1075D000F801F6CFEFE0F9E084918F01882351F0B4
:1075E000082E000C990B0E94E2860F5F1F4FF801D6
:1075F0008491F4CF8DE090E00E94E2868AE090E0F2
:107600000E94E286EFECF8E084918F010F5F1F4F3C
:10761000882321F00E943E44F801F6CFE6E5FBE026
:1076200084918F01882311F40C941232082E000CDF
:10763000990B0E94E2860F5F1F4FF8018491F2CFF1
:107640008091330990913409891B8F7011F00C944B
:1076500012328091070E823011F40C94123283366C
:1076600009F057C30C94123283E50E94B2CC8823F0
:1076700009F47AC0EFE6F8E084918F010F5F1F4FA5
:10768000882321F00E943E44F801F6CF87E498E079
:1076900090932407809323070E940A90E6E5FBE07D
:1076A00084918F01882311F40C941232082E000C5F
:1076B000990B0E94E2860F5F1F4FF8018491F2CF71
:1076C000E2E4F8E084918F01882351F0082E000C49
:1076D000990B0E94E2860F5F1F4FF8018491F4CF4F
:1076E000EDE3F8E084918F01882311F40C941232B9
:1076F000082E000C990B0E94E2860F5F1F4FF801C5
:107700008491F2CF88E50E94B2CC811106C089E550
:107710000E94B2CC882309F4FEC088E50E94B2CC56
:10772000882341F08DEF9BE09093240780932307FB
:107730000E940A9089E50E94B2CC882341F087EF2D
:107740009BE090932407809323070E940A908AE588
:107750000E94B2CC882341F081EF9BE090932407F4
:10776000809323070E940A908091000E9091010E51
:10777000019664E070E00E940FE69093010E809302
:10778000000E8091FC0D9091FD0D01969093FD0DE2
:107790008093FC0D1092040E1092030E0C94A030F6
:1077A0004091000E5091010E9F012F5F3F4F30938B
:1077B000040E2093030E90E6949F9001959F300D48
:1077C00011242458334FE20FF31F80830C94A03010
:1077D0000091050E1091060E580124E0A20EB11C76
:1077E0006AE270E0C5010E9471E6F80124812F323F
:1077F00021F4B8016B5F7F4F03C02C3339F4B5011E
:1078000085E39EE00E9485E60C9412321092350EBC
:10781000009719F0FC01319710828091050E90912C
:10782000060E40E061E004960E94E7CA8091C50B15
:10783000882331F1EEE9FCE084918F01882351F037
:10784000082E000C990B0E94E2860F5F1F4FF80173
:107850008491F4CF8DE090E00E94E2868AE090E08F
:107860000E94E286EFE6FCE084918F010F5F1F4FDC
:10787000882311F40C9412320E943E44F801F4CF94
:10788000EBE6FCE084918F01882351F0082E000C78
:10789000990B0E94E2860F5F1F4FF8018491F4CF8D
:1078A0008DE090E00E94E2868AE090E00E94E2860D
:1078B000E0E4FCE084918F010F5F1F4F882311F4F7
:1078C0000C941232DBD7F801F5CF0E942988ECE343
:1078D000FCE084918F01882351F0082E000C990B55
:1078E0000E94E2860F5F1F4FF8018491F4CF8DE074
:1078F00090E00E94E2868AE090E00E94E286E0E169
:10790000FCE084918F010F5F1F4F882309F42CCF77
:10791000B5D7F801F6CF8AE50E94B2CC8111FDCE31
:1079200083E40E94B2CC882309F41ECF8DEE9BE045
:1079300015CF86E40E94B2CC882309F44DC10E9481
:10794000CDCC0E9470E48B0189EE9BE090932407DC
:10795000809323070E940A9088E50E94B2CC882376
:1079600009F451C00E94CDCC2B013C012DEC3CEC24
:107970004CE45EE30E94E1DE9E012F5F3F4F590120
:10798000181674F020E030E0A901C301B2010E9492
:107990004DE518162CF41F930F938EED9BE005C157
:1079A0002DEC3CEC4CEC5DEBC301B2010E94E1DE3E
:1079B00018167CF020E030E040E85FEBC301B20134
:1079C0000E944DE518162CF41F930F9382ED9BE057
:1079D000ECC01F930F93C301B2010E946BE47F932D
:1079E0006F9388EC9BE09F938F93BF92AF920E941E
:1079F000B3DE0FB6F894DEBF0FBECDBFCE01019649
:107A00000E94E28FDFC089E50E94B2CC882309F48E
:107A100041C00E94CDCC2B013C012DEC3CEC4CE450
:107A20005EE30E94E1DEFE0131965F01181674F0FC
:107A300020E030E0A901C301B2010E944DE5181613
:107A40002CF41F930F938DEB9BE0AFC02DEC3CEC1F
:107A50004CEC5DEBC301B2010E94E1DE18167CF034
:107A600020E030E040E85FEBC301B2010E944DE549
:107A700018162CF41F930F9381EB9BE096C01F9375
:107A80000F93C301B2010E946BE47F936F9387EA67
:107A90009BE0A9CF8AE50E94B2CC882309F441C0BB
:107AA0000E94CDCC2B013C012DEC3CEC4CE45EE380
:107AB0000E94E1DEFE0131965F01181674F020E0AD
:107AC00030E0A901C301B2010E944DE518162CF463
:107AD0001F930F938CE99BE068C02DEC3CEC4CECC1
:107AE0005DEBC301B2010E94E1DE18167CF020E0DC
:107AF00030E040E85FEBC301B2010E944DE518168B
:107B00002CF41F930F9380E99BE04FC01F930F93BA
:107B1000C301B2010E946BE47F936F9386E89BE000
:107B200062CF85E40E94B2CC882309F44BC00E9446
:107B3000CDCC2B013C012DEC3CEC4CE45EE30E94EF
:107B4000E1DEFE0131965F01181674F020E030E0AE
:107B5000A901C301B2010E944DE518162CF41F9330
:107B60000F938BE79BE021C02DEC3CEC4CEC5DEBE4
:107B7000C301B2010E94E1DE18167CF020E030E083
:107B800040E85FEBC301B2010E944DE518162CF4EA
:107B90001F930F938FE69BE008C0C301B2010E94C0
:107BA0006BE47F936F9384E69BE09F938F93BF92E8
:107BB000AF920E94B3DE0F900F900F900F900F9036
:107BC0000F901CCF80E69BE09093240780932307BF
:107BD0000E940A900C94123200E010E0B5CE20E032
:107BE00030E040E251E460912204709123048091DE
:107BF0002404909125040E94E1DE87FF08C089E5F6
:107C00009BE090932407809323070E940A9082E3CD
:107C100090E090932D0480932C040E946D4C88EC8E
:107C200090E00E94F94AE6E5FBE084918F01882309
:107C300011F40C941232082E000C990B0E94E2866B
:107C40000F5F1F4FF8018491F2CF20E030E040E257
:107C500051E4609122047091230480912404909156
:107C600025040E94E1DE87FF08C08FE49BE090932B
:107C70002407809323070E940A9080E590E0909368
:107C80002D0480932C040E946D4C80EF90E00E94A4
:107C9000F94AE6E5FBE084918F01882311F40C9406
:107CA0001232082E000C990B0E94E2860F5F1F4FC4
:107CB000F8018491F2CF80E090E00E94F94A10929E
:107CC0002D0410922C040E946D4CEBE4FBE0849197
:107CD0008F01882351F0082E000C990B0E94E28638
:107CE0000F5F1F4FF8018491F4CF8DE090E00E9468
:107CF000E2868AE090E00E94E286E4E2FBE0849182
:107D00008F010F5F1F4F882309F42ECDB7D5F801DF
:107D1000F6CF83E50E94B2CC882309F475C0EAEC63
:107D2000F8E084918F01882351F0082E000C990B04
:107D30000E94E2860F5F1F4FF8018491F4CF20E08C
:107D400030E048EC52E46091150470911604809183
:107D50001704909118040E9446DF20E030E040E0D4
:107D60005FE30E9427E30E946BE4CB010E94EC4892
:107D70000E94D6CC8DE090E00E94E2868AE090E0FE
:107D80000E94E286EDE9F8E084918F010F5F1F4FBA
:107D9000882319F073D5F801F7CFE8E9F8E084916A
:107DA0008F010F5F1F4F882319F068D5F801F7CFB7
:107DB00020E030E048EC52E4609115047091160424
:107DC00080911704909118040E9446DF20E030E073
:107DD00040E05FE30E9427E30E946BE4CB010E9436
:107DE000EC488C01F80181918F01882311F046D570
:107DF000F9CFE5E9F8E084918F010F5F1F4F8823E9
:107E000019F03CD5F801F7CF84E40E94B2CC882366
:107E100011F40C9412320E94CDCC20E030E048ECFA
:107E200052E40E9403E420E030E048EC52E40E9477
:107E300046DF0E946BE44B015C0197FD0EC020E120
:107E400037E240E050E00E94F1E2CA01B901A70127
:107E500096010E94F1E2605D09C0B094A0949094F4
:107E60008094811C911CA11CB11C6DE260930E04D6
:107E7000C501B40128EE33E040E050E00E94F1E299
:107E8000CA01B901A70196010E94F1E2605D609309
:107E90000F04C501B40124E630E040E050E00E9448
:107EA000F1E2CA01B901A70196010E94F1E2605D09
:107EB000609310048EE280931104C501B401A70100
:107EC00096010E94F1E2162FCA01B901A70196019D
:107ED0000E94F1E2605D60931204105D1093130440
:107EE0008EE898E09F938F938E010F5F1F4F1F9333
:107EF0000F930E94B3DE6EE074E0C8010E9466E654
:107F0000C8010E94E28F89E898E09093240780934B
:107F100023070E940A900F900F900F900F900C94DF
:107F200012326F960FB6F894DEBF0FBECDBFDF9151
:107F3000CF911F910F91FF90EF90DF90CF90BF9066
:107F4000AF909F908F907F906F905F904F903F90F9
:107F50002F9008950F931F93CF93DF93FC01A68575
:107F6000B7858D0100581F4FE801888199810196DE
:107F70008F779927AD014E575F4FEA0128813981EC
:107F800028173907D1F3E80128813981A20FB31FDF
:107F90006C93A685B785A058BF4F11969C938E937E
:107FA000A689B7892C9181E090E0078C02C0880FE8
:107FB000991F0A94E2F7822B8C9381E081A30488B5
:107FC000F589E02D80818064808381E090E0DF91FD
:107FD000CF911F910F910895FC0181A1882329F071
:107FE000A489B5898C9186FFFBCF11A20895FC016D
:107FF000A485B585FD01E058FF4F2081318132967F
:10800000808191812817390779F080819181A80FAB
:10801000B91F8C91208131812F5F3F4F2F773327FC
:108020003183208390E008958FEF9FEF0895DC0166
:108030001C96ED91FC911D97DF01A058BF4F2D912B
:108040003C91119712968D919C91119728173907A1
:1080500039F08D919C91E80FF91F808190E008958F
:108060008FEF9FEF0895FC0124853585F901E058D5
:10807000FF4F8081918132962081318180589F4FBE
:10808000821B930B60E870E00C940FE6089508954E
:1080900080E090E008952F923F924F925F926F920E
:1080A0007F928F929F92AF92BF92CF92DF92EF9288
:1080B000FF920F931F93CF93DF9300D000D0CDB7E3
:1080C000DEB79A8389830E94407AE981FA81C6806B
:1080D000D780E084F184C114D104E104F10409F0F3
:1080E000ACC22485222309F469C332852150248738
:1080F00021E0230F22874585241301C01286E981E0
:10810000FA8124E0329FE00DF11D1124C684D7844A
:10811000E088F188E981FA81C282D382E482F58223
:10812000DC01CB018C0D9D1DA11DB11D86839783A4
:10813000A087B18784819581892B09F43FC3FFB75C
:10814000FD83F894E981FA81228033802101612C3A
:10815000712C04811581809107028F3121F08F3FAE
:1081600009F068C205C0EBE3F3E124912E83DAC085
:108170008FE180930702EBE3F3E184918E838F3FDD
:1081800009F458C2823009F469C030F5882309F433
:108190004CC0813009F0C6C010928000109281005E
:1081A000809181008860809381008091810081604E
:1081B00080938100E2E5FBE2E491F0E0EE0FFF1F27
:1081C000E150F54D85919491E8E9FBE2E491E0936B
:1081D0003B04E1E0EE8330C19E81943009F482C01B
:1081E00008F460C0953009F09DC0109220011092F3
:1081F00021018091210188608093210180912101DA
:10820000816080932101E2E5FBE2E491F0E0EE0F72
:10821000FF1FE150F54D85919491E8E9FBE2E4916F
:10822000E093380495E09E8307C114BC15BC84B567
:10823000826084BD85B5816085BDE2E5FBE2E491A5
:10824000F0E0EE0FFF1FE150F54D85919491E8E9C4
:10825000FBE2E491E0933C041E82ABC21092B000BA
:108260001092B1008091B00082608093B000809144
:10827000B10081608093B100E2E5FBE2E491F0E0BF
:10828000EE0FFF1FE150F54D85919491909382047C
:1082900080938104E8E9FBE2E491E0938304F2E057
:1082A000FE8387C2109290001092910080919100FD
:1082B000886080939100809191008160809391000B
:1082C000E2E5FBE2E491F0E0EE0FFF1FE150F54D37
:1082D00085919491E8E9FBE2E491E0933A0423E08C
:1082E0002E83AAC01092A0001092A1008091A1003C
:1082F00088608093A1008091A10081608093A1009B
:10830000E2E5FBE2E491F0E0EE0FFF1FE150F54DF6
:1083100085919491E8E9FBE2E491E093390484E0EB
:108320008E838AC0EE81E7FD85C161E08FE10E9406
:10833000B0B98E818D7F09F083C04801A12CB12C8A
:1083400060E072E18AE790E0A50194010E94F1E209
:1083500029833A834B835C8369017A01F1E0CF1A68
:10836000D108E108F1082FEFC216D104E104F104AD
:1083700009F008F44EC060E472E48FE090E0A501DB
:1083800094010E94F1E269017A0181E0C81AD108E2
:10839000E108F1089E81923009F5EFEFCE16D10485
:1083A000E104F10409F008F4CBC160E970ED83E069
:1083B00090E0A50194010E94F1E269017A01F1E0E7
:1083C000CF1AD108E108F1082FEFC216D104E10459
:1083D000F10411F008F041C183E027C08FEFC81607
:1083E000D104E104F104B9F0B0F068E478EE81E082
:1083F00090E0A50194010E94F1E269017A0191E007
:10840000C91AD108E108F108EE81EE2309F49AC1F6
:1084100063C181E001C082E09E81911106C095B5E3
:10842000987F892B85BD7AC085E09091B100987FB7
:10843000892B8093B10072C061E08FE10E94B0B9D6
:108440004801A12CB12C60E072E18AE790E0A5011F
:1084500094010E94F1E269017A01E1E0CE1AD108AB
:10846000E108F108C114D104F1E0EF06F10488F04D
:1084700068E478EE81E090E0A50194010E94F1E2C9
:1084800069017A0181E0C81AD108E108F10883E0A6
:1084900001C081E09E81913071F490918100987FBC
:1084A000892B80938100452846284728D9F52FEF4E
:1084B0003FEFA90168C0EE81E33071F49091910023
:1084C000987F892B8093910045284628472851F5AD
:1084D0002FEF3FEFA90179C0FE81F43071F4909144
:1084E000A100987F892B8093A10045284628472822
:1084F000C9F42FEF3FEFA9017AC02E81253071F426
:1085000090912101987F892B80932101452846284D
:10851000472841F42FEF3FEFA9017BC045284628AB
:10852000472869F0D801AA0FBB1F91010E9417E3E9
:1085300028EE33E040E050E00E94CFE203C02FEF8E
:108540003FEFA9018E81823081F12CF4882361F004
:108550008130C9F06FC09E81943009F448C0ACF1FD
:10856000953009F456C066C0C7BC20934D043093C3
:108570004E0440934F045093500480916E008260EB
:1085800080936E0057C0D0928900C09288002093DB
:10859000490430934A0440934B0450934C04809117
:1085A0006F00826080936F0045C0C092B30020933B
:1085B000840430938504409386045093870480910B
:1085C000700082608093700035C0D0929900C09294
:1085D00098002093450430934604409347045093F9
:1085E00048048091710082608093710023C0D09212
:1085F000A900C092A8002093410430934204409304
:10860000430450934404809172008260809372000E
:1086100011C0D0922901C092280120933D043093CB
:108620003E0440933F045093400480917300826065
:1086300080937300ED81EFBFC1C0DC01CB018C19C9
:108640009D09AE09BF09B7FDB9C04698E981FA8115
:108650001682178210861186B1C068E478EE81E038
:1086600090E0A50194010E94F1E269017A01F1E034
:10867000CF1AD108E108F1082FEFC216D104E104A6
:10868000F10441F138F164E274EF80E090E0A5017B
:1086900094010E94F1E269017A01F1E0CF1AD10858
:1086A000E108F1082FEFC216D104E104F10409F04A
:1086B00008F4BACE62E17AE780E090E0A501940187
:1086C0000E94F1E269017A0181E0C81AD108E1084B
:1086D000F10819C084E0A9CE2FEFC216D104E1043D
:1086E000F10409F008F463C062E17AE780E090E009
:1086F000A50194010E94F1E269017A01F1E0CF1A2B
:10870000D108E108F1082FEFC216D104E104F10409
:10871000A9F0A0F089819A81AB81BC812AE0B5954E
:10872000A795979587952A95D1F76C017D01F1E082
:10873000CF1AD108E108F10887E077CE86E075CE40
:1087400082E073CEEFEFCE16D104E104F10469F1BB
:1087500060F162E17AE780E090E0A50194010E9477
:10876000F1E269017A0181E0C81AD108E108F10853
:108770009FEFC916D104E104F104A9F0A0F08981AA
:108780009A81AB81BC813AE0B595A795979587957D
:108790003A95D1F76C017D01E1E0CE1AD108E108EC
:1087A000F10885E03CCE84E03ACE83E038CE84E028
:1087B00033CE61E08FE10E94B0B9BFCD26960FB6EF
:1087C000F894DEBF0FBECDBFDF91CF911F910F9107
:1087D000FF90EF90DF90CF90BF90AF909F908F90E1
:1087E0007F906F905F904F903F902F9008950F93E0
:1087F0001F93CF938091060490910704009711F185
:10880000FC018F01C1912C2F2F7DA9F0C53411F0EF
:10881000C536B9F7F801108260E070E08091060477
:10882000909107040E94E2DAF801C083562F472F87
:10883000382F292F0BC060E070E0CF911F910F916E
:108840000C94E2DA50E040E030E020E0652F742F35
:10885000832F922FCF911F910F910895FC012381B7
:1088600021110C9406A9089580E1EAE1F4E0AEE359
:10887000B5E001900D928A95E1F708959091C000BE
:1088800095FFFCCF8093C60008958F929F92AF9280
:10889000BF92EF92FF920F931F93CF93DF93CDB7C9
:1088A000DEB7A0970FB6F894DEBF0FBECDBF61153F
:1088B00071058105910589F100E0842E912CA12C90
:1088C000B12C102FEE24E394F12CEC0EFD1EE00EE3
:1088D000F11C07FDFA94A50194010E94CFE2F70173
:1088E0006083B901CA010F5F6115710581059105AA
:1088F00041F71F3F21F1E1E0F0E0EC0FFD1FE10F38
:10890000F11D17FDFA9580818A3010F097E301C0C0
:1089100090E3890FB3DF1150ECCF80E3A0960FB640
:10892000F894DEBF0FBECDBFDF91CF911F910F91A5
:10893000FF90EF90BF90AF909F908F909FCFA096A9
:108940000FB6F894DEBF0FBECDBFDF91CF911F9160
:108950000F91FF90EF90BF90AF909F908F900895F0
:10896000CF92DF92EF92FF926B017C0197FF0AC0DA
:108970008DE284DFF094E094D094C094C11CD11CAB
:10898000E11CF11C4AE0C701B601FF90EF90DF90B7
:10899000CF907BCF8F929F92AF92BF92CF92DF9278
:1089A000EF92FF92CF936B017C01B42E20E030E078
:1089B000A9010E94E1DE87FF06C08DE25FDFF7FAC2
:1089C000F094F7F8F094C0E060E070E080E09FE39E
:1089D000CB1541F02DEC3CEC4CEC5DE30E9446DF06
:1089E000CF5FF6CF9B01AC01C701B6010E9427E320
:1089F0006B017C010E9470E44B015C014AE045DFA1
:108A0000CC2379F1C501B4010E94E5DE9B01AC01E4
:108A1000C701B6010E9426E36B017C018EE22EDFC6
:108A200020E030E040E251E4C701B6010E9446DF99
:108A30004B015C010E946BE46B01770FEE08FF08AD
:108A4000C701B6018DDFC701B6010E94E7DE9B01B9
:108A5000AC01C501B4010E9426E36B017C01C15049
:108A6000F9F6CF91FF90EF90DF90CF90BF90AF904D
:108A70009F908F900895809170179091711798171B
:108A800059F0E92FF0E0E051F94E80819F5F9F7728
:108A90009093711790E008958FEF9FEF08951F92C4
:108AA0000F920FB60F9211240BB60F922F938F9344
:108AB0009F93EF93FF9320917117E091701781E0DE
:108AC0008E0F8F779091C600281729F0F0E0E051C3
:108AD000F94E9083E82FE0937017FF91EF919F91EB
:108AE0008F912F910F900BBE0F900FBE0F901F9084
:108AF00018958F929F92AF92BF92CF92DF92FF9282
:108B00000F931F93CF93DF93EC01C07F6B018FE036
:108B1000C82ACC15DD0508F057C08E01CE010E9491
:108B2000EFC45C01F50181915F01882311F0A6DE9D
:108B3000F9CF8AE3A3DE5E01F12CF50181915F019B
:108B40000E9420C54C01F40181914F01882311F04E
:108B500095DEF9CF80E292DEF394F0E1FF1631F07A
:108B6000F8E0FF12EACF8DE289DEE7CF69E170E03D
:108B700080E090E00E94EB538CE780DE6096F80185
:108B80008081F5E009391F0748F095E9093919078F
:108B900028F490EE980F9F3530F002C0853E11F416
:108BA00080E201C08FE36ADE0F5F1F4FC017D1075D
:108BB00031F78AE063DE69E170E080E090E00E94D6
:108BC000EB530E945567A5CFDF91CF911F910F9175
:108BD000FF90DF90CF90BF90AF909F908F900895BF
:108BE0008091060490910704009731F04AE050E02C
:108BF00060E070E00C9435DC60E070E0CB0108953B
:108C0000EFDF97FD0AC0ECDF6F3F7105810591052D
:108C100009F02CF4E5DF862F089580E008958FEFAA
:108C200008958091060490910704892B31F0E8DFC4
:108C300091E0811103C090E001C091E0892F089577
:108C400081548A3108F042C0E82FF0E04091E716E5
:108C50005091E8166091E9167091EA1604C0769575
:108C60006795579547958A95D2F7842F817040FF75
:108C70002FC0E353F94E9081992309F1E091D81068
:108C8000F091D910E90FF11D908120ED290F2A30C4
:108C900098F09E3211F491810CC09D3211F09B32FC
:108CA00071F4918120ED290F2A3030F09E3239F491
:108CB000928190539A3018F42E2F9F2F02C020E0FB
:108CC00090E02093060490930704089580E00895AF
:108CD0000895B6DF882341F081E0209106043091A9
:108CE0000704232B09F480E008952F923F924F92BE
:108CF0005F926F927F928F929F92AF92BF92CF922C
:108D0000DF92EF92FF920F931F93CF93DF9300D0E8
:108D1000CDB7DEB780919E1790919F170E94EFC448
:108D200060E472E084E890E10E94A8C884EA97E1D8
:108D30000E94EFC460E472E086E790E10E94A8C858
:108D400000919E1710919F170115110511F404EA67
:108D500017E1C8010E94EFC460E472E08EE590E183
:108D60000E94A8C82E0184E0480E511CC2010E9436
:108D7000EFC460E472E08CE490E10E94A8C88AE04D
:108D80007DDD809102028111CAC189E459DF811120
:108D9000C6C11FC07801E8E0EE0EF11CA60165EE29
:108DA0007FEFC7010E944CE6B6010D2C000C880B2A
:108DB000990BD6DDE2E9FEE084915F019FEFA91AED
:108DC000B90A8111CFC1A12CB12CAC14BD040CF493
:108DD000CCC184E435DF882321F0B201C80189DEEB
:108DE000E5C186E42DDF882309F45DC1401A510AEC
:108DF000A12CB12C212C312C612C712C88248A942B
:108E0000982CA414B504E4F56801CA0CDB1CF60127
:108E10008081853E89F5E12CF12C8191853E41F0E0
:108E2000F1E0EF1AF10889E0E816F1042CF108C02E
:108E30009FEFE91AF90AE1148DE7F80671F71CC0F3
:108E4000B7018FE090E10E948FC8C6010E94EFC475
:108E500060E472E08FEF9FE00E94A8C88AE00EDD18
:108E60008E149F0414F0610101C04701AE0CBF1CB9
:108E70009FEF691A790A1601EFEFAE1ABE0AC1CF49
:108E8000F2E06F167104DCF0EDECFFE084918F01ED
:108E90000F5F1F4F882319F0F1DCF801F7CFB40101
:108EA00085EB9FE00E948FC8C1010E94EFC460E47F
:108EB00072E08AEA9FE00E94A8C88AE0DFDC01E94C
:108EC00013E0F80181918F01882311F0D7DCF9CFED
:108ED000C0909E17D0909F17C114D10421F494EA3A
:108EE000C92E97E1D92E8E010D5F1F4F5801AC1886
:108EF000BD08B5018AE79FE00E948FC88EE997E11F
:108F00000E94EFC460E472E08DE69FE00E94A8C872
:108F100080919E1790919F170E94EFC460E472E0C9
:108F20008BE69FE00E94A8C884EA97E10E94EFC404
:108F300060E472E08EE59FE00E94A8C8C8010E942C
:108F4000EFC460E472E089E59FE00E94A8C80C15B8
:108F50001D0508F5EDE4FFE084918F010F5F1F4FC1
:108F6000882319F08BDCF801F7CF64E170E080E032
:108F700090E00E94EB5309E913E0F80181918F0121
:108F8000882311F07BDCF9CF8AE078DC6FEF71E2A7
:108F900080E89BE1AEDDE12CF12C00E010E0EA146A
:108FA000FB04CCF5F601EE0DFF1D8081853E79F5C1
:108FB00060E070E08191853EC9F04B01F1E08F1ACD
:108FC000910889E08816910414F1E80CF91C0F5FF0
:108FD0001F4FB8018AE49FE00E948FC8B40181E46A
:108FE0009FE00E948FC8EDE3FFE007C06F5F7F4FF7
:108FF00061159DE77907F1F60AC084914F019FEF53
:10900000891A990A882319F039DCF401F6CFEFEFB9
:10901000EE1AFE0AC4CFB8018EE29FE00E948FC80C
:109020000130110531F480919E1790919F17892B83
:1090300089F0ECEFFEE084917F019FEFE91AF90AD5
:10904000882319F01BDCF701F6CF0115110511F487
:109050000FEF1FEFE3EFFEE084917F019FEFE91A2E
:10906000F90A882319F00ADCF701F6CF013011055F
:1090700019F0EDEEFEE007C080E300DC8AE0FEDBE5
:1090800060E070E00BC084917F019FEFE91AF90A5C
:10909000882319F0F3DBF701F6CFB80184E89FE0ED
:1090A0000E948FC839C083E4CBDD882309F47EC0D9
:1090B00097DD6B019E01201B310B3A956F5F7F4F4F
:1090C000C9010E94FBE57B01ECE2F0E184915F01C4
:1090D0009FEFA91AB90A811108C0C7010896080FA5
:1090E000191FAA24A394B12C03C0C8DBF501EECF4D
:1090F000CA14DB0488F0F801A082C8010E94EFC402
:1091000060E472E086E190E10E94A8C8FFEFAF1A28
:10911000BF0A0E0D1F1DECCF8AE0B0DB47C01092D6
:109120000202EAECFEE084917F019FEFE91AF90A5E
:10913000882319F0A3DBF701F6CF6201C01AD10A28
:10914000EAEFCE1AD108D7FE25CEE2EBFEE08491FD
:109150007F019FEFE91AF90A882309F43ACE8EDBE2
:10916000F701F5CF8BDBF50127CEF7018081853E36
:10917000B1F0C7010E94EFC460E472E085E89EE0B0
:109180000E94A8C8F70180810E9420C5BC0183E825
:109190009EE00E94A8C88AE071DB8AE06FDBFFEFE7
:1091A000AF1ABF0A8FEFE81AF80A0FCE0F900F9090
:1091B0000F90DF91CF911F910F91FF90EF90DF9073
:1091C000CF90BF90AF909F908F907F906F905F9067
:1091D0004F903F902F9008959C0197FD0EC08436CC
:1091E000910584F064E670E00E940FE6CB016AE02E
:1091F00070E00E940FE6805D06C03195219531092F
:109200008DE201C080E2809311042A30310564F0C0
:10921000EAE0F0E0C901BF010E940FE6CB01BF0107
:109220000E940FE6805D01C080E280931204C901B4
:109230006AE070E00E940FE6805D8093130481E194
:1092400094E008951F920F920FB60F9211240BB65F
:109250000F922F933F938F939F93EF93FF932091C0
:10926000DA0E3091DB0E8091DC0E9091DD0E281726
:10927000390731F4809131018F7D8093310114C021
:10928000E091DC0EF091DD0EE65AF14F20818091E5
:10929000DC0E9091DD0E01968F7799279093DD0E6D
:1092A0008093DC0E20933601FF91EF919F918F9177
:1092B0003F912F910F900BBE0F900FBE0F901F90FC
:1092C00018951F920F920FB60F9211240BB60F92A2
:1092D0002F934F935F938F939F93EF93FF9380917F
:1092E000300182FD1CC02091360180915E0F90916B
:1092F0005F0F4091600F5091610F01968F77992712
:109300004817590771F0E0915E0FF0915F0FE2523C
:10931000F14F208390935F0F80935E0F02C0809186
:109320003601FF91EF919F918F915F914F912F9116
:109330000F900BBE0F900FBE0F901F901895CF92FD
:10934000DF92EF92FF920F931F93CF93DF936C0105
:109350007A018B01C0E0D0E0CE15DF0581F0D801A5
:109360006D918D01D601ED91FC910190F081E02D80
:10937000C6011995892B11F02196EECF7E01C70108
:10938000DF91CF911F910F91FF90EF90DF90CF90E1
:109390000895AF92BF92CF92DF92EF92FF920F9318
:1093A000CF93DF935C01EB0169017A0180E266DA19
:1093B0000F3F11F084E501C082E460DA8AE35EDAEF
:1093C000F501608171818281938142E0E3DA488115
:1093D00059816A817B818FE293E10E9472C820E00B
:1093E00030E040E85DE3C701B6010E9446DFAB0113
:1093F000BC018CE293E10E9472C889E23FDA62E02C
:1094000070E080E090E0DF91CF910F91FF90EF90BE
:10941000DF90CF90BF90AF900C9436BBCF92DF928D
:10942000EF92FF92C0903404D0903504E09036045F
:10943000F0903704609132047091330466507109E2
:10944000072E000C880B990B0E94E7DE9B01AC01F4
:10945000C701B6010E94E1DE87FF1FC020E030E0B7
:1094600040E050E4C701B6010E9427E30E9470E487
:109470007093B1046093B0040E94407ADC01CB0188
:10948000805E914BAF4FBF4F8093AC049093AD047F
:10949000A093AE04B093AF0408C01092AC04109235
:1094A000AD041092AE041092AF04FF90EF90DF90E5
:1094B000CF9008951F920F920FB60F9211240BB602
:1094C0000F922F933F934F935F936F937F938F935D
:1094D0009F93AF93BF93EF93FF93809184049091F8
:1094E0008504A0918604B0918704892B8A2B8B2B4D
:1094F00059F190918304E0918104F091820480817C
:10950000892780838091840490918504A0918604AA
:10951000B0918704181619061A061B060CF056C0DF
:109520008091840490918504A0918604B091870471
:109530000197A109B1098093840490938504A093B5
:109540008604B093870442C080910702EBE3F3E105
:10955000E4919FEF90930702E230C9F050F4EE23BC
:1095600099F0E13081F590916F009D7F90936F00AD
:109570002AC0E43019F1E0F0E53029F5909173004C
:109580009D7F909373001FC010926E001CC090913D
:1095900070009D7F9093700091E09093B000909147
:1095A000B100987F94609093B1001092B3000BC00B
:1095B000909171009D7F9093710005C09091720011
:1095C0009D7F9093720060E00E9482B9FF91EF91BD
:1095D000BF91AF919F918F917F916F915F914F91CB
:1095E0003F912F910F900BBE0F900FBE0F901F90C9
:1095F0001895909333048093320480E00FCF8F92BC
:109600009F92AF92BF92CF92DF92EF92FF920F9311
:109610001F93CF93DF93F0E2FF2EE12CAE2DB0E04D
:10962000BD016F0D711D759567956E1511F0F612E0
:109630000BC0EFE0F1E165917491072E000C880BEF
:10964000990B0E94E7DE62C09B0121503109220F75
:10965000331F220F331FF901EF56FF4E059114916E
:10966000AB01440F551F440F551FFA01EF56FF4E33
:10967000C591D4918017910714F4F62ED1CFC81755
:10968000D90714F4E62ECACFF901ED56FF4EE59046
:10969000F490FA01ED56FF4EC590D490BC01601BCA
:1096A000710B072E000C880B990B0E94E7DE4B0113
:1096B0005C01B6016E197F09072E000C880B990B0F
:1096C0000E94E7DE9B01AC01C501B4010E9446DFA8
:1096D0004B015C01C01BD10BBE01DD0F880B990B48
:1096E0000E94E7DE9B01AC01C501B4010E9403E4C6
:1096F0004B015C01B701FF0C880B990B0E94E7DE60
:109700009B01AC01C501B4010E9427E3DF91CF9119
:109710001F910F91FF90EF90DF90CF90BF90AF908F
:109720009F908F900895CF92DF92EF92FF920F93C8
:109730001F93CF93DF93CDB7DEB728970FB6F8947A
:10974000DEBF0FBECDBF6091D2047091D304072E4F
:10975000000C880B990B0E94E7DE6B017C01609185
:10976000320470913304072E000C880B990B0E9471
:10977000E7DE6D837E838F83988780913404909198
:109780003504A0913604B091370489839A83AB8362
:10979000BC830DEFA7019601BE016B5F7F4FCE0129
:1097A0000196F7DD6091D0047091D104072E000C72
:1097B000880B990B0E94E7DE6B017C0160912C0401
:1097C00070912D04072E000C880B990B0E94E7DE88
:1097D0006D837E838F83988780912E0490912F04D0
:1097E000A0913004B091310489839A83AB83BC8308
:1097F0000FEFA7019601BE016B5F7F4FCE0101966F
:10980000C8DDE7E3F3E184918F010F5F1F4F8823E9
:1098100019F034D8F801F7CFE0918004F0E0E25875
:10982000FB4F608170E080E090E09AD8E2E3F3E1E2
:1098300084918F010F5F1F4F882319F01FD8F80103
:10984000F7CF60917F0470E080E090E089D828969F
:109850000FB6F894DEBF0FBECDBFDF91CF911F9141
:109860000F91FF90EF90DF90CF9008950F930FB777
:109870000F9300916E000B7F00936E0078940F930E
:109880000BB70F930CB70F921F922F933F934F93E9
:109890005F936F937F938F939F93AF93BF93EF9358
:1098A000FF93112494D1FF91EF91BF91AF919F91BC
:1098B0008F917F916F915F914F913F912F911F9069
:1098C0000F900CBF0F910BBF0F910460F8940093A1
:1098D0006E000F910FBF0F911895CF92DF92EF920C
:1098E000FF92C0902E04D0902F04E0903004F090AE
:1098F000310460912C0470912D0466507109072E7B
:10990000000C880B990B0E94E7DE9B01AC01C7019C
:10991000B6010E94E1DE87FF1FC020E030E040E09A
:1099200050E4C701B6010E9427E30E9470E47093DF
:10993000B7046093B6040E94407ADC01CB01805AE0
:109940009541AF4FBF4F8093B2049093B304A0935F
:10995000B404B093B50408C01092B2041092B304DA
:109960001092B4041092B504FF90EF90DF90CF9066
:10997000089510927A0480E090E03BDE10922D046E
:1099800010922C04AADF0E943F9480E090E031DE28
:1099900010927E042C9810922D0410922C04109298
:1099A0007F048091020180728093000108958F925C
:1099B0009F92AF92BF92CF92DF92EF92FF920F935E
:1099C0001F93CF93DF93F0E4FF2EE12CAE2DB0E098
:1099D000BD016F0D711D759567956E1511F0F6122D
:1099E0000BC0E1E8F2E165917491072E000C880B41
:1099F000990B0E94E7DE62C09B0121503109220FC2
:109A0000331F220F331FF901ED57FE4E05911491BC
:109A1000AB01440F551F440F551FFA01ED57FE4E81
:109A2000C591D4918017910714F4F62ED1CFC817A1
:109A3000D90714F4E62ECACFF901EB57FE4EE59094
:109A4000F490FA01EB57FE4EC590D490BC01601B18
:109A5000710B072E000C880B990B0E94E7DE4B015F
:109A60005C01B6016E197F09072E000C880B990B5B
:109A70000E94E7DE9B01AC01C501B4010E9446DFF4
:109A80004B015C01C01BD10BBE01DD0F880B990B94
:109A90000E94E7DE9B01AC01C501B4010E9403E412
:109AA0004B015C01B701FF0C880B990B0E94E7DEAC
:109AB0009B01AC01C501B4010E9427E3DF91CF9166
:109AC0001F910F91FF90EF90DF90CF90BF90AF90DC
:109AD0009F908F90089560E08091D2049091D3047C
:109AE0008EDD609334047093350480933604909334
:109AF00037048091D0049091D10459DF60932E04F3
:109B000070932F048093300490933104A8951092A1
:109B10007B040895DF92EF92FF920F931F93CF93F0
:109B2000DF93F82ED62EE72E8A0180910302882338
:109B300009F439C0E0EAFAE18491EF012196882323
:109B400021F00E943E44FE01F7CFED2DFE2D8491C1
:109B5000EF012196882321F00E943E44FE01F7CFB9
:109B6000E2E2F1E18491EF012196882321F00E9445
:109B70003E44FE01F7CFF7FC0BC06F2DFF0C770BB7
:109B8000880B990B0E94B0448AE00E943E440BC0AF
:109B9000EDE1F1E18491EF012196882321F00E940B
:109BA0003E44FE01F7CF80918804811108C01092D5
:109BB000030281E080938804C8010E940367DF915B
:109BC000CF911F910F91FF90EF90DF90D2CEEF9247
:109BD000FF920F931F93CF93DF93809106028F37ED
:109BE000A0F08F5790917E049093CF04992311F0A9
:109BF0002C9A01C02C9820917F042093CE04909140
:109C00000201222369F090950BC09091CF0489172F
:109C100008F02C989091CE04891728F090910201B9
:109C20009072909300018F5F809306029091CD0413
:109C300081E089278093CD048091050285301CF452
:109C4000C1E0C80F01C0C0E0823009F4B4C054F4D0
:109C5000882301F1813009F0E3C088E080937B0024
:109C600085E4C0C0843009F4C5C00CF4B7C08530A9
:109C700009F0D6C09091CC04911102C08093CC041D
:109C80008091CC0481508093CC04882309F4C8C00F
:109C9000C5E0C6C0809104028F5F80311CF48093C0
:109CA0000402BEC01092040280917B04811113C093
:109CB0008091C2049091C3049093D3048093D20402
:109CC0008091C0049091C1049093D1048093D004FA
:109CD00081E080937B048AE0E2ECF4E0DF011D92F6
:109CE0008A95E9F71092C1041092C0040091D20441
:109CF0001091D3041195019511098091320490912E
:109D00003304D1E0181619062CF080917E048111DD
:109D100001C0D0E080918105909182059195819557
:109D200091098017910734F44AEB52E16BED72E12F
:109D300080E0F0DE8091220290912302919581953E
:109D400091090817190744F4DD2331F04DEE52E173
:109D50006EE073E180E0DEDE80912C0490912D04B2
:109D600011E0181619062CF080917F04811101C0B2
:109D700010E0E090D004F090D10480917F059091A4
:109D800080058E159F0534F04AEC52E16BED72E1CF
:109D90008FEFC0DE8091200290912102E816F90633
:109DA0000CF43EC01123E1F14DEF52E16EE073E19E
:109DB0008FEFB0DE35C080917A0086FD2EC0809195
:109DC0007800909179002091C2043091C304820FF1
:109DD000931F9093C3048093C20422C088E08093B1
:109DE0007B0086E480937C0080917A00806480937D
:109DF0007A0016C080917A0086FD11C080917800AB
:109E0000909179002091C0043091C104820F931F7A
:109E10009093C1048093C00403C0C2E001C0C4E0B9
:109E2000C09305020E943BC580917C0490917D0403
:109E30000097A9F0019790937D0480937C04892B6F
:109E400071F480E293E19093240780932307DF91DC
:109E5000CF911F910F91FF90EF900C940A90DF919A
:109E6000CF911F910F91FF90EF9008952F923F9205
:109E70004F925F926F927F928F929F92AF92BF921A
:109E8000CF92DF92EF92FF920F931F93CF93DF93C6
:109E900000D01F92CDB7DEB75C017A8369834A0197
:109EA000170107FD07C0802F002E000C990B9C8323
:109EB0008B8304C0E1E0F0E0FC83EB83F901408098
:109EC0005180628073808B819C81880F991F880FDD
:109ED000991F9C838B8388549B4F7C01A301920123
:109EE000FC0160817181828193810E94E1DE88237F
:109EF00091F0F701408251826282738211E020E08A
:109F000030E0A901C301B2010E944DE518160CF022
:109F100010E0F5011083F50180818230D1F08330AB
:109F200009F45EC0813009F07CC0EB81FC81E8540B
:109F3000FB4F2081318142815381F4016081718125
:109F4000828193810E94E1DE87FD6BC082E0F50192
:109F500080838B819C8188549B4F9C838B83B6012B
:109F600080E090E00E94E5DE9B01AC01EB81FC818A
:109F700060817181828193810E9426E39B01AC0103
:109F8000F40160817181828193810E944DE587FD9A
:109F900014C00E94407A6B017C019101A8EEB3E0ED
:109FA0000E9417E3C60ED71EE81EF91EE981FA814A
:109FB000C082D182E282F38234C00E94407AE98179
:109FC000FA81C080D180E280F380DC01CB018C1962
:109FD0009D09AE09BF09B7FD24C083E0F501808368
:109FE0000F3F19F043E852E102C046E952E16AEA44
:109FF00072E1802F0F900F900F900F90DF91CF9113
:10A000001F910F91FF90EF90DF90CF90BF90AF9096
:10A010009F908F907F906F905F904F903F902F9088
:10A0200079CD0F900F900F900F90DF91CF911F91EE
:10A030000F91FF90EF90DF90CF90BF90AF909F90E7
:10A040008F907F906F905F904F903F902F900895EA
:10A050007F928F929F92AF92BF92CF92DF92EF92B8
:10A06000FF920F931F93CF93DF9320E030E048E4FB
:10A0700052E46091340470913504809136049091DB
:10A0800037040E944DE518164CF4E7E1F1E1E49144
:10A09000C1E001C0CC0FEA95EAF701C0C0E081E160
:10A0A000E82E81E1F82E07E111E196E0A92E912C2E
:10A0B000D0E0CC24C394D12CF7017490F8018490A3
:10A0C00077FC23C0892D90E0082C02C095958795D8
:10A0D0000A94E2F780FD19C0BE01082C02C07595F4
:10A0E00067950A94E2F76170B62EB1946B2D872DB7
:10A0F0000E9482B96B2D70E0872D0E946FBAC60155
:10A1000001C0880F8A94EAF7982AAA94FFEFEF1A01
:10A11000FF0A0F5F1F4FA110CFCFDF91CF911F918B
:10A120000F91FF90EF90DF90CF90BF90AF909F90F6
:10A130008F907F9008954F925F926F927F928F924F
:10A140009F92AF92BF92CF92DF92EF92FF920F93C6
:10A150001F93CF93DF93CDB7DEB760970FB6F89418
:10A16000DEBF0FBECDBF80917B04811117C060960A
:10A170000FB6F894DEBF0FBECDBFDF91CF911F9118
:10A180000F91FF90EF90DF90CF90BF90AF909F9096
:10A190008F907F906F905F904F9008959CDC0E940D
:10A1A000407A4B015C016091320470913304072EB8
:10A1B000000C880B990B0E94E7DE69837A838B83FE
:10A1C0009C8348E0C42ED12C5CE3E52EF12C00E00A
:10A1D0009E012F5F3F4F44E354E068EA74E087EA52
:10A1E00094E044DEC0903404D0903504E09036040E
:10A1F000F09037046091830570918405072E000C60
:10A20000880B990B0E94E7DE9B01AC01C701B601E8
:10A210000E944DE518160CF009C16091240270915E
:10A220002502072E000C880B990B0E94E7DE9B018C
:10A23000AC01C701B6010E94E1DE87FFF7C00091C3
:10A24000320410913304B801012E000C880B990BD5
:10A250000E94E7DEA70196010E9426E32B013C0144
:10A2600020ED3CEC4CE45DE360917204709173046A
:10A2700080917404909175040E9446DF6D837E8303
:10A280008F83988720919E0430919F044091A00471
:10A290005091A104C701B6010E9426E39B01AC01C5
:10A2A0006D817E818F8198850E9446DF6D837E83DC
:10A2B0008F83988723E333E343E75FE360919A0456
:10A2C00070919B0480919C0490919D040E9446DFB4
:10A2D0009B01AC016D817E818F8198850E9427E36F
:10A2E0006D837E838F83988760939A0470939B0419
:10A2F00080939C0490939D04C0929E04D0929F04EE
:10A30000E092A004F092A10420E030E040E251E4A9
:10A31000C301B2010E944DE518160CF430C220E0D2
:10A3200030E040E251ECC301B2010E94E1DE87FD62
:10A330002FC2012B09F42CC28091990481112CC2E7
:10A34000209195043091960440919704509198047F
:10A3500029873A874B875C8720916E0430916F0480
:10A360004091700450917104C301B2010E9446DF14
:10A370006B017C01A301920169857A858B859C859F
:10A380000E9427E369877A878B879C87609395046F
:10A3900070939604809397049093980420916A0494
:10A3A00030916B0440916C0450916D040E9446DF23
:10A3B000A70196010E9427E32D813E814F81588598
:10A3C0000E9426E36B017C0120E030E04FE753E47C
:10A3D0000E944DE520E030E0A90118160CF4E3C11D
:10A3E000C701B6010E94E1DE87FD07C0C701B601C3
:10A3F0000E946BE4759567951AC020E030E0A901D2
:10A40000C301B2010E94E1DE87FF10C0A3019201E7
:10A4100069857A858B859C850E9426E360939504E7
:10A4200070939604809397049093980460E06093EF
:10A430007E048091AC049091AD04A091AE04B091E3
:10A44000AF040097A105B10521F1A5019401281BD6
:10A45000390B4A0B5B0B57FD1CC06091B004709127
:10A46000B10480E090E00E94E5DE9B01AC016091C8
:10A4700034047091350480913604909137040E9421
:10A48000E1DE87FF81C142E651E164E771E180E0EE
:10A4900041DB8091760490917704A0917804B0918B
:10A4A0007904A5019401281B390B4A0B5B0B57FD5E
:10A4B0000FC0CEDDD501C4018C53964FAF4FBF4FB7
:10A4C0008093760490937704A0937804B0937904F2
:10A4D0008091B2049091B304A091B404B091B504FA
:10A4E0000097A105B10511F1881A990AAA0ABB0AB9
:10A4F000B7FC1CC06091B6047091B70480E090E096
:10A500000E94E5DE9B01AC0160912E0470912F0446
:10A5100080913004909131040E94E1DE87FF20C1D8
:10A5200040E451E163E571E18FEFF4DA60912C04CE
:10A5300070912D04072E000C880B990B0E94E7DE0A
:10A5400069837A838B839C8392E0C92ED12C24E18A
:10A55000E22EF12C0FEF9E012F5F3F4F4EE254E0B1
:10A5600062EA74E086EA94E081DCC0902E04D09028
:10A570002F04E0903004F090310420E030E040EA15
:10A5800050E4C701B6010E944DE587FDE5C020E01B
:10A5900030E04CED52E4C701B6010E94E1DE18162E
:10A5A0000CF4DAC060912C0470912D04072E000C7D
:10A5B000880B990B0E94E7DEA70196010E9426E313
:10A5C0004B015C012091660430916704409168045E
:10A5D000509169040E9446DF69877A878B879C8740
:10A5E00020919104309192044091930450919404ED
:10A5F000C501B4010E9427E36D837E838F83988712
:10A6000060939104709392048093930490939404C4
:10A610002091620430916304409164045091650478
:10A620000E9446DF6D877E878F87988B20ED3CECFC
:10A630004CE45DE360915E0470915F04809160047E
:10A64000909161040E9446DF2B013C0120918D0412
:10A6500030918E0440918F0450919004C701B6014F
:10A660000E9426E39B01AC01C301B2010E9446DFB8
:10A670002B013C0123E333E343E75FE3609189046B
:10A6800070918A0480918B0490918C040E9446DF23
:10A690009B01AC01C301B2010E9427E32B013C01E5
:10A6A0006093890470938A0480938B0490938C0444
:10A6B000C0928D04D0928E04E0928F04F0929004A8
:10A6C0002D853E854F85588969857A858B859C8542
:10A6D0000E9427E3A30192010E9426E36B017C0103
:10A6E00020E030E04FE753E40E944DE520E030E009
:10A6F000A9011816BCF5C501B4010E944DE5181654
:10A7000084F4A50194016D817E818F8198850E94DA
:10A7100026E3609391047093920480939304909342
:10A7200094046FE71AC020E030E0A901C501B4012C
:10A730000E94E1DE87FF10C0A50194016D817E813A
:10A740008F8198850E9426E3609391047093920410
:10A75000809393049093940460E060937F0407CD0A
:10A76000BCD8E4CEC701B6010E94E1DE87FDDBCF95
:10A77000C701B6010E946BE475956795EECF81E045
:10A78000809399046FE753CE80E00E940E4A81CEF9
:10A7900081E0809399044ACE1092990419861A8612
:10A7A0001B861C86D9CDC301B2010E944DE5181647
:10A7B0004CF7A301920169857A858B859C850E945F
:10A7C00026E3609395047093960480939704909386
:10A7D00098046FE72CCECF92DF92EF92FF926B013D
:10A7E0007C0183E3C816D104E104F10468F082E33C
:10A7F000C81AD108E108F10862E370E080E090E057
:10A800000E9436BB98DCEDCFC701B6010E9436BB73
:10A81000FF90EF90DF90CF908ECC0F931F9380919D
:10A820005D04813019F40E94407A08C06091590497
:10A8300070915A0480915B0490915C0400915504DE
:10A84000109156042091570430915804601B710BED
:10A85000820B930B28EE33E040E050E00E94CFE201
:10A860008091510490915204A0915304B0915404EA
:10A87000BC01CD01620F731F841F951F1F910F91A3
:10A88000089510925D04109255041092560410928F
:10A890005704109258041092590410925A041092BE
:10A8A0005B0410925C0410925104109252041092B6
:10A8B00053041092540408952F923F924F925F9246
:10A8C0006F927F928F929F92AF92BF92CF92DF92C0
:10A8D000EF92FF920F931F93CF93DF93CDB7DEB725
:10A8E000C857D1090FB6F894DEBF0FBECDBFE091B7
:10A8F0007C04F0917D04EF2B11F00C94255D2896DB
:10A90000DFAECEAE28976E2C79016A015B01FC01A7
:10A9100020813181428153816C962CAF3DAF4EAF87
:10A920005FAF6C9720913411309135114091361101
:10A93000509137116C966CAD7DAD8EAD9FAD6C971F
:10A940000E9446DF0E9458E5E0966CAF7DAF8EAF67
:10A950009FAFE097D5018D919D910D90BC91A02D59
:10A96000A0968CAF9DAFAEAFBFAFA097209138112E
:10A970003091391140913A1150913B11BC01CD01F8
:10A980000E9446DF0E9458E5E4966CAF7DAF8EAF23
:10A990009FAFE497D6012D913D914D915C91A49686
:10A9A0002CAF3DAF4EAF5FAFA49720913C113091DB
:10A9B0003D1140913E1150913F11A4966CAD7DAD7B
:10A9C0008EAD9FADA4970E9446DF0E9458E5E896A1
:10A9D0006CAF7DAF8EAF9FAFE897D7012D913D91C2
:10A9E0004D915C9122962CAF3DAF4EAF5FAF229759
:10A9F00020914011309141114091421150914311E9
:10AA000022966CAD7DAD8EAD9FAD22970E9446DF44
:10AA10000E9458E560966CAF7DAF8EAF9FAF609798
:10AA20008091110583FF1CC060962CAD3DAD4EADED
:10AA30005FAD60972093650930936609409367097D
:10AA40005093680922968CAD9DADAEADBFAD2297F7
:10AA50008093550990935609A0935709B0935809CC
:10AA6000D801BC91BDA3F801F181F9ABD8011296D0
:10AA7000BC91BEABF801F381FAAF8091330990919C
:10AA80003409891B8F708F3019F40E945567F5CFF8
:10AA900000913309E9960FAFE99780913309082FA8
:10AAA00010E01CA30BA38091590990915A09A09121
:10AAB0005B09B0915C09E0968CAC9DACAEACBFACD0
:10AAC000E097881A990AAA0ABB0A80915D099091B9
:10AAD0005E09A0915F09B0916009E4962CAC3DAC91
:10AAE0004EAC5FACE497281A390A4A0A5B0A809197
:10AAF000610990916209A0916309B0916409E89697
:10AB00002CAD3DAD4EAD5FADE897281B390B4A0B20
:10AB10005B0B2DA73EA74FA758AB8091650990917D
:10AB20006609A0916709B091680960960CAD1DADEA
:10AB30002EAD3FAD6097081B190B2A0B3B0B09A7E5
:10AB40001AA72BA73CA7012B022B032B09F4BCC08F
:10AB50008091100581114BC06091340470913504CF
:10AB600080913604909137040E946BE420910C028E
:10AB700030910D02621773070CF039C060962CAD4E
:10AB80003DAD4EAD5FAD609720936509309366098A
:10AB9000409367095093680922968CAD9DADAEAD88
:10ABA000BFAD22978093550990935609A0935709FA
:10ABB000B0935809E5EBFAE184918F010F5F1F4FC5
:10ABC000811103C0EBE5F3E104C00E943E44F801AB
:10ABD000F3CF84918F010F5F1F4F882321F00E94D4
:10ABE0003E44F801F6CF19A61AA61BA61CA694E0AF
:10ABF000699E80011124085F1D4F69A57AA58BA568
:10AC00009CA50E94E7DED8012D913D914D915C916C
:10AC10000E9446DF6B017C0120E030E0A9010E9428
:10AC20004DE587FF04C0F7FAF094F7F8F0946091CF
:10AC300040117091411180914211909143110E94F5
:10AC40006BE49B01AC01A8ECB0E00E940DE30E9414
:10AC5000E7DEA70196010E94E1DE87FF39C060961A
:10AC60000CAD1DAD2EAD3FAD6097009365091093FF
:10AC70006609209367093093680922962CAD3DAD93
:10AC80004EAD5FAD229720935509309356094093FE
:10AC9000570950935809E5EBFAE184918F010F5F52
:10ACA0001F4F811103C0ECE3F3E104C00E943E4456
:10ACB000F801F3CF84918F010F5F1F4F882321F09C
:10ACC0000E943E44F801F6CF19A61AA61BA61CA6A0
:10ACD000D501C4018827B7FD83959927AA27BB27EB
:10ACE000782E57FE03C0382F3260732E8DA59EA597
:10ACF000AFA5B8A9B7FF03C0972D9460792E09A519
:10AD00001AA52BA53CA537FF03C0172D1860712E7F
:10AD100024E0629E80011124085F1D4F69A57AA579
:10AD20008BA59CA50E94E7DED8012D913D914D9108
:10AD30005C910E9446DF6B017C0120E030E0A901BC
:10AD40000E944DE587FF04C0C701B601905802C0BC
:10AD5000C701B60120E030E040E05FE30E9427E356
:10AD60000E9470E46AAB7BAB8CAB9DAB88E50BA11A
:10AD70001CA1809FF001819FF00D1124EC5BFE4E21
:10AD8000108276AAB501A401B7FE07C04427552753
:10AD9000BA01481959096A097B0988E50BA11CA168
:10ADA000809FF001819FF00D1124EC5BFE4E458BDE
:10ADB000568B678B708F2C962CAE3DAE4EAE5FAE31
:10ADC0002C9757FE0DC088279927DC01821993091B
:10ADD000A409B5092C968CAF9DAFAEAFBFAF2C9731
:10ADE00028E50BA11CA1209FF001219FF00D11244B
:10ADF000EC5BFE4E2C968CAD9DADAEADBFAD2C97F1
:10AE0000818F928FA38FB48F0DA51EA52FA538A972
:10AE100037FF07C030952095109501951F4F2F4F94
:10AE20003F4FE8E57E2EABA1BCA17A9EF0017B9E50
:10AE3000F00D1124EC5BFE4E058F168F278F30A38B
:10AE40008AA99BA9ACA9BDA981A392A3A3A3B4A3DA
:10AE500023964FAF2397752EF62FE72F2C968CADA8
:10AE60009DADAEADBFAD2C97481759076A077B075C
:10AE700078F429969FAD299723969FAF23972A961A
:10AE80007FAC2A972B96FFAD2B972C96EFAD2C9786
:10AE900023968FAD2397972DAF2FBE2F8017910745
:10AEA000A207B30710F4D901C8010AA91BA92CA94C
:10AEB0003DA980179107A207B30710F4D901C80173
:10AEC00028E50BA11CA1209FF001219FF00D11246A
:10AED000EC5BFE4E85A396A3A7A3B0A70697A1059A
:10AEE000B10508F4ABC5DF01AE5ABF4F80912A040B
:10AEF00090912B048D939C9361A6452B462B472B59
:10AF000009F05F9888E50BA11CA1809FF001819F4B
:10AF1000F00D1124EC5BFE4E818D928DA38DB48DCE
:10AF2000892B8A2B8B2B11F08A98479888E50BA1E7
:10AF30001CA1809FF001819FF00D1124EC5BFE4E5F
:10AF4000858D968DA78DB0A1892B8A2B8B2B31F007
:10AF50008091080181708093060147982AA93BA936
:10AF60004CA95DA9232B242B252B09F470C58091B6
:10AF70001605882319F0815080931605611004C0CE
:10AF8000129880E28093160560900C0570900D0574
:10AF900000910E0510910F059301A8016DA179A9EB
:10AFA0008EA99AAD0E94E1DE87FF04C06DA279AA46
:10AFB0000EAB1AAFC501B4010E94E7DE2091241147
:10AFC0003091251140912611509127110E9446DFA2
:10AFD00026966CAF7DAF8EAF9FAF2697698B7A8B2D
:10AFE0008B8B9C8BC201B1010E94E7DE209128115E
:10AFF0003091291140912A1150912B110E9446DF66
:10B000002B013C016D8B7E8B8F8B988F6DA57EA560
:10B010008FA598A90E94E7DE20912C1130912D1167
:10B0200040912E1150912F110E9446DF4B015C017F
:10B03000698F7A8F8B8F9C8F2091301130913111D5
:10B040004091321150913311C701B6010E9446DF81
:10B050006B017C016D8F7E8F8F8F98A388E50BA18C
:10B060001CA1809FF001819FF00D1124EC5BFE4E2E
:10B07000258936894789508D2DA73EA74FA758AB04
:10B08000263031054105510508F4EAC42896AEADD5
:10B09000BFAD2897CD90DD90ED90FC9020E030E0A2
:10B0A000A901C701B6010E94E1DE8111F8C426960C
:10B0B0002CAD3DAD4EAD5FAD2697CA01B9010E94E2
:10B0C00046DF6B017C01A3019201C301B2010E9422
:10B0D00046DF9B01AC01C701B6010E9427E36B016B
:10B0E0007C01A5019401C501B4010E9446DF9B01CA
:10B0F000AC01C701B6010E9427E30E9492E528E552
:10B100000BA11CA1209FF001219FF00D1124EC5BED
:10B11000FE4E658776878787908B88E50BA11CA1FB
:10B12000809FF001819FF00D1124EC5BFE4E458461
:10B13000568467847088A301920160E070E080E823
:10B140009FE30E9403E464966CAF7DAF8EAF9FAF28
:10B1500064972DA139A94EA95AAD0E9446DF4B0133
:10B160005C018091330990913109891B8F7027967A
:10B170008FAF2797A501940160E074E284E799E41A
:10B180000E9403E40E9458E56B017C0127968FAD75
:10B1900027978250863008F491C4A5019401C30119
:10B1A000B2010E9446DF9B01AC010E9446DF689617
:10B1B0006CAF7DAF8EAF9FAF689788E5ABA1BCA1A8
:10B1C0008A9F80018B9F100D11240C5B1E4E689688
:10B1D0002CAD3DAD4EAD5FAD6897D80111962D9366
:10B1E0003D934D935C93149795962D913D914D9180
:10B1F0005C9198972EAB3FAB48AF59AFCA01B901EC
:10B200000E94E5DE6AAF7BAF8CAF9DAF9B01AC01C6
:10B21000C501B4010E9446DF0E94EDE30E9470E484
:10B22000A8966CAF7DAF8EAF9FAFA897F801EE5B8D
:10B23000FF4F60837183828393838E010F5E1F4F64
:10B240002A961FAF0EAF2A970051110924961FAFFF
:10B250000EAF249704EF14E0AC961FAF0EAFAC977F
:10B260008E010F5D1F4F1AA309A324960EAD1FADCB
:10B270002497AA961FAF0EAFAA97312C212C10E865
:10B280001DA30FE309AB2A96AEADBFAD2A972D9152
:10B290003D914D915D912A96BFAFAEAF2A97C50102
:10B2A000B4010E9446DF6B017C01AA96EEADFFADB2
:10B2B000AA976193719381939193AA96FFAFEEAF92
:10B2C000AA9720E030E0A9010E944DE587FF04C065
:10B2D000F7FAF094F7F8F094AC96AEADBFADAC973A
:10B2E0004D905D906D907D90AC96BFAFAEAFAC973A
:10B2F000A7019601C301B2010E94E1DE87FD18C4D7
:10B3000009A11AA12A962EAD3FAD2A97021713075D
:10B3100009F0B9CF20E030E040E85FE3632D722D03
:10B320008DA199A90E94E1DE87FF58C07E0131E11D
:10B33000E30EF11C24960EAD1FAD2497232D322D64
:10B340004DA159A9D8016D917D918D919C910E943B
:10B3500046DFF80161937193819391938F01EE160B
:10B36000FF0661F728E50BA11CA1209FC001219FCA
:10B37000900D11249C012C5B3E4E790189010E5BDE
:10B380001F4FA8966CAD7DAD8EAD9FADA8970E9466
:10B39000E5DE232D322D4DA159A90E9446DF0E94E2
:10B3A00070E4D8016D937D938D939C931397232D17
:10B3B000322D4DA159A9632D722D8DA199A90E94FD
:10B3C00046DF68962CAD3DAD4EAD5FAD68970E94EF
:10B3D00046DFF70161837283838394832AAD3BAD9B
:10B3E0004CAD5DAD64966CAD7DAD8EAD9FAD64979B
:10B3F0000E9446DF6DA37EA38FA398A70DA51EA56F
:10B400002FA538A9012B022B032B09F0A9C388E52E
:10B410002BA13CA1829F8001839F100D11240C5B06
:10B420001E4EF801818D928DA38DB48D892B8A2BB0
:10B430008B2B09F095C3858D968DA78DB0A1892B97
:10B440008A2B8B2B09F08CC32091F0043091F104EE
:10B450004091F2045091F3046DA17EA18FA198A5B3
:10B460000E9446DF0E94EDE30E9470E42B013C0144
:10B47000D801D7961C9288E52BA13CA1829F800120
:10B48000839F100D11240C5B1E4EF801E25BFF4FF1
:10B490004082518262827382C301B2010E94E5DE62
:10B4A0006B017C012DA13EA14FA158A50E9403E490
:10B4B0006AAF7BAF8CAF9DAFD80151966D937D93F2
:10B4C0008D939C9354972DEB37E346E051E4C701ED
:10B4D000B6010E9446DF0E9470E4F80162AB73ABD4
:10B4E00084AB95AB87A9882371F1FE962091E40483
:10B4F0003091E5044091E6045091E7046081718148
:10B50000828193810E9446DF2AAD3BAD4CAD5DAD9B
:10B510000E9446DF2091401130914111409142112B
:10B52000509143110E9446DF9B01AC0160E074E240
:10B5300084EF99E40E9403E40E9470E4D801D99654
:10B540007C936E93D89788E50BA11CA1809FF00196
:10B55000819FF00D1124EC5BFE4E218132814381ED
:10B5600054812C962CAF3DAF4EAF5FAF2C97CA01E4
:10B57000B9010E9492E5362E272E8C0144ED54E04D
:10B5800062965FAF4EAF62973E0151E1650E711C4E
:10B5900084ED94E09FAB8EAB24964EAC5FAC2497C9
:10B5A00039A62DA60DA319AB1AAAD201CD90DD9014
:10B5B000ED90FD902D0120E030E0A901C701B6011A
:10B5C0000E944DE587FF04C0F7FAF094F7F8F09475
:10B5D000EEA9FFA981909190A190B190FFABEEAB45
:10B5E000A7019601C501B4010E94E1DE87FDD4C523
:10B5F00064147504D1F627965FAD2797552309F497
:10B6000044C6C0903509D0903609E0903709F090D3
:10B6100038092DEB37E346E855E3C701B6010E9430
:10B62000E1DE87FD32C6C701B6010E9492E56B01DB
:10B630007C019B01AC01632D722DC8010E94E1DEEB
:10B6400087FD03C03C2C2D2C87019601A701632D9B
:10B65000722DC8010E9403E468966CAF7DAF8EAF77
:10B660009FAF689789E399E028969FAF8EAF2897A0
:10B6700020E030E040E85FE32AAB3BAB4CAB5DAB96
:10B680001EAA2896AEADBFAD28972D913D914D9144
:10B690005D912896BFAFAEAF289768966CAD7DAD33
:10B6A0008EAD9FAD68970E9446DF4B015C012496EA
:10B6B000EEADFFAD2497C190D190E190F19024962A
:10B6C000FFAFEEAF2497FEA9FF2391F02AA93BA973
:10B6D0004CA95DA90E9446DF4B015C012AA93BA948
:10B6E0004CA95DA9C701B6010E9446DF6B017C0130
:10B6F000A7019601C501B4010E944DE520E030E0AC
:10B70000A90118160CF08EC5C701B6010E944DE5BF
:10B7100018160CF482C520E030E0A901C501B4017F
:10B720000E94E1DE87FD79C52601370177FA709422
:10B7300077F87094A3019201C501B4010E944DE510
:10B74000181614F4240135016296AEADBFAD6297B0
:10B75000CD90DD90ED90FD906296BFAFAEAF629759
:10B76000A3019201C701B6010E94E1DE87FF15C067
:10B77000A3019201C701B6010E9403E49B01AC0141
:10B780006AA97BA98CA99DA90E9446DF6AAB7BAB05
:10B790008CAB9DABBEA9BF5FBEABE9E4F9E02896D8
:10B7A0002EAD3FAD2897E217F30709F06ACF3EA907
:10B7B000332361F02AA93BA94CA95DA9632D722D01
:10B7C000C8010E9446DF362E272E8C0124EA30E77E
:10B7D0004DE75FE3632D722DC8010E9446DF6B01C8
:10B7E0007C01209112053091130540911405509170
:10B7F00015050E94E1DE87FD3EC589A59DA5ADA189
:10B80000B9A98093120590931305A0931405B093E2
:10B81000150528E54BA15CA1249FC001259F900D33
:10B820001124DC01AC5BBE4E7D01232D322DA8011D
:10B83000632D722DC8010E9446DFF7016187728770
:10B84000838794876AAD7BAD8CAD9DAD90589B018D
:10B85000AC010E9427E3D7011D962D913D914D919A
:10B860005C9150970E9446DF9B01AC016BE077ED45
:10B8700083E29BE30E9426E39B01AC018BE097ED02
:10B88000A3E2BBE3F70185839683A783B08710818A
:10B890002C966CAD7DAD8EAD9FAD2C970E94E1DEF8
:10B8A00018160CF4F7C483E0182B88E52BA13CA1F3
:10B8B000829FF001839FF00D1124EC5BFE4E1083FC
:10B8C00080E1FE013196A9E3B9E001900D928A95DD
:10B8D000E1F72C968CAD9DADAEADBFAD2C978093AE
:10B8E000350990933609A0933709B0933809E0964B
:10B8F0000CAD1DAD2EAD3FADE097009359091093EF
:10B900005A0920935B0930935C09E4962CAD3DAD58
:10B910004EAD5FADE49720935D0930935E0940938F
:10B920005F0950936009E8968CAD9DADAEADBFAD9B
:10B93000E8978093610990936209A0936309B0939B
:10B94000640960960CAD1DAD2EAD3FAD60970093C0
:10B9500065091093660920936709309368096C960E
:10B960002CAD3DAD4EAD5FAD6C9720934909309342
:10B970004A0940934B0950934C09A0968CAD9DAD5C
:10B98000AEADBFADA09780934D0990934E09A093A3
:10B990004F09B0935009A4960CAD1DAD2EAD3FAD2F
:10B9A000A49700935109109352092093530930939F
:10B9B000540922962CAD3DAD4EAD5FAD229720933C
:10B9C000550930935609409357095093580990915F
:10B9D000330980913409981303C084E680933009B9
:10B9E000E9968FADE9978F5F8F70809333098091CF
:10B9F00033099091320981508F7089134DC4109191
:10BA000034091BA30091330909A728E51BA109A547
:10BA10001013CDC4812C912CA12CB12C1DA61DA2DC
:10BA200019AA1EAE212C312C00E010E029A53BA163
:10BA30002313CAC42114310409F079C580916F0021
:10BA4000826080936F0081E0E2C680E0E0C6609093
:10BA500008057090090500910A0510910B059CCA14
:10BA6000818D928DA38DB48D0697A105B10508F047
:10BA70000DCB858D968DA78DB0A10697A105B1053B
:10BA800008F004CB20E030E0A901C701B6010E9414
:10BA90004DE587FF04C0F7FAF094F7F8F09488E5D5
:10BAA0000BA11CA1809FF001819FF00D1124EC5B84
:10BAB000FE4EC586D686E786F08A2FCB8091040598
:10BAC00090910505A0910605B0910705C816D90605
:10BAD000EA06FB0608F061CB8C199D09AE09BF0987
:10BAE000BC01CD01660F771F881F991F27964FADA8
:10BAF0002797042F10E020E030E0A90198010E9470
:10BB0000CFE2CA01B9010E94E5DE0E9458E56C0D42
:10BB10007D1D8E1D9F1D0E94E5DE9B01AC0160E036
:10BB200074E284E799E40E9403E44B015C0135CBA5
:10BB3000A7019601C301B2010E9403E47B018C01BD
:10BB40009B01AC01632D722D8DA199A90E944DE539
:10BB500018160CF0D5CB3E2C2F2C0DA319ABD0CB47
:10BB60000AA91BA92CA93DA9012B022B032B49F0E3
:10BB70002091EC043091ED044091EE045091EF04DB
:10BB800008C02091E8043091E9044091EA04509102
:10BB9000EB046DA17EA18FA198A50E9446DF0E94B3
:10BBA000EDE30E9470E42B013C012AA93BA94CA9BA
:10BBB0005DA9232B242B252BC9F020E030E0A9011F
:10BBC0006091E4047091E5048091E6049091E704AB
:10BBD0000E94E1DE882351F081E009A51AA52BA57A
:10BBE0003CA510161106120613060CF080E098E52D
:10BBF0002BA13CA1929F8001939F100D11240C5BFF
:10BC00001E4ED801D7968C93882309F4B2C0209198
:10BC1000490930914A0940914B0950914C096C9661
:10BC20006CAD7DAD8EAD9FAD6C970E9426E369A78C
:10BC30007AA78BA79CA720914D0930914E0940917E
:10BC40004F0950915009A0966CAD7DAD8EAD9FAD62
:10BC5000A0970E9426E34B015C012091510930918D
:10BC600052094091530950915409A4966CAD7DAD91
:10BC70008EAD9FADA4970E9426E36B017C0129A5A0
:10BC80003AA54BA55CA5CA01B9010E9446DF69A788
:10BC90007AA78BA79CA7A5019401C501B4010E94B6
:10BCA00046DF9B01AC0169A57AA58BA59CA50E94E6
:10BCB00027E34B015C01A7019601C701B6010E9471
:10BCC00046DF9B01AC01C501B4010E9427E30E943D
:10BCD00092E56B017C012091550930915609409104
:10BCE00057095091580922966CAD7DAD8EAD9FAD30
:10BCF00022970E9426E3A70196010E9403E46B01AC
:10BD00007C01F801FE96608371838283938320E037
:10BD100030E040E450E40E944DE518161CF4F801B0
:10BD200017AA27C02091E4043091E5044091E6046D
:10BD30005091E704C701B6010E9446DF9B01AC01A8
:10BD40006091E0047091E1048091E2049091E30439
:10BD50000E9403E42DA13EA14FA158A50E9446DFF9
:10BD60000E9470E4641575058605970510F42B0193
:10BD70003C018091001190910111A0910211B091AC
:10BD800003110EA91FA928AD39AD80179107A2078D
:10BD9000B30708F4DFC02DA53EA54FA558A9232B56
:10BDA000242B252B41F16091041170910511809194
:10BDB0000611909107116415750586059705D8F44D
:10BDC0002EA93FA948AD59AD0E94C0E26B017C018C
:10BDD0002DA53EA54FA558A9C301B2010E94C0E2FE
:10BDE000C616D706E806F90630F4C701B6010E9468
:10BDF000CFE229013A0188E50BA11CA1809FF00147
:10BE0000819FF00D1124EC5BFE4EC18CD28CE38C33
:10BE1000F48CC114D104E104F10431F160910811F2
:10BE20007091091180910A1190910B11641575059B
:10BE300086059705C8F42EA93FA948AD59AD0E94C3
:10BE4000C0E24B015C01A7019601C301B2010E944F
:10BE5000C0E286169706A806B90630F4C501B401FB
:10BE60000E94CFE229013A0188E50BA11CA1809F25
:10BE7000F001819FF00D1124EC5BFE4EC58CD68C39
:10BE8000E78CF0A0C114D104E104F10431F1609118
:10BE90000C1170910D1180910E1190910F1164157C
:10BEA000750586059705C8F42EA93FA948AD59AD7B
:10BEB0000E94C0E24B015C01A7019601C301B201DF
:10BEC0000E94C0E286169706A806B90630F4C5019E
:10BED000B4010E94CFE229013A0188E50BA11CA11F
:10BEE000809FF001819FF00D1124EC5BFE4EC1A0FC
:10BEF000D2A0E3A0F4A0C114D104E104F10409F438
:10BF0000BACA609110117091111180911211909123
:10BF10001311641575058605970508F0ACCA2EA99E
:10BF20003FA948AD59AD0E94C0E24B015C01A70199
:10BF30009601C301B2010E94C0E286169706A806C8
:10BF4000B90608F098CAC501B4010E94CFE22901E0
:10BF50003A0191CA2DA53EA54FA558A9232B242B04
:10BF6000252BC9F160910411709105118091061182
:10BF700090910711641575058605970560F50E9477
:10BF8000E5DE2AAD3BAD4CAD5DAD0E9446DF6B01F9
:10BF90007C016DA57EA58FA598A90E94E5DE4B01C9
:10BFA0005C01C301B2010E94E5DEA50194010E947B
:10BFB00046DF9B01AC01C701B6010E94E1DE87FFAD
:10BFC0000AC0A5019401C701B6010E9403E40E94C2
:10BFD00070E42B013C0188E50BA11CA1809FF001BE
:10BFE000819FF00D1124EC5BFE4E818C928CA38C12
:10BFF000B48C81149104A104B104B9F160910811C9
:10C000007091091180910A1190910B1164157505B9
:10C010008605970550F50E94E5DE2AAD3BAD4CAD97
:10C020005DAD0E9446DF6B017C01C501B4010E9439
:10C03000E5DE4B015C01C301B2010E94E5DEA50112
:10C0400094010E9446DF9B01AC01C701B6010E942A
:10C05000E1DE87FF0AC0A5019401C701B6010E9475
:10C0600003E40E9470E42B013C0188E50BA11CA1B4
:10C07000809FF001819FF00D1124EC5BFE4E858CBA
:10C08000968CA78CB0A081149104A104B104B9F1DD
:10C0900060910C1170910D1180910E1190910F1102
:10C0A000641575058605970550F50E94E5DE2AADF5
:10C0B0003BAD4CAD5DAD0E9446DF6B017C01C5011F
:10C0C000B4010E94E5DE4B015C01C301B2010E9494
:10C0D000E5DEA50194010E9446DF9B01AC01C7018A
:10C0E000B6010E94E1DE87FF0AC0A5019401C701E5
:10C0F000B6010E9403E40E9470E42B013C0188E534
:10C100000BA11CA1809FF001819FF00D1124EC5B1D
:10C11000FE4EC1A0D2A0E3A0F4A0C114D104E1045A
:10C12000F10409F4A8C96091101170911111809166
:10C13000121190911311641575058605970508F085
:10C140009AC90E94E5DE2AAD3BAD4CAD5DAD0E94C3
:10C1500046DF4B015C01C701B6010E94E5DE6B01C1
:10C160007C01C301B2010E94E5DEA70196010E9495
:10C1700046DF9B01AC01C501B4010E94E1DE87FFEF
:10C180007AC9A7019601C501B4010E9403E40E9487
:10C1900070E42B013C016FC9FAA9FF2331F1A5011D
:10C1A0009401632D722DC8010E9446DF4B015C0192
:10C1B00029A53DA54DA159A9C701B6010E9446DF99
:10C1C0009B01AC01C501B4010E94E1DE87FF22C0E2
:10C1D000A7019601C501B4010E9403E469A77DA7E8
:10C1E0008DA399AB21E02AAB03CAA7019601C50133
:10C1F000B4010E9403E49B01AC0169A57DA58DA15A
:10C2000099A90E9446DF69A77DA78DA399AB31E06C
:10C210003AABEEC941E04AABEBC9A7019601C501B3
:10C22000B40113C0C701B6010E94E1DE87FD09C059
:10C2300020E030E0A901C501B4010E944DE51816C7
:10C240004CF4A5019401C701B6010E9426E32B011D
:10C250003C017ACA2401350177FA709477F870941A
:10C26000A3019201C701B6010E94E1DE87FD6CCAFD
:10C270002601370169CA29A53DA54DA159A9C701C4
:10C28000B6010E94E1DE87FFB8CA39A42DA40DA132
:10C2900019A9B3CA81E008CBF09033098FEF8F0D55
:10C2A0008F708BA3B090320980913309B81609F4CE
:10C2B00054C0C12CD12C0BA10B1509F44EC0602E1B
:10C2C000712C28E5269D8001279D100D11240C5B03
:10C2D0001E4ED8018C9183FD2BC00EAF1AAB0115F9
:10C2E000110541F11996BC91B9A7F801F285FDA796
:10C2F000D8011B96BC91BDA3F801F485F9ABD80118
:10C3000015962D903D904D905C901897A20191014B
:10C3100069A57DA58DA19F2F0E94E1DE811180C1BD
:10C32000C114D10439F0F601808180FD79C102C0C9
:10C33000CEAEDAAA8BA181508F708BA38091320987
:10C340008B1103C0CEACDAA8B6CF0BA10B1529F028
:10C3500081E08B0D8F70B82EF1CF109132091BA3A5
:10C36000C12CD12C809133090BA1801709F447CB44
:10C37000802E912C28E5289D8001299D100D1124E7
:10C380000C5B1E4ED8018C9183FD0AC05801C1146C
:10C39000D10439F0C6010E947C94811102C0BFC152
:10C3A00056018BA18F5F8F708BA36501DBCF802F30
:10C3B00081508F70289FF0011124EC5BFE4E90811C
:10C3C00093FF28CB89A722CB48E5439FC0011124C6
:10C3D000DC01AC5BBE4E1D018C9183FD19C015962E
:10C3E0006D917D918D919C9118970E9492E5F62E0A
:10C3F000E72ED82EC92E0115110509F48AC0F801BF
:10C40000808180FD0AC0D1018C9180FD06C081C071
:10C41000FDA4EDA0D9A8CEAC81C0F80180818160D7
:10C420008083C8010E947C9481116FC0F8016181F2
:10C430007281838194810E9492E52B013C019B01D2
:10C44000AC0160E070E080E89FE30E9403E44B01F0
:10C450005C019B01AC016F2D7E2D8D2D9C2D0E94CA
:10C4600046DF69837A838B839C832DA53DA149A9EF
:10C470005EADC501B4010E9446DF698B7A8B8B8B60
:10C480009C8BAE014F5F5F4FBE016F5E7F4FC80157
:10C490000E9418C3D801D7968C918823B1F12091BE
:10C4A000E4043091E5044091E6045091E704F8017A
:10C4B000FE9660817181828193810E9446DF209186
:10C4C00040113091411140914211509143110E940D
:10C4D00046DF4B015C019B01AC01C301B2010E942C
:10C4E00046DF0E9470E4F80173AF62AFA5019401CA
:10C4F0006F2D7E2D8D2D9C2D0E9446DF0E9470E4B5
:10C50000D801DD967C936E93DC97F80180818E7F55
:10C5100080838F2C9E2CAD2CBC2C81018BA18F5F36
:10C520008F708BA3FDA6EDA2D9AACEAE7FCAD10192
:10C530008C9181608C93C8010E947C9481116BC0A6
:10C54000F10161817281838194810E9492E56B0186
:10C550007C019B01AC0160E070E080E89FE30E94F9
:10C5600003E42B013C012DEC3CEC4CE45DE30E9428
:10C5700046DF69837A838B839C839401A501C30181
:10C58000B2010E9446DF698B7A8B8B8B9C8BAE014C
:10C590004F5F5F4FBE016F5E7F4FC1010E9418C3A6
:10C5A000D101D7968C918823B1F12091E404309188
:10C5B000E5044091E6045091E704F101FE966081A4
:10C5C0007181828193810E9446DF209140113091D8
:10C5D000411140914211509143110E9446DF4B019D
:10C5E0005C019B01AC01C701B6010E9446DF0E94BD
:10C5F00070E4F10173AF62AF2DEC3CEC4CE45DE311
:10C60000C501B4010E9446DF0E9470E4D101DD96AD
:10C610007C936E93DC97F10180818E7F80830ECABC
:10C6200028E5269DF001279DF00D1124EC5BFE4EC0
:10C63000808181FD43C0C114D10441F0D60115961B
:10C64000CD90DD90ED90FC90189708C08BE0C82E3F
:10C6500087EDD82E83E2E82E8BE3F82EB8E5B69D61
:10C66000F001B79DF00D1124EC5BFE4E818992899B
:10C67000A389B489BC01CD0190589B01AC010E94F3
:10C6800027E3F80125853685478550890E9446DFD6
:10C690009B01AC01C701B6010E9426E3E62E872E5E
:10C6A000982EA92E262F372F482F592F69A57DA503
:10C6B0008DA199A90E94E1DE87FF04C0E9A48DA4A1
:10C6C0009DA0A9A82E2D382D492D5A2DC201B101AA
:10C6D0000E94E1DE882309F42DCEF8E5F69DC00125
:10C6E000F79D900D11249C012C5B3E4E6901D901F0
:10C6F0008C9181608C93C8010E947C94882329F0DE
:10C70000F60180818E7F808315CE8E2D982DA92DE8
:10C71000BA2DF60185839683A783B0870BCED60109
:10C720008C9181FD52C0D60115962D913D914D9170
:10C730005C91189729A73AA74BA75CA71501B5E00C
:10C740002B0E311CF8014580568067807084A30150
:10C75000920169A57AA58BA59CA50E94E1DE87FFC1
:10C7600034C0F60181899289A389B489BC01CD01C5
:10C7700090589B01AC010E9427E3D6011D962D9194
:10C780003D914D915C9150970E9446DF9B01AC0119
:10C7900069A57AA58BA59CA50E9426E36B017C0167
:10C7A0009B01AC01C301B2010E944DE518166CF467
:10C7B000D8018C9181608C93C5010E947C94882360
:10C7C000E1F0F80180818E7F808318E5189DF001EB
:10C7D000199DF00D1124EC5BFE4E218532854385B9
:10C7E000548565817681878190850E94E1DE811183
:10C7F000D8CD0BA100933209D4CDD101CD92DD92D9
:10C80000ED92FC9213970BA100933209DECFC8582A
:10C81000DF4F0FB6F894DEBF0FBECDBFDF91CF91D3
:10C820001F910F91FF90EF90DF90CF90BF90AF904E
:10C830009F908F907F906F905F904F903F902F9040
:10C8400008958091330990913409891B8F708F303E
:10C8500011F42BD3F6CF809133098F5F8F70E09165
:10C86000330998E59E9FF0011124EC5BFE4EDF0139
:10C870001D929A95E9F798E090834091590950915B
:10C880005A0960915B0970915C09458B568B678BE7
:10C89000708F40915D0950915E0960915F097091C0
:10C8A0006009418F528F638F748F4091610950915D
:10C8B00062096091630970916409458F568F678F93
:10C8C00070A3409165095091660960916709709164
:10C8D000680941A352A363A374A3209133099091E3
:10C8E0003409291303C094E69093300980933309E7
:10C8F00080916F00826080936F000895909133095A
:10C9000080913409981306C080917C0490917D0435
:10C91000892B11F0CAD2F2CF08958FEF8EBD0DB4DE
:10C9200007FEFDCF8EB50895CF92DF92EF92FF9272
:10C93000CF93DF93EC01C0904E05D0904F05E0906F
:10C940005005F0905105A7019601688179818A818F
:10C950009B810E94E1DE87FF04C0C882D982EA82FF
:10C96000FB82C0905205D0905305E0905405F090A2
:10C970005505A70196016C817D818E819F810E9462
:10C98000E1DE87FF04C0CC82DD82EE82FF82C090B0
:10C990001402D0901502E0901602F0901702A70141
:10C9A0009601688179818A819B810E944DE51816E4
:10C9B00024F4C882D982EA82FB82C0901802D09007
:10C9C0001902E0901A02F0901B02A70196016C81F7
:10C9D0007D818E819F810E944DE5181624F4CC82C2
:10C9E000DD82EE82FF82C0905605D0905705E09020
:10C9F0005805F0905905A7019601688579858A85C3
:10CA00009B850E94E1DE87FF04C0C886D986EA863E
:10CA1000FB86C0901C02D0901D02E0901E02F09098
:10CA20001F02A7019601688579858A859B850E94EA
:10CA30004DE5181624F4C886D986EA86FB86DF9170
:10CA4000CF91FF90EF90DF90CF9008954F925F923B
:10CA50006F927F928F929F92AF92BF92CF92DF920E
:10CA6000EF92FF920F931F93CF93DF93D82EC82F8F
:10CA7000D0E0FE01E45AFA4EC49082E0D81203C01E
:10CA800081E08093F70F7E01EE0CFF1CEE0CFF1C83
:10CA9000F701E05BFA4E45905590659074906C2DCF
:10CAA0000C2C000C770B880B990B0E94E7DE4B01D6
:10CAB0005C0120E030E040EC5FE3C301B2010E9482
:10CAC00046DFA50194010E9446DFAB01BC0100E0F6
:10CAD00010E098018D2D0E94107DF701EC5BFA4E5D
:10CAE0002591359145915491C501B4010E9446DFCD
:10CAF0004B015C0120E030E0A9010E94E1DE8823C7
:10CB000009F448C000E010E09801B501A401705894
:10CB10008D2D0E94107DFE01EF5BFA4EC491C11174
:10CB200017C0E5EBFAE18491EF012196882321F00B
:10CB30000E943E44FE01F7CFEFE1F5E18491EF0161
:10CB40002196882321F00E943E44FE01F7CFCAE0DF
:10CB5000F701E15FFA4E45905590659074906C2F07
:10CB600070E080E090E00E94E7DE9B01AC01C30131
:10CB7000B2010E9403E42B013C01A5019401C5010F
:10CB8000B4010E9427E3AB01BC01930182018D2D0A
:10CB90000E94107D82E0D81249C040906F105090E2
:10CBA0007010609071107090721020E030E0A90158
:10CBB000C301B2010E944DE55301420187FF04C049
:10CBC000B7FAB094B7F8B09420E030E0A901C501FD
:10CBD000B4010E94E1DE882349F120E030E0A901A0
:10CBE000C301B2011C142CF40E944DE518162CF060
:10CBF00008C00E94E1DE87FF04C081E08093F40F4B
:10CC000003C081E08093F30F1C1424F4B7FAB094AE
:10CC1000B7F8B09400E010E09801B501A40182E0FB
:10CC20000E94107D1092F40F1092F30F1092F70FE4
:10CC300081E090E00D2C01C0880F0A94EAF79091F2
:10CC40001904982B909319049091F310892B8093D9
:10CC5000F310F701EE5CFA4F1082118212821382F8
:10CC60008D2D0E94608FF701ED5FFA4E85919591B1
:10CC7000A591B491E701C65EDB4F88839983AA83AF
:10CC8000BB830E94FE92F701E25CFA4F8881998192
:10CC9000AA81BB8180839183A283B383DF91CF91EB
:10CCA0001F910F91FF90EF90DF90CF90BF90AF90CA
:10CCB0009F908F907F906F905F904F9008954F92CC
:10CCC0005F926F927F928F929F92AF92BF92CF921C
:10CCD000DF92EF92FF92CF936B017C0149015A01E1
:10CCE00020E030E044E052E40E9426E32B013C01C6
:10CCF00021E338E040EA50EC0E944DE587FD50C04A
:10CD000022E430E042E553E4C301B2010E94E1DED7
:10CD100018160CF445C020E030E040EA50E4C501AC
:10CD2000B4010E9426E32B013C012FE632E143E8E7
:10CD30005AEB0E944DE587FD33C022E430E042E526
:10CD400053E4C301B2010E94E1DE18164CF124EF56
:10CD50003DEF4FED51E4C701B6010E944DE587FD5F
:10CD60001FC022E430E048E453E4C701B6010E944A
:10CD7000E1DE1816ACF027EE3BEF4FE151E4C501C0
:10CD8000B4010E944DE587FD0BC0C1E022E430E014
:10CD900048E453E4C501B4010E94E1DE18160CF426
:10CDA000C0E08C2FCF91FF90EF90DF90CF90BF909D
:10CDB000AF909F908F907F906F905F904F9008956D
:10CDC00029EF32E0FC013183208304960C942E4439
:10CDD0005F9A809119048E7F809319048A9A479AEA
:10CDE000809119048D7F80931904809108018095AA
:10CDF000817080930601479A809119048B7F8093FC
:10CE00001904129A0895E0EAFAE18491EF0121965B
:10CE1000882321F00E943E44FE01F7CFE3EEF4E1C7
:10CE20008491EF012196882321F00E943E44FE0167
:10CE3000F7CF0E94B94CCCDFEFEDF4E18491EF0124
:10CE4000882349F0082E000C990B0E94E286219657
:10CE5000FE018491F5CF8DE090E00E94E2868AE0A9
:10CE600090E00E94E286E8EBF4E18491EF012196E4
:10CE7000882321F00E943E44FE01F7CFFFEF2BE410
:10CE80008DE1F15020408040E1F700C00000F894AF
:10CE90009FEFE4E3FCE09150E040F040E1F700C098
:10CEA00000000E94B94CA895FECF2F923F924F925E
:10CEB0005F926F927F928F929F92AF92BF92CF922A
:10CEC000DF92EF92FF920F931F93CF93DF9300D0E7
:10CED0001F92CDB7DEB70E947B2F0E94407A6B0174
:10CEE0007C0110910F02112309F47BC0809124056D
:10CEF000882309F476C040916605509167056091DA
:10CF000068057091690546015701841A950AA60AB9
:10CF1000B70AB7FC78C0833051F134F481300CF497
:10CF200060C0E5EBFAE106C0843009F05AC0E5EBD9
:10CF3000FAE13BC084919F012F5F3F4F3B832A83DF
:10CF4000882329F00E943E44EA81FB81F3CFEFED74
:10CF5000F3E184919F012F5F3F4F3B832A83882316
:10CF600009F43FC00E943E44EA81FB81F2CFE5EB29
:10CF7000FAE184919F012F5F3F4F3B832A838823EF
:10CF800029F00E943E44EA81FB81F3CFE8ECF3E113
:10CF900084919F012F5F3F4F3B832A83882309F1B0
:10CFA0000E943E44EA81FB81F3CF84919F012F5F71
:10CFB0003F4F3B832A83882329F00E943E44EA8125
:10CFC000FB81F3CFE0EBF3E184919F012F5F3F4FB3
:10CFD0003B832A83882329F00E943E44EA81FB8117
:10CFE000F3CF212F30E0A8EEB3E00E9417E3C60E86
:10CFF000D71EE81EF91EC0926605D0926705E09222
:10D000006805F092690589B182FB882780F98093D1
:10D01000540E9091550E98170CF052C08091560EF8
:10D020009091570EA091580EB091590E0196A11DE6
:10D03000B11D883B3DE39307A105B1050CF45BC02E
:10D040001092560E1092570E1092580E1092590EC2
:10D050008091F909882319F00E9449882CC0EBE1DE
:10D06000F4E18491FB83EA83882371F0082E000C9D
:10D07000990B0E94E2862A813B812F5F3F4F3B83C1
:10D080002A83F9018491F0CF8DE090E00E94E2863E
:10D090008AE090E00E94E286E1EFF3E184919F0153
:10D0A0002F5F3F4F3B832A83882329F00E943E4411
:10D0B000EA81FB81F3CF8091540E8093550E23C0FB
:10D0C000891709F11092560E1092570E1092580EB1
:10D0D0001092590E8093550EEFE1F4E184919F0177
:10D0E0002F5F3F4F3B832A83882369F00E943E4491
:10D0F000EA81FB81F3CF8093560E9093570EA09355
:10D10000580EB093590E8091F610843010F40E949E
:10D1100062900E94407AC0902905D0902A05E09044
:10D120002B05F0902C05C114D104E104F10489F120
:10D13000009125051091260520912705309128059D
:10D140000C0D1D1D2E1D3F1D4B015C01801A910A07
:10D15000A20AB30AB7FC1DC0E0EAFAE184919F017C
:10D160002F5F3F4F3B832A83882329F00E943E4450
:10D17000EA81FB81F3CF6091D8107091D9108EE7CE
:10D1800094E10E94A8C88AE00E943E4485E794E1A9
:10D1900081C0C0901002D0901102E0901202F09075
:10D1A0001302C114D104E104F104E9F1309133090F
:10D1B00020913409321749F06093250570932605B4
:10D1C00080932705909328052EC000912505109186
:10D1D000260520912705309128050C0D1D1D2E1DBB
:10D1E0003F1DDC01CB01801B910BA20BB30BB7FDE4
:10D1F0001AC05F9A809119048E7F809319048A9ACD
:10D20000479A809119048D7F8093190480910801B9
:10D210008095817080930601479A809119048B7FD5
:10D2200080931904129A80917605909177059099D0
:10D2300002C0019604C0181619062CF401979093A9
:10D2400077058093760580917605909177058E3EDF
:10D2500092400CF1E0EAFAE184919F012F5F3F4F89
:10D260003B832A83882329F00E943E44EA81FB8184
:10D27000F3CFE5E5F4E184919F012F5F3F4F3B83BE
:10D280002A83882329F00E943E44EA81FB81F3CF60
:10D290008CE494E1B8DD0E94407A0091720510910F
:10D2A000730520917405309175054B015C01801A5E
:10D2B000910AA20AB30AB7FC4EC08B019C010C5321
:10D2C000164F2F4F3F4F0093720510937305209315
:10D2D0007405309375054F9BA9C17A9BA7C1209116
:10D2E000060120FFA3C120917F0421119FC1379B1C
:10D2F0009DC1379B9BC1029B99C100916E05109106
:10D300006F052091700530917105011511052105FA
:10D31000310599F0DC01CB01801B910BA20BB30B03
:10D3200080569A4EA109B1098827B7FD83959927A0
:10D33000AA27BB27682F619501C060E0262F30E047
:10D340008091020161118095807180930001B90183
:10D3500087E00E946FBA9091330980913409981741
:10D3600091F0E091340928E5E29FF0011124EA569A
:10D37000FE4E60818091340990913309981729F00D
:10D380008F5F8F70F9CF60912A0470E089E00E946E
:10D390006FBA80917A04882309F4F8C00091510291
:10D3A00010915202809053028C82909054029A8283
:10D3B00060913204709133046E5F7F4F072E000C32
:10D3C000880B990B0E94E7DE9801A4010E94E1DE20
:10D3D00087FDDCC0F0903409212C312CE12C19821E
:10D3E000809133098F1509F462C08F2D90E038E5E4
:10D3F000A32EA89EF001A99EF00D1124EC5BFE4E19
:10D40000458956896789708D452B462B472B81F4BA
:10D41000418D528D638D748D452B462B472B41F4E6
:10D42000458D568D678D70A1452B462B472BD1F12D
:10D4300028E5B22EB89E9001B99E300D1124C90185
:10D440008C5B9E4E6C01FC016181728183819481B1
:10D450000E9492E54B015C01F60161A172A183A1DA
:10D4600094A10E94E5DE2B013C01F60165A176A1A5
:10D4700087A190A50E94E5DE9B01AC01C301B2012A
:10D480000E9403E4A50194010E9446DF5B016C0148
:10D4900091014E2D59810E944DE518161CF415017D
:10D4A000EC2CD98281E08F0D8F70F82E99CF2091CE
:10D4B0005502309156024091570250915802B101E5
:10D4C0008E2D99810E9446DF98014C815A810E94DD
:10D4D00027E36B017C019B01AC01B8018C819A812F
:10D4E0000E944DE51816ACF000914D0210914E02CD
:10D4F00080904F028C82909050029A829801A401F1
:10D50000B601C7010E944DE518161CF08601EC8299
:10D51000FA82C0906A05D0906B05E0906C05F0909F
:10D520006D0598014C815A81C701B6010E944DE5F5
:10D530001816D4F420E037ED43EA5CE3B8018C819F
:10D540009A810E9446DF4B015C0128E431EE4AE7F4
:10D550005FE3C701B6010E9446DFA50194010E9466
:10D5600027E38B018C839A83C801AC81BA818093B5
:10D570006A0590936B05A0936C05B0936D05B80197
:10D58000CD010E946BE4CB010E94F94A0E949B509E
:10D5900089ED99E00E944B40A0903105A982AA2014
:10D5A00009F44DC00E94407A00912D0510912E057E
:10D5B00020912F0530913005DC01CB01801B910BB0
:10D5C000A20BB30BB7FD3BC00E94407A6B017C01FC
:10D5D000B9802B2D30E0A8EEB3E00E9417E3C60E11
:10D5E000D71EE81EF91EC0922D05D0922E05E0929E
:10D5F0002F05F09230050E94934B8AE00F900F9018
:10D600000F900F90DF91CF911F910F91FF90EF90AE
:10D61000DF90CF90BF90AF909F908F907F906F9052
:10D620005F904F903F902F900C943E4460936E0516
:10D6300070936F0580937005909371055ECE0F9087
:10D640000F900F900F90DF91CF911F910F91FF904E
:10D65000EF90DF90CF90BF90AF909F908F907F9092
:10D660006F905F904F903F902F9008952F923F9230
:10D670004F925F926F927F928F929F92AF92BF92E2
:10D68000CF92DF92EF92FF920F931F93CF93DF938E
:10D69000CDB7DEB7CC54D1090FB6F894DEBF0FBEBC
:10D6A000CDBF80910E02882319F08EE395E03CD91E
:10D6B0008091110583FDA9C0C0904A05D0904B050B
:10D6C000E0904C05F0904D05209126043091270400
:10D6D0004091280450912904C701B6010E94E1DE5F
:10D6E000882309F492C080911005811133C06091A4
:10D6F00034047091350480913604909137040E946F
:10D700006BE420910C0230910D026217730714F53F
:10D71000C0922604D0922704E0922804F0922904B3
:10D72000E5EBFAE184917F019FEFE91AF90A88237A
:10D7300021F00E943E44F701F5CFE5E9F3E1849141
:10D740007F01AFEFEA1AFA0A882321F00E943E44D3
:10D75000F701F5CF80904A0590904B05A0904C05BD
:10D76000B0904D0520912604309127044091280463
:10D7700050912904C501B4010E9426E36B017C018C
:10D7800020E030E0A9010E944DE587FF04C0F7FAD0
:10D79000F094F7F8F094E0912305B4E0EB9FF001EA
:10D7A0001124E85FFD4F2081318142815381C701FF
:10D7B000B6010E9446DF20E030E048E453E40E94D6
:10D7C0004DE5181614F58092260490922704A09235
:10D7D0002804B0922904E5EBFAE184917F019FEFE0
:10D7E000E91AF90A882321F00E943E44F701F5CF97
:10D7F000E6E7F3E184917F01AFEFEA1AFA0A8823A2
:10D8000021F00E943E44F701F5CF8091EE10609028
:10D81000000270900102C0903E05D0903F05E0905C
:10D820004005F09041058090420590904305A090FE
:10D830004405B0904505882309F482C22090EF107A
:10D840003090F0104090F1105090F21020E030E055
:10D85000A901C201B1010E94E1DE882379F0209183
:10D860004605309147054091480550914905C20150
:10D87000B1010E944DE518160CF062C2B301770C9D
:10D88000880B990B0E94E7DE20913C0230913D020B
:10D8900040913E0250913F020E9446DF2AE037ED60
:10D8A00043E25CE30E9446DF6DA77EA78FA798AB9B
:10D8B00020911A0430911B0440911C0450911D04C6
:10D8C000C701B6010E9426E32B013C0120911E04F2
:10D8D00030911F044091200450912104C501B401EE
:10D8E0000E9426E325966CAF7DAF8EAF9FAF259744
:10D8F00020E030E0A901C301B2010E94E1DE811104
:10D9000041C020E030E0A90125966CAD7DAD8EAD23
:10D910009FAD25970E94E1DE811134C070902305F0
:10D9200019AA1AAA1BAA1CAAC982DA82EB82FC8253
:10D930008D829E82AF82B886809146059091470580
:10D94000A0914805B091490589879A87AB87BC8724
:10D95000AE01475F5F4FBE016B5F7F4FCE01019607
:10D960000E943EC2FE01F1966F01E72C8E01035D1D
:10D970001F4F2AE435E0AE01475F5F4FBE016B5F8A
:10D980007F4F2BC220912204309123044091240424
:10D990005091250460914605709147058091480596
:10D9A000909149050E9426E329966CAF7DAF8EAF1A
:10D9B0009FAF299720912604309127044091280495
:10D9C0005091290460914A0570914B0580914C0556
:10D9D00090914D050E9426E321966CAF7DAF8EAFEE
:10D9E0009FAF2197A3019201C301B2010E9446DFBC
:10D9F0006B017C0125962CAD3DAD4EAD5FAD2597FD
:10DA0000CA01B9010E9446DF9B01AC01C701B60102
:10DA10000E9427E36B017C0129962CAD3DAD4EADF4
:10DA20005FAD2997CA01B9010E9446DF9B01AC0195
:10DA3000C701B6010E9427E30E9492E56B017C01B9
:10DA40002DEB37E346E855E30E94E1DE87FF17C080
:10DA500020E030E0A90121966CAD7DAD8EAD9FAD8B
:10DA600021970E944DE52196CCACDDACEEACFFAC2D
:10DA7000219787FF04C0F7FAF094F7F8F0942DEBA4
:10DA800037E346E855E3C701B6010E94E1DE87FDB2
:10DA9000A8C120E030E040EA50E4C701B6010E948E
:10DAA00003E40E9470E41B01672B19F422242394E1
:10DAB000312CB10180E090E00E94E5DE9B01AC01D9
:10DAC00060E070E080E89FE30E9403E44B015C01AA
:10DAD0009B01AC01C701B6010E9446DF2D966CAFD9
:10DAE0007DAF8EAF9FAF2D97A5019401C301B20109
:10DAF0000E9446DF698B7A8B8B8B9C8BA5019401EE
:10DB000025966CAD7DAD8EAD9FAD25970E9446DF0D
:10DB10006D8B7E8B8F8B988FA501940129966CADB0
:10DB20007DAD8EAD9FAD29970E9446DF698F7A8FBC
:10DB30008B8F9C8FA501940121966CAD7DAD8EAD30
:10DB40009FAD21970E9446DF6D8F7E8F8F8F98A3A8
:10DB500080E1EAE1F4E0DE01119601900D928A95F0
:10DB6000E1F799249394F1E02F1A310809F04BC0A2
:10DB7000E09023052D968CAD9DADAEADBFAD2D973C
:10DB800089AF9AAFABAFBCAF80913E0590913F0596
:10DB9000A0914005B091410589A39AA3ABA3BCA372
:10DBA0008091420590914305A0914405B0914505AF
:10DBB0008DA39EA3AFA3B8A780914605909147057A
:10DBC000A0914805B091490589A79AA7ABA7BCA722
:10DBD000AE01475D5F4FBE016B5D7F4FCE01819609
:10DBE0000E943EC2DE01D9966D018E01035D1F4F7A
:10DBF0002AE435E0AE01475D5F4FBE016B5D7F4FAC
:10DC0000CE018196ECC080915E05811112C00E9408
:10DC1000407ADC01CB0188539F4FAF4FBF4F8093B9
:10DC20005A0590935B05A0935C05B0935D059092B7
:10DC30005E050E949B500E94407AC0905A05D09089
:10DC40005B05E0905C05F0905D05DC01CB018C1973
:10DC50009D09AE09BF09B7FD11C00E94407ADC01E1
:10DC6000CB0188539F4FAF4FBF4F80935A0590937E
:10DC70005B05A0935C05B0935D0517D96E01B1E11A
:10DC8000CB0ED11CFE0131967F015601D6012D919C
:10DC90003D914D915D916D01F701608171818281AE
:10DCA00093810E9427E3D7016D937D938D939D937C
:10DCB0007D01AA16BB0651F7E09023052D968CAD89
:10DCC0009DADAEADBFAD2D978DAB9EABAFABB8AF3D
:10DCD00089819A81AB81BC8189A39AA3ABA3BCA3A0
:10DCE0008D819E81AF81B8858DA39EA3AFA3B8A778
:10DCF00089859A85AB85BC8589A79AA7ABA7BCA760
:10DD0000AE01475D5F4FBE016B5D7F4FCE018196D7
:10DD10000E943EC2DE01D5966D018E01035D1F4F4C
:10DD20009E01235F3F4FAE01475D5F4FBE016B5DBC
:10DD30007F4FCE0181960E945C54811114CF18CF81
:10DD4000B301770C880B990B0E94E7DE20913C020F
:10DD500030913D0240913E0250913F020E9446DFC9
:10DD60002AE037ED43E25CE30E9446DF69AB7AAB21
:10DD70008BAB9CAB70902305809146059091470535
:10DD8000A0914805B0914905C982DA82EB82FC82F4
:10DD9000898A9A8AAB8ABC8A89A39AA3ABA3BCA3BB
:10DDA0001DA61EA61FA618AAAE014F5D5F4FBE019D
:10DDB0006F5E7F4FCE0101960E943EC2FE01BD966E
:10DDC0006F01E72C8E010F5C1F4F2AE435E0AE0196
:10DDD0004F5D5F4FBE016F5E7F4FCE0101960E9487
:10DDE0005C5480E1EEE3F5E0AAE1B4E001900D922D
:10DDF0008A95E1F7C45BDF4F0FB6F894DEBF0FBE24
:10DE0000CDBFDF91CF911F910F91FF90EF90DF90E9
:10DE1000CF90BF90AF909F908F907F906F905F90CA
:10DE20004F903F902F900895CF93DF9380E00E9412
:10DE30009DC1C7E1D5E0688379838A839B8381E0B4
:10DE40000E949DC16C837D838E839F8382E00E94AC
:10DE50009DC1688779878A879B87DF91CF910895D5
:10DE6000CF93DF938B3D9240B1F0E0EAFAE18491E9
:10DE7000EF012196882321F00E943E44FE01F7CF56
:10DE8000EFE5F5E18491EF012196882331F00E94BE
:10DE90003E44FE01F7CF80E001C081E0DF91CF91E9
:10DEA00008952F923F924F925F926F927F928F923E
:10DEB0009F92AF92BF92CF92DF92EF92FF920F9319
:10DEC0001F93CF93DF93CDB7DEB7C257D1090FB6FB
:10DED000F894DEBF0FBECDBF2DB63EB6A3961FAEE3
:10DEE0001EAEA39784E690E0A5969FAF8EAFA59750
:10DEF00001E09E012F593F4F44E050E0BE01695AB6
:10DF00007F4FCE018D599F4F0E9470BB9E012F59AC
:10DF10003F4F42E050E0BE016B597F4FCE018D591B
:10DF20009F4F0E9470BB43E050E0BE01695A7F4F93
:10DF30008BEE92E00E948CE6892B09F43FC06B9631
:10DF40008FAD6B97882339F08FE368968FAF689712
:10DF500069961FAE6997E5EBFAE184917F012FEF97
:10DF6000E21AF20A811103C0E2E2F6E104C00E9463
:10DF70003E44F701F2CF84917F019FEFE91AF90A3D
:10DF8000882321F00E943E44F701F5CFBE01695A73
:10DF90007F4F89E196E10E94A8C8EBE0F6E1849109
:10DFA0007F012FEFE21AF20A882321F00E943E44FB
:10DFB000F701F5CF81E080937C0554C58DB79EB7FE
:10DFC000E1969FAF8EAFE19767961CAE1DAE1EAE79
:10DFD0001FAE6797A3961FAE1EAEA39701E09E01EA
:10DFE0002F593F4F41E050E0BE0164597F4FCE01B1
:10DFF0008D599F4F0E9470BB80E1E7E6F2E0DE01A1
:10E00000919601900D928A95E1F780E1E7E7F2E0C1
:10E01000DE01519601900D928A95E1F780E1E7E8E3
:10E02000F2E0DE01119601900D928A95E1F7AD962E
:10E030004FADAD9750E04D5F5F4F440F551F440FFC
:10E04000551FEDB7FEB7E41BF50B0FB6F894FEBFF6
:10E050000FBEEDBF8DB79EB701967C0100E09E011B
:10E060002F593F4FBC01CE018D599F4F0E9470BB6D
:10E070009E012F593F4F44E050E064E075E0CE012F
:10E080008D599F4F0E9470BBAD968FACAD97912C70
:10E0900093E0890E911C880C991C880C991CEDB793
:10E0A000FEB7E819F9090FB6F894FEBF0FBEEDBF31
:10E0B0008DB79EB701966C01E819F9090FB6F8946F
:10E0C000FEBF0FBEEDBF8DB79EB701965C019E01EE
:10E0D0002F593F4FA401B601CE018D599F4F0E9489
:10E0E00070BB9E012F593F4FA401B501CE018D5940
:10E0F0009F4F0E9470BB90917D05AF969FAFAF97E9
:10E10000992309F4A2C000E09E012F593F4F44E03B
:10E1100050E06CEE74E0CE018D599F4F0E9470BBB1
:10E120009E012F593F4F44E050E060EF74E0CE0174
:10E130008D599F4F0E9470BB9E012F593F4F44E065
:10E1400050E068EE74E0CE018D599F4F0E9470BB85
:10E150009E012F593F4F44E050E06CE075E0CE0146
:10E160008D599F4F0E9470BB9E012F593F4F44E035
:10E1700050E068E075E0CE018D599F4F0E9470BB62
:10E180009E012F593F4F40E150E064ED74E0CE0115
:10E190008D599F4F0E9470BB9E012F593F4F44E005
:10E1A00050E0BE016D5A7F4FCE018D599F4F0E94A6
:10E1B00070BB9E012F593F4F4CE050E068E875E07E
:10E1C000CE018D599F4F0E9470BB9E012F593F4F2A
:10E1D00044E050E067E670E1CE018D599F4F0E9408
:10E1E00070BB9E012F593F4F44E050E0BE016D5A75
:10E1F0007F4FCE018D599F4F0E9470BB01E09E0161
:10E200002F593F4F41E050E0BE0165597F4FCE018D
:10E210008D599F4F0E9470BB9E012F593F4F41E087
:10E2200050E0BE0166597F4FCE018D599F4F0E942D
:10E2300070BBAC968FADAC97AB96CFACAB978C9DCB
:10E2400060011124E12CF12C71C0AD968FADAD971A
:10E2500090E0029604EF14E0B501DE011196E4E3CC
:10E260008E2EE1E19E2EAE014F5E5F4FF4E1AF2EA8
:10E27000F1E1BF2EE396FFAEEEAEE3977E01E1E261
:10E28000EE0EF11C20E030E0821793072CF0E396AD
:10E29000EEADFFADE39701C0F70140805180628091
:10E2A0007380F50141925192619271925F018217E0
:10E2B000930714F0F60101C0FA014080518062809A
:10E2C0007380F40141925192619271924F018217D1
:10E2D000930734F0FB01408051806280738005C059
:10E2E0004D905D906D907C901397F8014192519202
:10E2F000619271928F012F5F3F4F6C5F7F4F149639
:10E30000F4E0CF0ED11C4C5F5F4FE396EEADFFAD56
:10E31000E3973496E396FFAFEEAFE397F4E0EF0EAA
:10E32000F11C2430310509F0AFCFEDCE00E09E01A5
:10E330002F593F4F44E050E0EC14FD0461F0BE0162
:10E340006D5A7F4FCE018D599F4F0E9470BB2FEFAA
:10E35000E21AF20AEBCF65E174E0CE018D599F4FCE
:10E360000E9470BB6AE0F62EFA94FF2079F000E07C
:10E370009E012F593F4F44E050E0BE016D5A7F4F40
:10E38000CE018D599F4F0E9470BBEECF01E09E01E0
:10E390002F593F4F41E050E0BE0167597F4FCE01FA
:10E3A0008D599F4F0E9470BB9E012F593F4F41E0F6
:10E3B00050E0BE0168597F4FCE018D599F4F0E949A
:10E3C00070BBAA968FADAA97853091F5A9968FADAF
:10E3D000A997853069F5AF968FADAF97811102C0CF
:10E3E0000E94459300E09E012F593F4F44E050E0CA
:10E3F0006BE670E1CE018D599F4F0E9470BB9E016C
:10E400002F593F4F44E050E068E775E0CE018D5949
:10E410009F4F0E9470BB9E012F593F4F44E650E032
:10E4200063E770E1CE018D599F4F0E9470BB3BC0E6
:10E4300000E09E012F593F4F44E050E0BE01635C75
:10E440007F4FCE018D599F4F0E9470BB9E012F5967
:10E450003F4F44E050E0BE016F5C7F4FCE018D59CD
:10E460009F4F0E9470BBAA968FADAA97A996CFAC7A
:10E47000A9978C9D60011124E12CF12CCE14DF04AE
:10E4800091F000E09E012F593F4F44E050E0BE0163
:10E490006D5A7F4FCE018D599F4F0E9470BB9FEFE9
:10E4A000E91AF90AEBCF00E09E012F593F4F41E0F6
:10E4B00050E0BE0163597F4FCE018D599F4F0E949E
:10E4C00070BB9E012F593F4F41E050E0BE0169599A
:10E4D0007F4FCE018D599F4F0E9470BB9E012F59D7
:10E4E0003F4F44E050E0BE016D5A7F4FCE018D5941
:10E4F0009F4F0E9470BB9E012F593F4F44E050E058
:10E50000BE016D5A7F4FCE018D599F4F0E9470BB47
:10E510009E012F593F4F44E050E06FE670E1CE017D
:10E520008D599F4F0E9470BB9E012F593F4F44E071
:10E5300050E0BE01615B7F4FCE018D599F4F0E941D
:10E5400070BB9E012F593F4F44E050E0BE01655B18
:10E550007F4FCE018D599F4F0E9470BB9E012F5956
:10E560003F4F44E050E0BE01695B7F4FCE018D59C3
:10E570009F4F0E9470BB10E000E09E012F593F4F5B
:10E5800044E050E0BE016D5A7F4FCE018D599F4F40
:10E590000E9470BB111110C06796CCACDDACEEAC24
:10E5A000FFAC679720E030E84BE355E4C701B601C4
:10E5B0000E94E1DE811103C054E0F52E33C080914A
:10E5C0007D05811108C0C0926E04D0926F04E09264
:10E5D0007004F092710400E09E012F593F4F44E017
:10E5E00050E06AE674E0CE018D599F4F0E9470BBE7
:10E5F0009E012F593F4F44E050E062E774E0CE01A6
:10E600008D599F4F0E9470BB9E012F593F4F44E090
:10E6100050E0BE016D5A7F4FCE018D599F4F0E9431
:10E6200070BB12C0FA94FF2079F000E09E012F59D0
:10E630003F4F44E050E0BE016D5A7F4FCE018D59EF
:10E640009F4F0E9470BBEECF1F5F153009F094CF33
:10E6500000E09E012F593F4F42E050E0BE01615A59
:10E660007F4FCE018D599F4F0E9470BB9E012F5945
:10E670003F4F44E050E0BE016D5A7F4FCE018D59AF
:10E680009F4F0E9470BB6796CCACDDACEEACFFAC8C
:10E69000679720E030E84BE355E4C701B6010E94DC
:10E6A000E1DE882329F180917D05811108C0C092A7
:10E6B0006604D0926704E0926804F092690400E076
:10E6C0009E012F593F4F44E050E062E674E0CE01D6
:10E6D0008D599F4F0E9470BB9E012F593F4F44E0C0
:10E6E00050E06EE574E0CE018D599F4F0E9470BBE3
:10E6F00000E09E012F593F4F42E050E0BE01635AB7
:10E700007F4FCE018D599F4F0E9470BB9E012F59A4
:10E710003F4F41E050E0BE0163597F4FCE018D591C
:10E720009F4F0E9470BB19E0115000E09E012F59CD
:10E730003F4F112359F044E050E0BE016D5A7F4F26
:10E74000CE018D599F4F0E9470BBEECF41E050E04B
:10E7500067EF70E1CE018D599F4F0E9470BBF12C85
:10E7600000E09E012F593F4F44E050E0BE016D5A3A
:10E770007F4FCE018D599F4F0E9470BB10917D0538
:10E78000111110C0F1100EC067968CAD9DADAEADED
:10E79000BFAD67978093FC109093FD10A093FE107F
:10E7A000B093FF10F394E5E0FE12DACF111102C02E
:10E7B0000E94CF944CE0F42EFA94F11003C03CE098
:10E7C000F32E0FC000E09E012F593F4F42E050E072
:10E7D000BE01655A7F4FCE018D599F4F0E9470BB7D
:10E7E000EBCFFA9400E09E012F593F4FFF2059F0E4
:10E7F00044E050E0BE016D5B7F4FCE018D599F4FCD
:10E800000E9470BBEECF46E050E0BE01635C7F4FDC
:10E81000CE018D599F4F0E9470BB9E012F593F4FD3
:10E8200044E050E064EE74E0CE018D599F4F0E94A9
:10E8300070BB9E012F593F4F4CE050E0BE016F5C12
:10E840007F4FCE018D599F4F0E9470BB2CE1F22E5D
:10E85000FA94F11003C094E0F92E1DC000E09E016F
:10E860002F593F4F44E050E0BE016D5A7F4FCE011B
:10E870008D599F4F0E9470BBEBCF00E09E012F5936
:10E880003F4F44E050E0BE016D5A7F4FCE018D599D
:10E890009F4F0E9470BBFA94F110EFCF8BE0F82EDF
:10E8A000FA94FF2079F000E09E012F593F4F44E099
:10E8B00050E0BE016D5A7F4FCE018D599F4F0E948F
:10E8C00070BBEECFA5968EAD9FADA59784569109EE
:10E8D000C7DA80937C05882309F1E5EBFAE184919E
:10E8E0007F012FEFE21AF20A882321F00E943E44B2
:10E8F000F701F5CFA5966EAD7FADA597645671096A
:10E9000083E096E10E948FC86BED72E08BEF95E19A
:10E910000E948FC88AE00E943E4499C0A3962EAD03
:10E920003FADA397A7968EAD9FADA7972817390740
:10E9300009F44BC081E080937C05E0EAFAE1849120
:10E940007F019FEFE91AF90A811103C0EBEDF5E1B0
:10E9500004C00E943E44F701F2CF84917F012FEF63
:10E96000E21AF20A882321F00E943E44F701F5CF13
:10E97000A7966EAD7FADA79780E090E04AE00E9439
:10E980004544E6EDF5E184917F019FEFE91AF90A2C
:10E99000882321F00E943E44F701F5CFA3966EAD87
:10E9A0007FADA39780E090E04AE00E944544E6EC0A
:10E9B000F5E184917F012FEFE21AF20A882309F42E
:10E9C00046C00E943E44F701F4CF111142C0E5EB6E
:10E9D000FAE184917F019FEFE91AF90A811103C0DE
:10E9E0000BEE12E004C00E943E44F701F2CFF801A2
:10E9F00081918F01882319F00E943E44F8CFA5969B
:10EA00006EAD7FADA5976456710989EA95E10E94C4
:10EA10008FC8A3964EAD5FADA39760E070E08CE920
:10EA200095E10E9455C8E9E9F5E184917F012FEF56
:10EA3000E21AF20A811107C080917C05811109C098
:10EA40000E942FBC06C00E943E44F701EECF112366
:10EA500099F3E1968EAD9FADE1970FB6F8949EBF06
:10EA60000FBE8DBF80917D05811102C00E9486AFCF
:10EA700090917C0581E089270FB6F8943EBE0FBEC9
:10EA80002DBECE58DF4F0FB6F894DEBF0FBECDBF00
:10EA9000DF91CF911F910F91FF90EF90DF90CF907A
:10EAA000BF90AF909F908F907F906F905F904F90AE
:10EAB0003F902F90089581E080937D05F2D91092C8
:10EAC0007D058111EEC90E9469B481E008958F929D
:10EAD0009F92AF92BF92CF92DF92EF92FF920F93ED
:10EAE0001F93CF93DF93CDB7DEB7CE59D1090FB6C1
:10EAF000F894DEBF0FBECDBFE9961CAE1DAE1EAEB4
:10EB00001FAEE9978091C5039091C603A091C703FA
:10EB1000B091C803ED968CAF9DAFAEAFBFAFED9790
:10EB2000C157DF4F19821882CF58D04084E690E059
:10EB3000CF56DF4F99838883C159D04010927C050E
:10EB40009E0121573F4F44E050E0BE0167587F4F80
:10EB5000CE018F569F4F0E94BCBBCF56DF4F88819E
:10EB60009981C159D0400296CF56DF4F998388834F
:10EB7000C159D040C157DF4F19821882CF58D040B9
:10EB800081E0C956DF4F8883C759D0409E01215785
:10EB90003F4F41E050E0BE0169567F4FCE018F5696
:10EBA0009F4F0E94BCBB9E0121573F4F40E150E068
:10EBB00064E171E1CE018F569F4F0E94BCBB9E0164
:10EBC00021573F4F44E050E064E075E0CE018F569E
:10EBD0009F4F0E94BCBB9E0121573F4F40E150E038
:10EBE00064E371E1CE018F569F4F0E94BCBB9E0132
:10EBF00021573F4F40E150E064EF74E0CE018F5663
:10EC00009F4F0E94BCBB9E0121573F4F44E050E004
:10EC10006CEE74E0CE018F569F4F0E94BCBB9E01EC
:10EC200021573F4F44E050E060EF74E0CE018F5633
:10EC30009F4F0E94BCBB9E0121573F4F44E050E0D4
:10EC400068EE74E0CE018F569F4F0E94BCBB9E01C0
:10EC500021573F4F44E050E06CE075E0CE018F5605
:10EC60009F4F0E94BCBB9E0121573F4F44E050E0A4
:10EC700068E075E0CE018F569F4F0E94BCBB9E019D
:10EC800021573F4F40E150E064ED74E0CE018F56D4
:10EC90009F4F0E94BCBB8AE097EDA3EABCE3E996D4
:10ECA0008CAF9DAFAEAFBFAFE9979E0121573F4FED
:10ECB00044E050E0BE016B587F4FCE018F569F4F0E
:10ECC0000E94BCBB9E0121573F4F4CE050E068E8DA
:10ECD00075E0CE018F569F4F0E94BCBB8091EF1014
:10ECE0009091F010A091F110B091F210C358DF4F45
:10ECF00088839983AA83BB83CD57D0409E01215737
:10ED00003F4F44E050E0BE0163587F4FCE018F5625
:10ED10009F4F0E94BCBBE9961CAE1DAE1EAE1FAE3F
:10ED2000E99783E0C856DF4F8883C859D040C7565B
:10ED3000DF4F8883C959D0409E0121573F4F44E09F
:10ED400050E0BE016B587F4FCE018F569F4F0E94FF
:10ED5000BCBB9E0121573F4F41E050E0BE016856C9
:10ED60007F4FCE018F569F4F0E94BCBB9E01215703
:10ED70003F4F41E050E0BE0167567F4FCE018F56B6
:10ED80009F4F0E94BCBB1AE011509E0121573F4F7C
:10ED900044E050E0112349F0BE016B587F4FCE0193
:10EDA0008F569F4F0E94BCBBEFCF65E174E0CE0150
:10EDB0008F569F4F0E94BCBBE9961CAE1DAE1EAE87
:10EDC0001FAEE9971AE0115071F09E0121573F4F95
:10EDD00044E050E0BE016B587F4FCE018F569F4FED
:10EDE0000E94BCBBF0CF85E0C656DF4F8883CA596E
:10EDF000D040C556DF4F8883CB59D0409E01215764
:10EE00003F4F41E050E0BE0166567F4FCE018F5626
:10EE10009F4F0E94BCBB9E0121573F4F41E050E0F5
:10EE2000BE0165567F4FCE018F569F4F0E94BCBBDF
:10EE30009E0121573F4F44E050E06BE670E1CE0168
:10EE40008F569F4F0E94BCBB9E0121573F4F44E00D
:10EE500050E068E775E0CE018F569F4F0E94BCBB23
:10EE60009E0121573F4F44E650E063E770E1CE0139
:10EE70008F569F4F0E94BCBBC456DF4F1882CC599F
:10EE8000D0408FEFC356DF4F8883CD59D0409E01CD
:10EE900021573F4F41E050E0BE0164567F4FCE0105
:10EEA0008F569F4F0E94BCBB9E0121573F4F41E0B0
:10EEB00050E0BE0163567F4FCE018F569F4F0E9498
:10EEC000BCBBE9961CAE1DAE1EAE1FAEE9979E01FF
:10EED00021573F4F44E050E0BE016B587F4FCE01B9
:10EEE0008F569F4F0E94BCBB9E0121573F4F44E06D
:10EEF00050E0BE016B587F4FCE018F569F4F0E944E
:10EF0000BCBB9E0121573F4F44E050E06FE670E1EB
:10EF1000CE018F569F4F0E94BCBB8091970290916B
:10EF20009802A0919902B0919A02CF57DF4F88833F
:10EF30009983AA83BB83C158D04080919B02909152
:10EF40009C02A0919D02B0919E02CB57DF4F888317
:10EF50009983AA83BB83C558D040C757DF4F198216
:10EF60001882C958D040C557DF4F19821882CB5834
:10EF7000D0409E0121573F4F44E050E0BE016F5703
:10EF80007F4FCE018F569F4F0E94BCBB9E012157E1
:10EF90003F4F44E050E0BE016B577F4FCE018F568C
:10EFA0009F4F0E94BCBB9E0121573F4F44E050E061
:10EFB000BE0167577F4FCE018F569F4F0E94BCBB4B
:10EFC00010E0C12C80E8D82E8BE3E82E85E4F82EE3
:10EFD000812C912C90E8A92E9FE3B92E111138C0F5
:10EFE0009E0121573F4F44E050E06EE674E0CE01B1
:10EFF0008F569F4F0E94BCBB9E0121573F4F44E05C
:10F0000050E06AE674E0CE018F569F4F0E94BCBB71
:10F010009E0121573F4F44E050E062E774E0CE018B
:10F020008F569F4F0E94BCBBE9968CAE9DAEAEAE94
:10F03000BFAEE9979E0121573F4F44E050E0BE012B
:10F040006B587F4FCE018F569F4F0E94BCBB2AC08A
:10F05000E996CCAEDDAEEEAEFFAEE9979E0121574C
:10F060003F4F44E050E0BE016B587F4FCE018F56BA
:10F070009F4F0E94BCBBE9961CAE1DAE1EAE1FAEDC
:10F08000E99704E0015071F09E0121573F4F44E0A1
:10F0900050E0BE016B587F4FCE018F569F4F0E94AC
:10F0A000BCBBF0CF1F5F153009F098CF84E190E032
:10F0B000CD56DF4F99838883C359D0409E01215795
:10F0C0003F4F42E050E0BE016D567F4FCE018F565C
:10F0D0009F4F0E94BCBB9E0121573F4F44E050E030
:10F0E00066E674E0CE018F569F4F0E94BCBB9E0126
:10F0F00021573F4F44E050E062E674E0CE018F5666
:10F100009F4F0E94BCBB9E0121573F4F44E050E0FF
:10F110006EE574E0CE018F569F4F0E94BCBB80E22B
:10F1200090E0CB56DF4F99838883C559D0409E012C
:10F1300021573F4F42E050E0BE016B567F4FCE015A
:10F140008F569F4F0E94BCBBC256DF4F1882CE59CC
:10F15000D04080E2EFE9F2E0DE019D9601900D9251
:10F160008A95E1F79E0121573F4F41E050E0BE01F3
:10F1700062567F4FCE018F569F4F0E94BCBB9E01AF
:10F1800021573F4F40E250E0BE01635D7F4FCE010B
:10F190008F569F4F0E94BCBB9E0121573F4F41E0BD
:10F1A00050E067EF70E1CE018F569F4F0E94BCBBCD
:10F1B00010E011110EC08091FC109091FD10A091F3
:10F1C000FE10B091FF10E9968CAF9DAFAEAFBFAF10
:10F1D000E9979E0121573F4F44E050E0BE016B5834
:10F1E0007F4FCE018F569F4F0E94BCBB1F5F1530D3
:10F1F00001F7BE01635B7F4F86E1FB0111928A95A7
:10F20000E9F79E0121573F4F46E150E0CE018F566E
:10F210009F4F0E94BCBB8CE2EFEBF2E0DE01119647
:10F2200001900D928A95E1F79E0121573F4F4CE2E4
:10F2300050E0BE016F5F7F4FCE018F569F4F0E94FF
:10F24000BCBBBE0161597F4F86E0FB0111928A95DC
:10F25000E9F79E0121573F4F46E050E0CE018F561F
:10F260009F4F0E94BCBB9E0121573F4F44E050E09E
:10F2700064EE74E0CE018F569F4F0E94BCBBBE016E
:10F280006D597F4F8CE0FB0111928A95E9F79E0141
:10F2900021573F4F4CE050E0CE018F569F4F0E94C8
:10F2A000BCBBE9961CAE1DAE1EAE1FAEE9971CE1BD
:10F2B000115071F09E0121573F4F44E050E0BE01D4
:10F2C0006B587F4FCE018F569F4F0E94BCBBF0CF33
:10F2D000E9961CAE1DAE1EAE1FAEE99714E01150AC
:10F2E00071F09E0121573F4F44E050E0BE016B5842
:10F2F0007F4FCE018F569F4F0E94BCBBF0CFE99647
:10F300001CAE1DAE1EAE1FAEE9971BE0115071F092
:10F310009E0121573F4F44E050E0BE016B587F4FA4
:10F32000CE018F569F4F0E94BCBBF0CF80917C05D1
:10F33000811167C0CF56DF4FE880F980C159D040B6
:10F34000F4E6EF1AF108C157DF4F88819981CF5851
:10F35000D040C357DF4F99838883CD58D04084E68F
:10F3600090E0CF56DF4F99838883C159D0409E01EA
:10F3700021573F4F44E050E06BEE72E0CE018F56D4
:10F380009F4F0E94BCBB9E0121573F4F42E050E07F
:10F39000BE0163577F4FCE018F569F4F0E94BCBB6B
:10F3A000E5EBFAE184918F010F5F1F4F882321F075
:10F3B0000E943E44F801F6CFB70187E895E10E942C
:10F3C0008FC8C357DF4F48815981CD58D04060E086
:10F3D00070E08AE795E10E9455C8E7E7F5E184917E
:10F3E0008F010F5F1F4F882321F00E943E44F801D8
:10F3F000F6CFC7010E94306F90917C05892B8093D6
:10F400007C0590917C0581E08927C256DF4F0FB6BD
:10F41000F894DEBF0FBECDBFDF91CF911F910F914A
:10F42000FF90EF90DF90CF90BF90AF909F908F9024
:10F4300008950E942AE63FB7F89480911F079091A3
:10F440002007A0912107B091220726B5A89B05C0EF
:10F450002F3F19F00196A11DB11D3FBFBA2FA92F53
:10F46000982F8827820F911DA11DB11DBC01CD01D0
:10F4700042E0660F771F881F991F4A95D1F70895BC
:10F480002FB7F89460911B0770911C0780911D079E
:10F4900090911E072FBF08951F920F920FB60F92E3
:10F4A00011242F933F938F939F93AF93BF9380919A
:10F4B0001B0790911C07A0911D07B0911E0730916A
:10F4C0001A0723E0230F2D3720F40196A11DB11D4B
:10F4D00005C026E8230F0296A11DB11D20931A072F
:10F4E00080931B0790931C07A0931D07B0931E07E2
:10F4F00080911F0790912007A0912107B0912207CA
:10F500000196A11DB11D80931F0790932007A09322
:10F510002107B0932207BF91AF919F918F913F91A7
:10F520002F910F900FBE0F901F9018952F923F9222
:10F530004F925F926F927F928F929F92AF92BF9203
:10F54000CF92DF92EF92FF920F931F93CF93DF93AF
:10F55000CDB7DEB762970FB6F894DEBF0FBECDBF52
:10F560008091110583FDBFC183E50E9469468C87A8
:10F57000811106C082E50E946946882309F4B3C15F
:10F580000E94F7430E946BE46E3671050CF0A8C12F
:10F5900070932D0460932C040E946D4C0E94F743DD
:10F5A00020E030E040EA50E40E944DE5181614F4E3
:10F5B0000E941B94EDE8F9E18491FB83EA838823A0
:10F5C00071F0082E000C990B0E94E2864A815B8143
:10F5D0004F5F5F4F5B834A83FA018491F0CF8DE0E8
:10F5E00090E00E94E2868AE090E00E94E286E4E6F3
:10F5F000F9E184919F012F5F3F4F3B832A8388234A
:10F6000029F00E943E44EA81FB81F3CF81E08093A0
:10F6100026021092240580912305809380041A828B
:10F620001B821C821D82188619861A861B861982E7
:10F630001D863CE33E874CE14F8756E4588B312CC6
:10F64000212C80E8898B9FEB9A8B812C912C540183
:10F6500060912C0470912D04072E000C880B990BDF
:10F660000E94E7DE7B018C019B01AC01632D722DB2
:10F6700089899A890E94E1DE882339F120912E043C
:10F6800030912F044091300450913104AC85B70182
:10F69000C801A1110BC00E94E1DE881F8827881FC6
:10F6A00089833E2C2F2C098B1A8B0FC00E94E1DE20
:10F6B00087FF06C0EFEBF9E18491FB83EA83E5C0A5
:10F6C0003E2C2F2C098B1A8B1982DADE6B017C0100
:10F6D000DC01CB01288539854A855B85821B930B2C
:10F6E000A40BB50BB7FD3BC0D701C60188519C4F99
:10F6F000AF4FBF4F88879987AA87BB870E94934BDC
:10F70000E3ECF9E184913F019FEF691A790A8823BC
:10F7100021F00E943E44F301F5CF81149104A1042D
:10F72000B104B9F0D501C401805F984DAF4FBF4F10
:10F73000BC01CD016C197D098E099F0928EE33E0CB
:10F7400040E050E00E94CFE2CA01B9010E94B044FB
:10F7500003C08FE30E943E448AE00E943E440E9420
:10F7600055678EDE609325057093260580932705E7
:10F7700090932805A0912E04AE83B0912F04BF83EF
:10F7800000913004109131040E947B2F2E813F8123
:10F79000A801632D722D89899A890E9426E32B0185
:10F7A0003C0120E030E0A9010E944DE587FF04C044
:10F7B00077FA709477F8709481149104A104B104DD
:10F7C00059F420E030E040E85FE3C301B2010E9459
:10F7D000E1DE87FF0DC00AC020E030E040E450E4E5
:10F7E000C301B2010E944DE5181614F446015701F9
:10F7F000E981EE2391F12A813B814C815D812115C4
:10F8000031054105510541F0D701C601821B930B1B
:10F81000A40BB50BB7FD21C02E813F81A8016D85DA
:10F820007E858F8598890E9426E320E030E040ECB9
:10F830005FE30E94E1DE87FD3DCFD701C601805A1C
:10F840009541AF4FBF4F8A839B83AC83BD839E811D
:10F850009D87AF81AE870F87188B80912602882302
:10F8600009F428CF81149104A104B10409F4F0CE65
:10F87000B0E1CB1AB7E2DB0AE108F108C818D908F1
:10F88000EA08FB08F7FE16CFE3CE882361F0082EC6
:10F89000000C990B0E94E286EA81FB813196FB8382
:10F8A000EA838491F2CF8DE090E00E94E2868AE0C4
:10F8B00090E00E94E286E1E9F9E184919F012F5FE7
:10F8C0003F4F3B832A83882329F00E943E44EA81EC
:10F8D000FB81F3CF8091260281E08093240503C051
:10F8E0006EE670E055CE62960FB6F894DEBF0FBE9E
:10F8F000CDBFDF91CF911F910F91FF90EF90DF90DF
:10F90000CF90BF90AF909F908F907F906F905F90BF
:10F910004F903F902F9008959F92AF92BF92CF92B9
:10F92000DF92EF92FF920F931F93CF93DF9383E6C3
:10F93000A82E82E0B82E0EE315E0CAE1D4E09AEDDD
:10F94000C92E90E1D92E28E0E22E24E0F22E912C4F
:10F95000F50181915F010E942046882309F10E94F0
:10F96000F743F7012081211104C020910C042223C8
:10F9700039F0288139814A815B810E9427E30AC0DE
:10F98000F3E09F1639F0F6012081318142815381E5
:10F990000E9426E3F801608371838283938309C008
:10F9A00088819981AA81BB81F80180839183A28398
:10F9B000B38393940C5F1F4F2496F4E0CF0ED11CB9
:10F9C0002FEFE21AF20A84E09812C2CF86E40E9476
:10F9D00069468823C9F00E94F74320E030E0A9017E
:10F9E0000E944DE5181684F40E94F74320E030E0B1
:10F9F00040E752E40E9403E460933C0270933D02AE
:10FA000080933E0290933F02DF91CF911F910F911F
:10FA1000FF90EF90DF90CF90BF90AF909F900895B0
:10FA20002F923F924F925F926F927F929F92AF92EE
:10FA3000BF92CF92DF92EF92FF920F931F93CF93DB
:10FA4000DF93CDB7DEB764970FB6F894DEBF0FBE75
:10FA5000CDBF1A012B01922EF32EC82ED12CF60108
:10FA6000E45AFA4EE491AA24A3941E160CF4A12C95
:10FA7000BB24B39420E030E0A901C201B1010E948F
:10FA80004DE518160CF0B12CCC0CDD1CCC0CDD1C9B
:10FA9000C601865E9B4F3C01FC01108211821282DE
:10FAA00013820E94FE92F3012082318242825382AD
:10FAB000E090230520E030E0A901B801892D9F2DB9
:10FAC0000E94E1DE81110AC0F601E15FFA4E8591E4
:10FAD0009591A591B4918C019A2EFB2EC801A92D68
:10FAE000BF2D898B9A8BAB8BBC8B8091220490911C
:10FAF0002304A0912404B091250440911E04509148
:10FB00001F04609120047091210400911A04109147
:10FB10001B0420911C0430911D0409831A832B833C
:10FB20003C834D835E836F83788789879A87AB8711
:10FB3000BC871D861E861F86188AAE01475F5F4FF1
:10FB4000BE016B5F7F4FCE0101960E943EC2CE0187
:10FB50000D966C018E010F5E1F4F26E234E0AE0160
:10FB6000475F5F4FBE016B5F7F4F0C970E945C54F5
:10FB70000E947E64AB1459F080919805882319F097
:10FB80001092980504C085EF97E10E940367649680
:10FB90000FB6F894DEBF0FBECDBFDF91CF911F919E
:10FBA0000F91FF90EF90DF90CF90BF90AF909F901C
:10FBB0007F906F905F904F903F902F900895CF92DD
:10FBC000DF92EF92FF9260916B1070916C10072E94
:10FBD000000C880B990B0E94E7DE6B017C012DEB7A
:10FBE00037E346E855EB0E944DE587FD0AC02DEB53
:10FBF00037E346E855E3C701B6010E94E1DE181677
:10FC00004CF4A701960160E070E080E89FE30E9459
:10FC100003E403C060E070E0CB016093721770935F
:10FC20007317809374179093751760916D1070918E
:10FC30006E10072E000C880B990B0E94E7DE6B01FB
:10FC40007C012DEB37E346E855EB0E944DE587FD3F
:10FC50000AC02DEB37E346E855E3C701B6010E9421
:10FC6000E1DE18164CF4A701960160E070E080E830
:10FC70009FE30E9403E403C060E070E0CB01609367
:10FC80007617709377178093781790937917FF9072
:10FC9000EF90DF90CF9008952F923F924F925F9216
:10FCA0006F927F928F929F92AF92BF92CF92DF928C
:10FCB000EF92FF920F931F93CF93DF93CDB7DEB7F1
:10FCC000A5970FB6F894DEBF0FBECDBF0E9409B650
:10FCD000811141C48091EE10882369F08FE40E9465
:10FCE0006946882319F00E94114603C08FE40E94E0
:10FCF0002046811130C41091EE1087E50E94204605
:10FD0000882309F428C180916B1090916C10892B85
:10FD1000D1F4E0EAFAE184918F010F5F1F4F811166
:10FD200003C0E4E7F8E104C00E943E44F801F3CFC9
:10FD300084918F010F5F1F4F882309F40CC40E9428
:10FD40003E44F801F5CF8AE50E946946882379F0A0
:10FD50000E94F7432091E2103091E3104091E410AB
:10FD60005091E5100E9426E34B015C0108C0809091
:10FD7000220490902304A0902404B090250420E055
:10FD800030E040E251ECC501B4010E944DE587FD31
:10FD90000AC020E030E040E251E4C501B4010E9415
:10FDA000E1DE1816D4F4E0EAFAE184918F010F5FE6
:10FDB0001F4F811103C0E7E6F8E104C00E943E44F2
:10FDC000F801F3CF84918F010F5F1F4F882309F44F
:10FDD000C2C30E943E44F801F5CF88E50E946946FF
:10FDE000882319F00E94F74304C060E070E080ECC3
:10FDF0009FE72091DA103091DB104091DC10509198
:10FE0000DD100E9426E36B017C0189E50E946946B2
:10FE1000882319F00E94F74304C060E070E080EC92
:10FE20009FE72091DE103091DF104091E01050915B
:10FE3000E1100E9426E32B013C0189E40E946946FF
:10FE4000882319F00E94004601C08FEF382E8AE403
:10FE50000E946946882319F00E94004601C08FEF76
:10FE6000082FA7019601C701B6010E94D3E58111B1
:10FE70004EC0A3019201C301B2010E94D3E58111DA
:10FE800046C06091780570917905072E000C880BAB
:10FE9000990B0E94E7DE9B01AC01C701B6010E94ED
:10FEA00026E320E030E0A9010E9427E320E030E0D3
:10FEB000A9010E9403E40E946BE4F62E60917A058A
:10FEC00070917B05072E000C880B990B0E94E7DED2
:10FED0009B01AC01C301B2010E9426E320E030E0A7
:10FEE000A9010E9427E320E030E0A9010E9403E479
:10FEF0000E946BE4EF2DE5300CF0E4E03E2EE7FDD0
:10FF0000312C062F65300CF004E007FD00E024E002
:10FF1000231508F420C3063008F01DC380E00E94BA
:10FF20004593332D85E03802F0011124E00FF11DD7
:10FF300007FDFA95EE0FFF1FEE0FFF1FED58FF4E66
:10FF400080829182A282B382812F0E9445931123E5
:10FF500009F401C3B6C08AE40E942046882309F44C
:10FF6000B3C00E949693F7C2E418F508F7FE03C0E9
:10FF700033E0E30EF11C5701B594A794B594A79410
:10FF8000B5010B2C000C880B990B0E94E7DE6A8FE1
:10FF90007B8F8C8F9D8FC618D708D7FE03C083E058
:10FFA000C80ED11C46019594879495948794B4010A
:10FFB000092C000C880B990B0E94E7DE6B017C0179
:10FFC0000E94968D60916B1070916C10072E000C42
:10FFD000880B990B0E94E7DE9B01AC016A8D7B8D3B
:10FFE0008C8D9D8D0E94E1DE81117AC160916D1032
:10FFF00070916E10072E000C880B990B0E94E7DEA3
:020000021000EC
:100000009B01AC01C701B6010E94E1DE811168C10C
:1000100080917805909179054816590609F060C1DC
:1000200080917A0590917B056816790609F058C190
:1000300085E40E946946882309F466C10E9411463E
:1000400081111CC292E0998B212C312CA1E0A88B4C
:10005000812C912C5401B1E0BE87E5E0ED87198633
:10006000888991E08927888BC101032C000CAA0B99
:10007000BB0B8AA39BA3ACA3BDA39D85A9859A13A3
:1000800047C1F4E02F16310449F0A5019401C501E0
:10009000B4010E94D3E5882309F44AC280E00E949B
:1000A000C38E882309F4EDC1812F0E9445930E94DD
:1000B0007D8D81E0809324058091EE1081110E9456
:1000C000FE920E9479A547C286E50E946946882370
:1000D00009F4EFC00E94F0457B876A87AA85BB853B
:1000E000159768F0EFE3F8E184918F010F5F1F4FE0
:1000F000882309F430C20E943E44F801F5CF84E41D
:100100000E946946882319F00E94114603C084E4C6
:100110000E9420468C878AE50E946946882339F030
:100120000E94F7436E8F7F8F88A399A304C01E8E11
:100130001F8E18A219A283E50E946946882319F030
:100140000E94F74304C060E070E08AEF95E420E08D
:1001500030E040E752E40E9403E460933802709379
:10016000390280933A0290933B028CE40E946946E4
:10017000882381F00E94F7432091DA103091DB1040
:100180004091DC105091DD100E9426E30E946BE448
:100190002B0103C0E1E24E2E512C82E50E946946FC
:1001A000882381F00E94F7432091DA103091DB1010
:1001B0004091DC105091DD100E9426E30E946BE418
:1001C0007B0103C078ECE72EF12C86E40E9469469F
:1001D000882381F00E94F7432091DE103091DF10D8
:1001E0004091E0105091E1100E9426E30E946BE4E0
:1001F0003B0103C06AE0662E712C82E40E946946CE
:10020000882381F00E94F7432091DE103091DF10A7
:100210004091E0105091E1100E9426E30E946BE4AF
:100220006B0103C058ECC52ED12CB301072C000C78
:10023000880B990B0E94E7DE6A8B7B8B8C8B9D8BE6
:10024000B201052C000C880B990B0E94E7DE6E8B27
:100250007F8B888F998F2A893B894C895D890E9481
:100260005F66811103C0E3E2F8E118C0B6010D2C0E
:10027000000C880B990B0E94E7DE4B015C01B70173
:100280000F2C000C880B990B0E94E7DEA50194014E
:100290000E945F668F8781110FC0E5CF84918F0127
:1002A0000F5F1F4F882309F456C10E943E44F80196
:1002B000F5CF1B861A8612CFAA85BB85AB2B09F01A
:1002C000BCC00E947E6480E00E94459381E00E9451
:1002D000C38E882309F448CE812F0E9445933BC1E9
:1002E0000E949693B0926C10A0926B1090926E1038
:1002F00080926D10509279054092780570927B053E
:1003000060927A0510E094CE85E40E94204698CE53
:100310006A2FAA0F770B880B990B0E94E7DE2A8DB4
:100320003B8D4C8D5D8D0E9446DF2E893F89488D27
:10033000598D0E9427E32B013C016AA17BA18CA16E
:100340009DA10E94E7DEA70196010E9446DF2A894F
:100350003B894C895D890E9427E34B015C0120E0C9
:1003600030E0A901C301B2010E94E1DE87FF04C0B1
:1003700060E070E0CB0104C060E070E080E09FE3EB
:10038000A30192010E9427E30E949CE469837A837F
:100390008B839C8320E030E0A901C501B4010E9459
:1003A000E1DE87FF04C060E070E0CB0104C060E0E4
:1003B00070E080E09FE3A50194010E9427E30E9482
:1003C0009CE46D837E838F8398872A854989BE014B
:1003D0006B5F7F4FCE0101960E9406B74B015C0117
:1003E0009B01AC010E94D3E5882321F0812F0E945C
:1003F000459354CE25E03985320380011124020D46
:10040000131D000F111F000F111F0D581F4E2E8DB1
:100410003F8D48A159A1C501B4010E9427E3D8012D
:100420006D937D938D939C9313970E945567BE8522
:10043000E985BE0FB98710E020CEEDE0F8E18491A8
:100440005F01BFEFAB1ABB0A882321F00E943E4434
:10045000F501F5CFEC85EE2369F0E3E0F8E1849156
:100460005F012FEFA21AB20A882321F00E943E44B6
:10047000F501F5CF8AE00E943E4423CFB1E0B98B6D
:10048000E3CDA5019401C501B4010E94D3E581111A
:100490000ECE2C852223F9F00E947F8C90DB3C85C8
:1004A000311141C08AE194E00E94E2CD9B01AC0190
:1004B000609122047091230480912404909125047A
:1004C0000E9426E360932204709323048093240403
:1004D0009093250429C002E094E0E92E82E0F82EF2
:1004E000DE2CD01ACE2CCF1821E041E06F2D802FCA
:1004F0000E944ED921E04FEF6F2D8D2D0E944ED9D5
:100500002FEF41E06C2D802F0E944ED92FEF4FEF3F
:100510006C2D8D2D0E944ED9FA948FEFF812E2CFF8
:100520000150E0F6B9CF1F879F859093EE10BFCDA5
:10053000E889EE2349F0F1E0FE8725E02D87198652
:100540003FEF231A330A8CCDFFEFFE872FEF2D8765
:1005500034E03987F5CFA5960FB6F894DEBF0FBE0D
:10056000CDBFDF91CF911F910F91FF90EF90DF9062
:10057000CF90BF90AF909F908F907F906F905F9043
:100580004F903F902F9008952F923F924F925F92FD
:100590006F927F928F929F92AF92BF92CF92DF9293
:1005A000EF92FF920F931F93CF93DF93CDB7DEB7F8
:1005B00062970FB6F894DEBF0FBECDBF8DE690E018
:1005C0000E94A08F8111E7C18091110583FDE3C1D5
:1005D00083E50E9469468C87811106C082E50E94EE
:1005E0006946182F8823A9F00E94F7430E946BE404
:1005F000CB010E94F94A0E94F74320E030E044EB2F
:1006000052E40E94E1DE18160CF4C2C10E943F942D
:1006100011E0E7EEF8E18491FB83EA83882369F037
:10062000082E000C990BCED34A815B814F5F5F4F40
:100630005B834A83FA018491F1CF8DE090E0C2D3CD
:100640008AE090E0BFD3EBEBF8E184919F012F5F4C
:100650003F4F3B832A83882329F00E943E44EA814E
:10066000FB81F3CF0E94C3C8112309F494C181E038
:1006700080932602109224051A821B821C821D82FE
:10068000188619861A861B8619821D863CE33E87CA
:100690004CE14F8756E4588B312C212C80E8898B14
:1006A0009FEB9A8B812C912C5401609132047091B4
:1006B0003304072E000C880B990B0E94E7DE7B01A8
:1006C0008C019B01AC01632D722D89899A890E944E
:1006D000E1DE882349F120913404309135044091C2
:1006E000360450913704AC85B701C801A1110BC085
:1006F0000E94E1DE881F8827881F89833E2C2F2CCB
:10070000098B1A8B11C00E94E1DE87FF08C080911F
:100710002602ECE5F9E18491FB83EA83E7C03E2CF5
:100720002F2C098B1A8B19820E94407A6B017C0155
:10073000DC01CB01288539854A855B85821B930BBB
:10074000A40BB50BB7FD3BC0D701C60188519C4F28
:10075000AF4FBF4F88879987AA87BB870E94934B6B
:10076000E0E6F9E184913F019FEF691A790A882355
:1007700021F00E943E44F301F5CF81149104A104BD
:10078000B104B9F0D501C401805F984DAF4FBF4FA0
:10079000BC01CD016C197D098E099F0928EE33E05B
:1007A00040E050E00E94CFE2CA01B9010E94B0448B
:1007B00003C08FE30E943E448AE00E943E440E94B0
:1007C00055670E94407A60932505709326058093B3
:1007D000270590932805A0913404AE83B091350489
:1007E000BF8300913604109137040E947B2F2E8125
:1007F0003F81A801632D722D89899A890E9426E381
:100800002B013C0120E030E0A9010E944DE587FF6B
:1008100004C077FA709477F8709481149104A1045D
:10082000B10459F420E030E040E85FE3C301B201D5
:100830000E94E1DE87FF0DC00AC020E030E040E406
:1008400050E4C301B2010E944DE5181614F44601AC
:100850005701E981EE2391F12A813B814C815D8131
:10086000211531054105510541F0D701C601821B13
:10087000930BA40BB50BB7FD21C02E813F81A801BE
:100880006D857E858F8598890E9426E320E030E083
:1008900040EC5FE30E94E1DE87FD39CFD701C6015E
:1008A000805A9541AF4FBF4F8A839B83AC83BD83F2
:1008B0009E819D87AF81AE870F87188B809126021E
:1008C000882309F424CF81149104A104B10409F40C
:1008D000ECCEB0E1CB1AB7E2DB0AE108F108C818A8
:1008E000D908EA08FB08F7FE12CFDFCE882359F0BB
:1008F000082E000C990B66D2EA81FB813196FB83AE
:10090000EA838491F3CF8DE090E05CD28AE090E0BE
:1009100059D2EBE2F9E184919F012F5F3F4F3B8376
:100920002A83882329F00E943E44EA81FB81F3CF89
:100930008091070E813041F5E7E2F9E18491FB8374
:10094000EA83882361F0082E000C990B3BD28A8140
:100950009B8101969B838A83FC018491F2CF8DE079
:1009600090E030D28AE090E02DD2EBEEF8E1849175
:100970009F012F5F3F4F3B832A83882329F00E94EA
:100980003E44EA81FB81F3CF81E08093240503C0DC
:100990000E941B943DCE62960FB6F894DEBF0FBE48
:1009A000CDBFDF91CF911F910F91FF90EF90DF901E
:1009B000CF90BF90AF909F908F907F906F905F90FF
:1009C0004F903F902F900895EF92FF920F931F93B7
:1009D000CF93DF93CDB7DEB76D970FB6F894DEBF38
:1009E0000FBECDBF8091FA09882309F483C082EC41
:1009F0009BE00E942FBF82EC9BE00E9406A9109210
:100A0000F8091092F7098091FA09882309F472C055
:100A10000091EB161091EC161AD4B801CE014C9649
:100A20002AD68C01892B09F465C06C8D7D8D6115EA
:100A3000710511F06C5F7F4F19821C8222E0A801C2
:100A4000CE0101960E9499AE811102C0F12C13C013
:100A5000CE0101966AD38823C9F361E0CE010196E5
:100A60000E940FA9009791F325EEFC0120831C82C0
:100A70000E94D8BCF82ECE0101960E942E44FF2081
:100A800009F1E6E8F8E184917F019FEFE91AF90A9C
:100A9000882321F00E943E44F701F5CFF8018191AF
:100AA0008F01882319F00E943E44F8CF8AE00E940B
:100AB0003E441092730C1092740C1092750C1092AC
:100AC000760C18C0E4E9F8E184917F019FEFE91A00
:100AD000F90A882321F00E943E44F701F5CFF8017E
:100AE00081918F01882319F00E943E44F8CF8EE255
:100AF0000E943E446D960FB6F894DEBF0FBECDBF88
:100B0000DF91CF911F910F91FF90EF9008958F92F9
:100B10009F92AF92BF92CF92DF92EF92FF921F937C
:100B2000CF93DF93C82F8BE99BE090932F0980939D
:100B30002E091092B70B82E090E0A0E0B0E0809325
:100B4000A00B9093A10BA093A20BB093A30B1092B8
:100B50002D091092290910922A0910922B0910923E
:100B60002C098FEF9FEFDC018093250990932609D4
:100B7000A0932709B0932809CC2379F1C53008F058
:100B8000F8C040E060E070E0CB010E9418BD88230F
:100B900009F4EFC020E1C29FC00111248B5E984F81
:100BA000FC01E254FE4F20812F7709F0E2C03C9611
:100BB000408151816281738144365105610571051F
:100BC00008F4D7C03497C080D180E280F380C1148C
:100BD000D104E104F10421F4CCC0C12CD12C760164
:100BE00040E0C701B6010E9418BD182F882309F400
:100BF000C0C080913007909131078115924009F073
:100C0000B8C0A0913507AA2309F4B3C06091330797
:100C1000709134076115710509F4ABC0209132075A
:100C2000222309F4A6C0A093B20B2093A40B80E06A
:100C300030E041E050E0C82FFA01082E02C0EE0F6C
:100C4000FF1F0A94E2F72E173F0739F08F5FC83075
:100C500091F789E08093AD0B8CC08093AD0B209110
:100C60003B0730913C072115310519F040E050E079
:100C700008C02091490730914A0740914B07509195
:100C80004C072093A50B3093A60B4093A70B5093D2
:100C9000A80B46015701860E971EA11CB11C80921D
:100CA000B30B9092B40BA092B50BB092B60BE0913F
:100CB0003607F0913707F093B90BE093B80BB0E02B
:100CC0000E940DE3860E971EA81EB91E8092BA0BD5
:100CD0009092BB0BA092BC0BB092BD0B85E0EE0FC7
:100CE000FF1F8A95E1F7E150FE4FEF2FFF27E695B2
:100CF0008E0E9F1EA11CB11C8092AE0B9092AF0B6A
:100D0000A092B00BB092B10B209138073091390707
:100D10002115310521F0A90160E070E008C0409183
:100D20004507509146076091470770914807D701E2
:100D3000C60188199909AA09BB09840F951FA61F26
:100D4000B71F04C0B695A79597958795CA95D2F712
:100D50008093A90B9093AA0BA093AB0BB093AC0B11
:100D6000853F2FE09207A105B10528F48CE0809320
:100D7000B70B10E01AC0853F9F4FA105B10510F4D5
:100D800080E111C08091510790915207A0915307C3
:100D9000B09154078093BA0B9093BB0BA093BC0BFC
:100DA000B093BD0B80E28093B70B812FDF91CF9181
:100DB0001F91FF90EF90DF90CF90BF90AF909F90EA
:100DC0008F900895682F82E69FE00C94AA3FCF92FF
:100DD000DF92EF92FF921F93CF93DF931092FA0965
:100DE00080912D0A882321F08AE29AE00E9406A9C8
:100DF00010929F0B10929C0B85E380939B0B0E949B
:100E0000407AEB01A89561E080919B0B0E94B0B9FC
:100E10008BE99BE00E9467AA2398229A219A209A44
:100E2000289A85E080939D0B82E58CBD1DBC1AE05D
:100E30008FEF0E946CAA1150D9F720E030E0A90191
:100E400060E08BE99BE00E9471AA182F80939E0BB3
:100E5000813049F00E94407A6C1B7D0B613D7740E8
:100E600060F381E054C02AEA31E040E050E068E0FD
:100E70008BE99BE00E9471AA82FF03C010939F0B35
:100E80000EC014E00E948D6480939E0B1150D1F728
:100E90008A3A11F082E03BC082E080939F0B809100
:100EA0009F0B823021F0C12CD12C760105C0C12CC2
:100EB000D12CE12C80E4F82E20E030E0A90167E39A
:100EC0008BE99BE00E9471AAA701960169E28BE978
:100ED0009BE00E9471AA80939E0B882349F00E9498
:100EE000407A6C1B7D0B613D774030F38AE00FC088
:100EF00080919F0B823011F520E030E0A9016AE378
:100F00008BE99BE00E9471AA882351F088E08093CE
:100F10009C0B8BE99BE00E9467AAE5EBFAE119C004
:100F20000E948D64807C803C19F483E080939F0B49
:100F30000E948D640E948D640E948D648BE99BE009
:100F40000E9467AA10929D0B81E0E1DD811131C002
:100F500015C08491EF012196882321F00E943E4420
:100F6000FE01F7CFE7EAFAE18491EF0121968823A9
:100F700009F456C00E943E44FE01F6CF80E0C7DD72
:100F8000811117C0E0EAFAE18491EF0121968823EC
:100F900021F00E943E44FE01F7CFECE8FAE1849193
:100FA000EF012196882309F43BC00E943E44FE01D4
:100FB000F6CF60EA7BE08AE29AE00E94B3A8811152
:100FC00016C0E0EAFAE18491EF012196882321F02E
:100FD0000E943E44FE01F7CFEBE7FAE18491EF0176
:100FE00021968823E9F00E943E44FE01F7CF81E07C
:100FF0008093FA09E5EBFAE18491EF0121968823C9
:1010000021F00E943E44FE01F7CFEFE6FAE1849121
:10101000EF012196882321F00E943E44FE01F7CF84
:101020008BE1EAE2FAE0A9E4BAE001900D928A9538
:10103000E1F78091280A9091290A9093480A8093B9
:10104000470ADF91CF911F91FF90EF90DF90CF90F3
:1010500008958091070E823039F48AE59AE19093E1
:10106000240780932307D6D70E94407A60930B0E03
:1010700070930C0E80930D0E90930E0E8091FA09D2
:10108000882319F081E08093F90981E08093070EAD
:101090000895CF93DF931092F90983E08093070EB0
:1010A0008091540E8823F9F0E9E1FAE18491EF018F
:1010B000882341F0082E000C990B84DE2196FE0156
:1010C0008491F6CF8DE090E07DDE8AE090E07ADEDC
:1010D000EFEEF9E18491EF012196882319F10E9446
:1010E0003E44FE01F7CFE6E5FAE18491EF01882363
:1010F00041F0082E000C990B65DE2196FE018491CB
:10110000F6CF8DE090E05EDE8AE090E05BDEEDE120
:10111000FAE18491EF012196882321F00E943E4458
:10112000FE01F7CFDF91CF9108958F929F92AF92FA
:10113000BF92CF92DF92EF92FF920F931F93CF93C4
:10114000DF9300D01F92CDB7DEB7FC0183818130E1
:1011500079F5818181FF2CC081899289A389B48925
:10116000892B8A2B8B2B09F448C07F0140E050E08B
:10117000BA01CF010E941CA88823D1F0F70185880D
:101180009688A788B08CC18CD28C82E090E0A0E0D9
:10119000B0E0F60180839183A283B3839E012F5F29
:1011A0003F4FB501A401C6010E94E1BD811102C0FB
:1011B00080E03CC000E010E09801B501A401C60148
:1011C0000E9450BD8823A1F389809A80AB80BC80A7
:1011D000F6018789803141F4F8EF8F16FFEF9F0603
:1011E000A104B10460F4DACF88EF88168FEF980677
:1011F000A8068FE0B80618F4D1CF81E017C0F70138
:10120000158A168A178A108E118A128A138A148AEE
:10121000818180688183C7010E942FBF882341F2AA
:1012200040E050E0BA01C7010E941CA80F900F9047
:101230000F900F90DF91CF911F910F91FF90EF9042
:10124000DF90CF90BF90AF909F908F9008951092B5
:10125000FC091092F9098091C50B882321F082ECDA
:101260009BE00C9406A908952F923F924F925F92B3
:101270006F927F928F929F92AF92BF92CF92DF92A6
:10128000EF92FF920F931F93CF93DF93CDB7DEB70B
:10129000C257D1090FB6F894DEBF0FBECDBF8C0187
:1012A0003B014A014DB75EB7E1965FAF4EAFE197A4
:1012B000AD961FAEAD971B0154E0250E311C7E018B
:1012C0008FE5E80EF11C99EF492E92E0592EE0E4EB
:1012D000F0E0EC0FFD1F3496E396FFAFEEAFE3971F
:1012E000F3018781823008F462C184859585A685E3
:1012F000B7858F719927AA27BB27892B8A2B8B2B20
:1013000009F055C110920A0A4AE05AE0BE016F5F27
:101310007F4FC1010E94C7BE18160CF048C18C85D2
:10132000982F9871903129F42091770C2150223018
:1013300078F42981222309F43AC1253E89F22E321C
:1013400079F220910A0A2E3259F28A7049F6B8C011
:101350004DB75EB7AF965FAF4EAFAF97BE016F5F51
:101360007F4FC7010E94C2BC0115110521F0F80191
:10137000808181119BC021E081E090E0F701019024
:101380000020E9F73197EE19FF098E0F9F1F029693
:101390004DB75EB7481B590B0FB6F8945EBF0FBE32
:1013A0004DBF8DB79EB701965C01211102C0B801F7
:1013B00002C062E373E0C5010E9485E6B701C50182
:1013C0000E9466E662E373E0C5010E9466E6259628
:1013D0001FAE259728961FAE289724961FAE1EAEE7
:1013E000249722965FAE4EAE229721E0A701B1016D
:1013F000E3968EAD9FADE3970E9499AE81112AC00E
:101400008091770C811126C0E5EBFAE184916F01A0
:101410009FEFC91AD90A882321F00E943E44F601A1
:10142000F5CFEBEDF9E184916F012FEFC21AD20AEB
:10143000882321F00E943E44F601F5CF6701F601B2
:1014400081916F01882319F00E943E44F8CF8AE011
:101450000E943E448BE1FE01EC5BFF4FDE0195965E
:1014600001900D928A95E1F724968EAD9FAD249759
:101470009CA38BA35AA249A240E050E0BE016F5D3D
:101480007F4FC501F1DECE0181960E94E066CE015C
:10149000805C9F4F0E94E066AF964EAD5FADAF9708
:1014A0000FB6F8945EBF0FBE4DBF1ACFF801019082
:1014B0000020E9F73197CF01801B910B20E05ECF30
:1014C00081E0903109F080E08093FB09903141F098
:1014D0008985873409F004CF8A858E3709F400CFD7
:1014E0008091770C813029F08230D9F18111F8CECA
:1014F0000AC08091780C9091790C01969093790CA8
:101500008093780CEDCEBE016F5F7F4F8DEF99E039
:101510000E94C2BC0115110529F48DEFC82E89E087
:10152000D82E09C06801F60181916F018823A9F3C3
:101530000E943E44F8CFF60181916F01882319F093
:101540000E943E44F8CF80E20E943E446D8D7E8D25
:101550008F8D98A14AE00E9445448AE00E943E4453
:10156000BFCEBE016F5F7F4F8DEF99E00E94C2BC7E
:101570008114910441F06DEF79E0C4010E9453E6BB
:10158000892B69F414C0AD96FFADAD978F2F90E015
:101590002091840F3091850F8217930741F0AD960B
:1015A0002FADAD972F5FAD962FAFAD9799CEE1964A
:1015B0008EAD9FADE1970FB6F8949EBF0FBE8DBF65
:1015C000CE58DF4F0FB6F894DEBF0FBECDBFDF9110
:1015D000CF911F910F91FF90EF90DF90CF90BF9030
:1015E000AF909F908F907F906F905F904F903F90C3
:1015F0002F9008950F931F93CF93DF93CDB7DEB74E
:101600006F970FB6F894DEBF0FBECDBF8B0122E0FF
:101610002093770C9093850F8093840F89E49AE050
:101620000E9463AA8BE1E9E4FAE0DE0115960190DD
:101630000D928A95E1F78091470A9091480A9C8320
:101640008B8389EF92E09A838983A801BE016F5F43
:101650007F4F80E090E008DECE0101960E94E066B8
:101660006F960FB6F894DEBF0FBECDBFDF91CF915E
:101670001F910F9108952F923F924F925F926F9218
:101680007F928F929F92AF92BF92CF92DF92EF9212
:10169000FF920F931F93CF93DF93CDB7DEB76F9772
:1016A0000FB6F894DEBF0FBECDBF6C012DB63EB6AF
:1016B0001D8218861C821B8289EF92E09A8389839F
:1016C000FB0180819E012F5F3F4F39018F3241F036
:1016D00085E49AE0F60191838083F62E172F64C08B
:1016E00086E29AE0F601918380838B010F5F1F4FA2
:1016F0000115110509F456C04DB65EB66FE270E0F3
:10170000C8010E9471E64C010817190708F048C08B
:101710007C01E01AF10AFF24C70101962DB73EB7FC
:10172000281B390B0FB6F8943EBF0FBE2DBF8DB7E7
:101730009EB701965C01A701B8010E949AE6F501E7
:10174000EE0DFF1D1082F60160817181611571053A
:1017500011F06C5F7F4F21E0A501CE0105960E943C
:1017600099AE811111C0B50187EC99E10E94A8C81A
:101770008EE20E943E448AE00E943E440FB6F894F6
:101780005EBE0FBE4DBE0EC0F60171826082840146
:101790000F5F1F4F0FB6F8945EBE0FBE4DBEA8CFB1
:1017A000F02E02C0F12C10E0C3010E94E0668F2DE4
:1017B000912F0FB6F8943EBE0FBE2DBE6F960FB69A
:1017C000F894DEBF0FBECDBFDF91CF911F910F9177
:1017D000FF90EF90DF90CF90BF90AF909F908F9051
:1017E0007F906F905F904F903F902F9008959091D1
:1017F000F510E92FF0E0EC56FA4F80839F5F9430AC
:1018000018F49093F51002C01092F5108091F61024
:101810008F5F8093F6100895CF92DF92EF920F932F
:101820001F93CF93DF93CDB7DEB760970FB6F894D1
:10183000DEBF0FBECDBFE0902305EAE1F4E0808576
:101840009185A285B3854481558166817781008128
:1018500011812281338109831A832B833C834D8339
:101860005E836F83788789879A87AB87BC871D865D
:101870001E861F86188AAE01475F5F4FBE016B5FF1
:101880007F4FCE0101960E943EC2CE010D966C01A3
:101890000CE312E026E234E0AE01475F5F4FBE0189
:1018A0006B5F7F4F0C970E945C5460960FB6F89464
:1018B000DEBF0FBECDBFDF91CF911F910F91EF9093
:1018C000DF90CF900895CF93FC0120812B33A1F0BE
:1018D0002091F610243080F4C62FBC018091F510C1
:1018E000F0E68F9FC001112487569A4F0E9485E62B
:1018F0008C2F7DDF81E001C080E0CF9108958F9231
:101900009F92AF92BF92CF92DF92EF92FF920F938E
:101910001F93CF93DF93E6EFFCE18491EF012196D3
:10192000882321F00E943E44FE01F7CFC12CD12C28
:101930007601C0E080E20E943E44CF5FC630D1F71E
:10194000C701B6010E94B0448FEFC81AD80AE80A4E
:10195000F80A95E0C916D104E104F10451F78AE0D0
:101960000E943E4403E710E1C12CD12C760180E2B5
:101970000E943E44C701B6010E94B044C0E0D0E0DE
:1019800080E20E943E44F801EC0FFD1F80809180B0
:10199000A280B380A5019401C501B4010E94D3E5E2
:1019A000811112C020E030E0A901C501B4010E94FC
:1019B0004DE587FD03C08BE20E943E4443E0C50134
:1019C000B4010E94CA4409C0B12C80E20E943E4486
:1019D000B3948DE396E0B912F9CF6496C436D1057D
:1019E00079F68AE00E943E448FEFC81AD80AE80AC6
:1019F000F80A0C5F1F4F95E0C916D104E104F10409
:101A000009F0B5CF8AE0DF91CF911F910F91FF9040
:101A1000EF90DF90CF90BF90AF909F908F900C94FD
:101A20003E44BC0186ED99E00E9420C767E771E063
:101A300080E090E00C94EB531F93CF93DF938823C7
:101A400029F0649908C08AE090E002C08AE590E03D
:101A5000E8DF10E04DC080EA90E0E3DF8AE090E04C
:101A6000E0DF8AE590E0DDDF6CED75E080E090E09E
:101A70000E94EB53649BE7CFE0EAFAE18491EF0127
:101A80002196882321F00E943E44FE01F7CFECEB23
:101A9000FCE18491EF012196882321F00E943E44CD
:101AA000FE01F7CF0E94B94C109103021123F9F007
:101AB000E0EAFAE18491EF012196882321F00E9467
:101AC0003E44FE01F7CFE5E4FCE18491EF0121966D
:101AD000882321F00E943E44FE01F7CF6EE571E0BD
:101AE00080E090E00E94EB531092030201C011E0ED
:101AF000812FDF91CF911F9108958091EF0F9091E9
:101B0000F00FA091F10FB091F20F80933C029093EF
:101B10003D02A0933E02B0933F028091ED0F909161
:101B2000EE0F9093010280930002089580913C0291
:101B300090913D02A0913E02B0913F028093EF0F41
:101B40009093F00FA093F10FB093F20F80910002E9
:101B5000909101029093EE0F8093ED0F84E690E058
:101B6000909301028093000208952F923F924F922A
:101B70005F926F927F928F929F92AF92BF92CF921D
:101B8000DF92EF92FF920F931F93CF93DF93CDB726
:101B9000DEB72A970FB6F894DEBF0FBECDBF2B017C
:101BA0003C012D833E834F83588747015801DA86D5
:101BB000C98680913C0290913D02A0913E02B09175
:101BC0003F0289839A83AB83BC83D6011C91119613
:101BD0000C91119712963C90129713962C9020E03E
:101BE00030E0A901612F702F832D922D0E94E1DE3C
:101BF00081110AC0E7E1F5E185919591A591B49134
:101C0000182F092F3A2E2B2EA50194016091220442
